:1000000000000320D55D0100B95D0100715D0100B4
:10001000715D0100715D0100715D0100715D0100A4
:10002000715D0100715D0100715D0100B95D01004C
:10003000B95D0100715D01008D520100055501009F
:10004000B95D0100B95D0100B95D0100B95D010054
:10005000B95D0100B95D0100B95D0100B95D010044
:10006000B95D0100B95D0100B95D0100B95D010034
:10007000B95D0100B95D0100B95D0100B95D010024
:10008000B95D0100B95D0100B95D0100B95D010014
:10009000B95D0100B95D0100B95D0100B95D010004
:1000A00089130100E5140100B95D0100B95D01008B
:1000B000B95D0100B95D0100B95D01002970010061
:1000C000B95D010051920100B95D0100AD930100DD
:1000D000B95D0100DD940100B95D0100B95D010069
:1000E000B95D0100B95D0100B95D0100B95D0100B4
:1000F000B95D0100B95D0100B95D0100B95D0100A4
:10010000B95D0100B95D0100B95D0100B95D010093
:10011000B95D010015730100B95D0100B95D010011
:10012000B95D0100B95D0100B95D0100B95D010073
:10013000B95D0100B95D0100B95D0100B95D010063
:10014000D94F0100B95D01000D960100B95D0100B4
:10015000B95D0100B95D0100B95D0100B95D010043
:10016000B95D0100B95D010041160100B95D0100F2
:10017000B95D0100B95D0100B95D0100B95D010023
:10018000B95D010099F90000B95D0100B95D010098
:10019000B95D0100B95D01003D970100B95D010045
:1001A000B95D0100B95D0100B95D0100B95D0100F3
:1001B000B95D0100B95D0100B95D0100B95D0100E3
:1001C000B95D0100B95D0100B95D0100B95D0100D3
:1001D000FFFFFFFFFFFFFFFFFFFFFFFFFFFFFFFF2F
:10040000FFFFFFFFFFFFFFFFFFFFFFFFDEF9FFFF23
:1004100010B5054C237833B9044B13B10448AFF33E
:1004200000800123237010BD00B0FF1F00000000FA
:10043000C4060F00084B10B51BB108490848AFF3BC
:1004400000800848036803B910BD074B002BFBD0A0
:10045000BDE81040184700BF0000000004B0FF1FB7
:10046000C4060F0050A2FF1F0000000049F2F8234D
:10047000C1F6FF731B7C022B9DBF41F2B462C0F238
:10048000020252F823000020704700BF49F2F8230F
:10049000C1F6FF735B7C032B9DBF41F2C862C0F2C3
:1004A000020252F823000020704700BF49F2F823EF
:1004B000C1F6FF7349F2A422987C49F2B023C1F639
:1004C000FF72C1F6FF7300280CBF10461846704734
:1004D00049F2F823C1F6FF7393F822306BB149F269
:1004E0002C33C1F6FF7346F64F62C0F2200249F288
:1004F0002C301A60C1F6FF70704749F22C33C1F6F8
:10050000FF7346F24F62C0F2660249F22C301A6065
:10051000C1F6FF70704700BF704700BF704700BF53
:10052000704700BF704700BF08B549F2F823C1F615
:10053000FF73DA7C72B140F2201149F22030C0F230
:100540000201C1F6FF701CF0A3FB49F22030C1F696
:10055000FF7008BD40F2141149F22030C0F20201D0
:10056000C1F6FF701CF094FB49F22030C1F6FF7019
:1005700008BD00BF10B549F2F823C1F6FF73B2EE13
:10058000047A1B7D07EE903AF8EE677A49F2BC24B4
:10059000C7EE876AC1F6FF7416EE900A1BF0A0F84A
:1005A0000B4640F22C110246C0F2020120461CF01C
:1005B0006FFB204610BD00BF10B549F2F823C1F60D
:1005C000FF73B2EE047A5B7D07EE903AF8EE677A3D
:1005D00049F23834C7EE876AC1F6FF7416EE900A06
:1005E0001BF07EF80B4640F22C110246C0F20201CD
:1005F00020461CF04DFB204610BD00BF10B549F24F
:10060000F823C1F6FF7349F24434C1F6FF7440F297
:10061000381193F90A202046C0F202011CF038FB81
:10062000204610BD10B5044614F058FC204610BDFD
:1006300008B549F2F823C1F6FF7393F8212072B18F
:1006400040F24C1149F2C420C0F20201C1F6FF7021
:100650001CF01EFB49F2C420C1F6FF7008BD40F239
:100660004413C0F2020393E8030049F2C423C1F625
:10067000FF731860197149F2C420C1F6FF7008BDFC
:1006800000F0F703F52B06D0F92804D0EF2803D8A3
:1006900000F0F00070470020704700BF38B549F205
:1006A000E464C1F6FF74014600230A22204615F0D7
:1006B00031F80546204615F01BF8284438BD00BF28
:1006C00010B504461CF01CFB01462046BDE8104056
:1006D00018F0C2BB10B504461CF012FB01462046C0
:1006E00018F0BAFB044649F2E460C1F6FF7014F05A
:1006F000FFFF204410BD00BF40F2541070B5C0F29F
:100700000200FFF7E7FF40F27810C0F202004DF25E
:10071000E034FFF7DFFFC2F200044CF69031C2F282
:100720000001204611F092FF40F27C10C0F202005E
:100730004DF21806FFF7CEFFC1F6FF764CF2982374
:10074000C2F2000340F2801049F2F8257268DA70B4
:10075000C1F6FF75C0F20200FFF7BCFF40F2841043
:100760006B7E7360C0F20200FFF7B4FF44F27013B7
:10077000C2F20003002114206A7E986383F83C10C3
:10078000596372B68242A8BF02469200DA6262B62C
:1007900040F28810C0F20200FFF79CFF204611F0E3
:1007A000A1FF40F28C10C0F20200BDE87040FFF7DC
:1007B00091BF00BF40F2901008B5C0F202001621B0
:1007C00018F04AFB49F2F823C1F6FF7393F8223080
:1007D000E3B14DF65053C1F6FF73F621986C0368F0
:1007E000DB6C984740F2A810C0F20200FFF768FFE8
:1007F0004DF66060C2F200004FF20F6113F016FE7A
:1008000040F2B810C0F20200FFF75AFF49F2E4606C
:10081000C1F6FF70BDE8084014F06ABF40F2D01086
:1008200010B51621C0F2020018F016FB49F2E46080
:10083000C1F6FF704DF2E03414F05AFFC2F200042A
:100840004CF290712046C2F2000111F0FFFE4DF211
:100850001802C1F6FF724CF29823C2F200035268EC
:100860001A702046BDE8104011F03CBF38B5044670
:1008700040F2E8100D46C0F202000D2118F0ECFA2B
:1008800049F2F823C1F6FF7393F822300BB32B041F
:1008900003F4FE03013C43F45043240243F00D03F0
:1008A00004F470641C434DF660602146C2F20000FF
:1008B00013F0BCFD40F2B810C0F20200FFF700FFD9
:1008C000204617F03FFC40F2F810C0F20200FFF79C
:1008D000F7FE49F2E460C1F6FF70BDE8384014F05D
:1008E00007BF00BF38B5044640F208200D46C0F2ED
:1008F00002000D2118F0B0FA49F2F823C1F6FF7397
:1009000093F822300BB32B0403F4FE03013C43F4B1
:100910004043240243F00C0304F470641C434DF67E
:1009200060602146C2F2000013F080FD40F2B81072
:10093000C0F20200FFF7C4FE204617F003FC40F2AD
:10094000F810C0F20200FFF7BBFE49F2E460C1F606
:10095000FF70BDE8384014F0CBBE00BF70B506464E
:1009600040F218200C46C0F202001221154618F081
:1009700073FA49F2F823C1F6FF7393F822303BB9BA
:1009800049F2E460C1F6FF70BDE8704014F0B0BEFB
:100990006B1E1B02240404F4FE0403F4706323435F
:1009A00043F45043340143F00D03E4B21C434DF6CD
:1009B0006060C2F20000214613F038FD40F2B8102A
:1009C000C0F20200FFF77CFE6EB140F2F810C0F2F8
:1009D0000200FFF775FE49F2E460C1F6FF70BDE862
:1009E000704014F085BE204617F0ACFBEDE700BF69
:1009F00038B5044640F22C20C0F202001A2118F04B
:100A00002BFA49F2F823C1F6FF7393F822301BB397
:100A10004DF65055C1F6FF75F321A86C03681B68AD
:100A20009847A86C036804F07F01DB6C984740F29C
:100A3000A810C0F20200FFF743FE200400F4FE00FD
:100A400040F4734040F0020017F07CFB40F2F810D5
:100A5000C0F20200FFF734FE49F2E460C1F6FF7015
:100A6000BDE8384014F044BE38B5054640F2482091
:100A70000C46C0F202000D2118F0EEF949F2F823FD
:100A8000C1F6FF7393F822304BB304F30D0404F561
:100A900000536C1E1A04240202F4FE0204F4706473
:100AA000144344F460445B0403F0FE4344F00E043A
:100AB0001C434DF660602146C2F2000013F0B6FC04
:100AC00040F2B810C0F20200FFF7FAFD204617F01E
:100AD00039FB40F2F810C0F20200FFF7F1FD49F2D5
:100AE000E460C1F6FF70BDE8384014F001BE00BFFD
:100AF00038B5044640F25820C0F20200242118F014
:100B0000ABF949F2F823C1F6FF7393F822301BB317
:100B10004DF65055C1F6FF75F121A86C03681B68AE
:100B20009847A86C036821461B68984740F2A810B4
:100B3000C0F20200FFF7C4FD04F00F044FF20210F0
:100B40002404C0F21000204317F0FCFA40F2F81021
:100B5000C0F20200FFF7B4FD49F2E460C1F6FF7095
:100B6000BDE8384014F0C4BD38B5044640F28020DA
:100B7000C0F20200152118F06FF949F2F823C1F60E
:100B8000FF7393F822303BB34DF65055C1F6FF7515
:100B9000F321A86C03681B689847A86C036804F0ED
:100BA0007F01DB6C984740F2A810C0F20200FFF70B
:100BB00087FD210401F4FE0141F473414DF66060AC
:100BC000C2F2000041F0020113F030FC40F2B81014
:100BD000C0F20200FFF774FD49F2E460C1F6FF7055
:100BE000BDE8384014F084BD38B5044640F2982082
:100BF000C0F202001F2118F02FF949F2F823C1F6C4
:100C0000FF7393F822303BB34DF65055C1F6FF7594
:100C1000F121A86C03681B689847A86C03682146FB
:100C20001B68984740F2A810C0F20200FFF748FD89
:100C300004F00F044FF202112404C0F210014DF62B
:100C40006060C2F20000214313F0F0FB40F2B810E4
:100C5000C0F20200FFF734FD49F2E460C1F6FF7014
:100C6000BDE8384014F044BD10B540F2B8204CF255
:100C70009824C2F200042A21C0F2020018F0ECF815
:100C800049F2E46094F90310C1F6FF7014F0D2FC4D
:100C900049F2E460C1F6FF7014F02AFD4EF2C8710B
:100CA0004DF2E030C2F20001C2F2000011F0CEFCC1
:100CB0004DF2E0300221C2F2000011F0EFFC4DF2E3
:100CC0001801C1F6FF7194F903204B682370002AC4
:100CD00044F27013C2F2000315DB12240020A2427A
:100CE0004A609C6383F83C005863D4BF920048225A
:100CF00072B6DA6262B64DF2E030C2F20000BDE8D0
:100D0000104011F0EFBC00221220986383F83C20C1
:100D10005A63E2704A6072B6DA6262B64DF2E0304F
:100D2000C2F20000012111F0B3FCE4E738B505463A
:100D300049F2E46440F2E420C1F6FF741E21C0F2DF
:100D4000020018F089F8294600230A22204614F0F0
:100D5000E1FC40F204300E21C0F2020018F07CF8F1
:100D600049F2F823C1F6FF730A2293F821102046B6
:100D7000002314F0CFFC40F214300121C0F2020035
:100D800018F06AF8204614F0B3FC002038BD00BF0C
:100D9000F8B549F2F824C1F6FF740F4694F82130F3
:100DA0001646054623B1984202D0FFF7BFFF50B167
:100DB0004BF2CC13C2F2000394F9091018683944BD
:100DC00000220BF01FFE40F21830C0F20200122188
:100DD00018F042F894F822302BB3330603F0FE43A8
:100DE00043F400433F04013D43F0080307F4FE07CA
:100DF0002D023B4305F470651D434DF660602946A6
:100E0000C2F2000013F012FB40F2B810C0F2020070
:100E1000FFF756FC284617F095F940F2F810C0F29B
:100E20000200FFF74DFC49F2E460C1F6FF70BDE837
:100E3000F84014F05DBC00BFF8B549F2F824C1F6E3
:100E4000FF740F4694F821301646054623B19842A8
:100E500002D0FFF76BFF50B14BF2CC13C2F200038C
:100E600094F909101868394432460BF0CBFD40F272
:100E70002C30C0F20200112117F0EEFF94F822305E
:100E80002BB3360606F0FE4646F410463F04013DFD
:100E900046F0090607F4FE072D023E4305F470658F
:100EA00035434DF660602946C2F2000013F0BEFAE9
:100EB00040F2B810C0F20200FFF702FC284617F01B
:100EC00041F940F2F810C0F20200FFF7F9FB49F2D5
:100ED000E460C1F6FF70BDE8F84014F009BC00BF43
:100EE000F8B549F2F826C1F6FF760F4696F821309C
:100EF0001546044623B1984202D0FFF717FF48B1C8
:100F00004BF2CC13C2F200032A4618680368394634
:100F10005B68984740F24030C0F202000D2117F0A4
:100F20009BFF96F822302BB32D0605F0FE4545F4C5
:100F300030453F04013C45F00B0507F4FE07240251
:100F40003D4304F470642C434DF660602146C2F2C8
:100F5000000013F06BFA40F2B810C0F20200FFF785
:100F6000AFFB204617F0EEF840F2F810C0F2020096
:100F7000FFF7A6FB49F2E460C1F6FF70BDE8F84058
:100F800014F0B6BB40F2503038B51B21C0F202005D
:100F900017F062FF49F2E460C1F6FF704DF2E034F1
:100FA00014F0A6FBC2F200044CF220412046C2F22B
:100FB000000111F04BFB4DF21801C1F6FF7149F22F
:100FC000F8224CF29820C2F20000C1F6FF7244F2FF
:100FD0007013C2F200034D68C570127C4A60002095
:100FE00002259D6383F83C00586372B6AA42A8BFED
:100FF0002A46AA40DA6262B62046BDE8384011F0BF
:1010000071BB00BF40F26C3038B51E21C0F2020047
:1010100017F022FF49F2E460C1F6FF704DF2E034B0
:1010200014F066FBC2F200044CF258212046C2F2D2
:10103000000111F00BFB4DF21801C1F6FF7149F2EE
:10104000F8224CF29820C2F20000C1F6FF7244F27E
:101050007013C2F200034D68C570127E4A60002012
:1010600063259D6383F83C00586372B6AA42A8BF0B
:101070002A469200DA6262B62046BDE8384011F096
:1010800031BB00BF40F28C3038B51921C0F20200EC
:1010900017F0E2FE49F2E460C1F6FF704DF2E03471
:1010A00014F026FBC2F200044CF62C112046C1F6C7
:1010B000FF7111F0CBFA4DF21801C1F6FF7149F240
:1010C000F8224CF29820C2F20000C1F6FF7244F2FE
:1010D0007013C2F200034D68857052794A60002097
:1010E00063259D6383F83C00586372B6AA42A8BF8B
:1010F0002A469200DA6262B62046BDE8384011F016
:10110000F1BA00BF40F2A83038B52021C0F2020089
:1011100017F0A2FE49F2E460C1F6FF704DF2E03430
:1011200014F0E6FAC2F200044DF24C012046C2F27D
:10113000000111F08BFA4DF21801C1F6FF7149F26E
:10114000F8224CF29820C2F20000C1F6FF7244F27D
:101150007013C2F200034D68C570D27D4A60002052
:1011600063259D6383F83C00586372B6AA42A8BF0A
:101170002A469200DA6262B62046BDE8384011F095
:10118000B1BA00BF40F2CC3038B52021C0F2020025
:1011900017F062FE49F2E460C1F6FF704DF2E034F0
:1011A00014F0A6FAC2F200044DF20C012046C2F27D
:1011B000000111F04BFA4DF21801C1F6FF7149F22E
:1011C000F8224CF29820C2F20000C1F6FF7244F2FD
:1011D0007013C2F200034D68C570927B4A60002014
:1011E00063259D6383F83C00586372B6AA42A8BF8A
:1011F0002A469200DA6262B62046BDE8384011F015
:1012000071BA00BF40F2F03038B52421C0F20200BC
:1012100017F022FE49F2E460C1F6FF704DF2E034AF
:1012200014F066FAC2F200044BF2D0312046C2F24A
:10123000000111F00BFA4DF21801C1F6FF7149F2ED
:10124000F8224CF29820C2F20000C1F6FF7244F27C
:101250007013C2F200034D68C570527B4A600020D3
:1012600063259D6383F83C00586372B6AA42A8BF09
:101270002A469200DA6262B62046BDE8384011F094
:1012800031BA00BF40F2184038B51E21C0F202004A
:1012900017F0E2FD49F2E460C1F6FF704DF2E03470
:1012A00014F026FAC2F200044DF654412046C1F66D
:1012B000FF7111F0CBF94DF21801C1F6FF7149F23F
:1012C000F8224CF29820C2F20000C1F6FF7244F2FC
:1012D0007013C2F200034D68C570927E4A60002010
:1012E00014259D6383F83C00586372B6AA42A8BFD8
:1012F0002A469200DA6262B62046BDE8384011F014
:10130000F1B900BF40F2384038B51C21C0F20200EC
:1013100017F0A2FD49F2E460C1F6FF704DF2E0342F
:1013200014F0E6F9C2F200044BF694212046C1F60F
:10133000FF7111F08BF94DF21801C1F6FF7149F2FE
:10134000F8224CF29820C2F20000C1F6FF7244F27B
:101350007013C2F200034D68C570927C4A60002091
:1013600001259D6383F83C00586372B69200DA62EF
:1013700062B62046BDE8384011F0B4B940F258409A
:1013800038B52121C0F2020017F066FD49F2E46091
:10139000C1F6FF704DF2E03414F0AAF9C2F2000475
:1013A0004DF62C212046C2F2000111F04FF94DF20A
:1013B0001801C1F6FF7149F2F8224CF29820C2F2EE
:1013C0000000C1F6FF7244F27013C2F200034D68D0
:1013D000C570927D4A60002063259D6383F83C00C0
:1013E000586372B6AA42A8BF2A469200DA6262B671
:1013F0002046BDE8384011F075B900BF40F27C408E
:1014000038B51721C0F2020017F026FD49F2E4605A
:10141000C1F6FF704DF2E03414F06AF9C2F2000434
:101420004BF6E8312046C2F2000111F00FF94DF2FF
:101430001801C1F6FF7149F2F8224CF29820C2F26D
:101440000000C1F6FF7244F27013C2F200034D684F
:10145000857012794A60002063259D6383F83C0003
:10146000586372B6AA42A8BF2A469200DA6262B6F0
:101470002046BDE8384011F035B900BF40F2944035
:1014800038B52121C0F2020017F0E6FC49F2E46011
:10149000C1F6FF704DF2E03414F02AF9C2F20004F4
:1014A0004CF654612046C2F2000111F0CFF84DF223
:1014B0001801C1F6FF7149F2F8224CF29820C2F2ED
:1014C0000000C1F6FF7244F27013C2F200034D68CF
:1014D000C570527F4A60002063259D6383F83C00FD
:1014E000586372B6AA42A8BF2A469200DA6262B670
:1014F0002046BDE8384011F0F5B800BF40F2B840D2
:10150000F8B51B21C0F2020017F0A6FC49F2E46016
:10151000C1F6FF704DF2E03414F0EAF8C2F20004B4
:101520004DF610012046C2F2000111F08FF849F289
:10153000F823C1F6FF734DF21801C1F6FF7193F95C
:1015400009304F684B604CF2982044F27012C2F29E
:1015500000026FF01701C2F20000002618258B422E
:101560008770B8BF0B46516382F83C60956372B6D2
:10157000AB42A8BF2B469B00D36262B62046BDE8B3
:10158000F84011F0AFB800BF40F2D440F8B51B21CD
:10159000C0F2020017F060FC49F2E460C1F6FF708F
:1015A0004DF2E03414F0A4F8C2F200044AF6883197
:1015B0002046C2F2000111F049F849F2F823C1F6C1
:1015C000FF734DF21801C1F6FF7193F91F304F6898
:1015D0004B604CF2982044F27012C2F200026FF09D
:1015E0003101C2F20000002632258B42C770B8BF1D
:1015F0000B46516382F83C60956372B6AB42A8BF5C
:101600002B469B00D36262B62046BDE8F84011F03D
:1016100069B800BF40F2F04038B51A21C0F20200AC
:1016200017F01AFC49F2E460C1F6FF704DF2E034A5
:1016300014F05EF8C2F200044DF690612046C1F647
:10164000FF7111F003F84DF21801C1F6FF7149F274
:10165000F8224CF29820C2F20000C1F6FF7244F268
:101660007013C2F200034D68857092794A600020C1
:1016700063259D6383F83C00586372B6AA42A8BFF5
:101680002A469200DA6262B62046BDE8384011F080
:1016900029B800BF40F20C5038B51E21C0F202003C
:1016A00017F0DAFB49F2E460C1F6FF704DF2E03466
:1016B00014F01EF8C2F200044DF260312046C2F26E
:1016C000000110F0C3FF4DF21801C1F6FF7149F29D
:1016D000F8224CF29820C2F20000C1F6FF7244F2E8
:1016E0007013C2F200034D68457192F821204A60E0
:1016F000002010259D6383F83C00586372B6AA420F
:10170000A8BF2A469200DA6262B62046BDE8384099
:1017100010F0E8BF40F22C5038B51821C0F202009A
:1017200017F09AFB49F2E460C1F6FF704DF2E03425
:1017300013F0DEFFC2F200044DF638012046C1F678
:10174000FF7110F083FF4DF21801C1F6FF7149F2ED
:10175000F8224CF29820C2F20000C1F6FF7244F267
:101760007013C2F200034D688570D27A4A6000207F
:1017700063259D6383F83C00586372B6AA42A8BFF4
:101780002A469200DA6262B62046BDE8384010F080
:10179000A9BF00BF40F2485070B51821C0F2020046
:1017A00017F05AFB49F2E460C1F6FF704DF2E034E5
:1017B00013F09EFFC2F200044CF2C4212046C2F294
:1017C000000110F043FF49F2F823C1F6FF734DF218
:1017D0001801C1F6FF714CF2982044F27012C2F267
:1017E000000293F908304E684B60C2F200000021FD
:1017F000632523EAE3738670956382F83C10516396
:1018000072B6AB42A8BF2B469B00D36262B620469D
:10181000BDE8704010F066BF40F26450F8B5162184
:10182000C0F2020017F018FB49F2E460C1F6FF7045
:101830004DF2E03413F05CFFC2F200044BF23C4185
:101840002046C1F6FF7110F001FF49F2F823C1F6FE
:10185000FF734DF21801C1F6FF7193F90A304F681A
:101860004B604CF2982044F27012C2F200026FF00A
:101870003101C2F20000002632258B428770B8BFCA
:101880000B46516382F83C60956372B6AB42A8BFC9
:101890002B469B00D36262B62046BDE8F84010F0AC
:1018A00021BF00BF40F27C5038B52021C0F20200B9
:1018B00017F0D2FA49F2E460C1F6FF704DF2E0345D
:1018C00013F016FFC2F200044DF6D8012046C2F212
:1018D000000110F0BBFE4DF21801C1F6FF7149F294
:1018E000F8224CF29820C2F20000C1F6FF7244F2D6
:1018F0007013C2F200034D688570127B4A600020AD
:1019000063259D6383F83C00586372B6AA42A8BF62
:101910002A469200DA6262B62046BDE8384010F0EE
:10192000E1BE00BF40F2A05038B51B21C0F202005A
:1019300017F092FA49F2E460C1F6FF704DF2E0341C
:1019400013F0D6FEC2F200044CF2D8512046C2F287
:10195000000110F07BFE4DF21801C1F6FF7149F253
:10196000F8224CF29820C2F20000C1F6FF7244F255
:101970007013C2F200034D68C570D27B4A6000202C
:1019800063259D6383F83C00586372B6AA42A8BFE2
:101990002A469200DA6262B62046BDE8384010F06E
:1019A000A1BE00BF40F2BC5038B51C21C0F20200FD
:1019B00017F052FA49F2E460C1F6FF704DF2E034DC
:1019C00013F096FEC2F200044BF200112046C1F65D
:1019D000FF7110F03BFE4DF21801C1F6FF7149F2A4
:1019E000F8224CF29820C2F20000C1F6FF7244F2D5
:1019F0007013C2F200034D68C570527D4A6000202A
:101A000063259D6383F83C00586372B6AA42A8BF61
:101A10002A469200DA6262B62046BDE8384010F0ED
:101A200061BE00BF40F2DC5038B51F21C0F2020099
:101A300017F012FA49F2E460C1F6FF704DF2E0349B
:101A400013F056FEC2F200044DF608312046C1F6EE
:101A5000FF7110F0FBFD4DF21801C1F6FF7149F264
:101A6000F8224CF29820C2F20000C1F6FF7244F254
:101A70007013C2F200034D68C570527C4A600020AA
:101A800003259D6383F83C00586372B6AA42A8BF41
:101A90002A469200DA6262B62046BDE8384010F06D
:101AA00021BE00BF40F2FC5038B51821C0F2020040
:101AB00017F0D2F949F2E460C1F6FF704DF2E0345C
:101AC00013F016FEC2F200044BF27C312046C2F243
:101AD000000110F0BBFD4DF21801C1F6FF7149F293
:101AE000F8224CF29820C2F20000C1F6FF7244F2D4
:101AF0007013C2F200034D688570D2794A600020ED
:101B000063259D6383F83C00586372B6AA42A8BF60
:101B10002A469200DA6262B62046BDE8384010F0EC
:101B2000E1BD00BF40F2186038B52021C0F20200CC
:101B300017F092F949F2E460C1F6FF704DF2E0341B
:101B400013F0D6FDC2F200044DF6F4112046C1F6A2
:101B5000FF7110F07BFD4DF21801C1F6FF7149F2E3
:101B6000F8224CF29820C2F20000C1F6FF7244F253
:101B70007013C2F200034D68C570D27C4A60002029
:101B800060259D6383F83C00586372B6AA42A8BFE3
:101B90002A469200DA6262B62046BDE8384010F06C
:101BA000A1BD00BF40F23C6038B52021C0F2020068
:101BB00017F052F949F2E460C1F6FF704DF2E034DB
:101BC00013F096FDC2F200044BF2C0012046C1F6AC
:101BD000FF7110F03BFD4DF21801C1F6FF7149F2A3
:101BE000F8224CF29820C2F20000C1F6FF7244F2D3
:101BF0007013C2F200034D68457192F822204A60CA
:101C0000002001259D6383F83C00586372B6920062
:101C1000DA6262B62046BDE8384010F063BD00BF0E
:101C200040F2606038B51E21C0F2020017F014F9CE
:101C300049F2E460C1F6FF704DF2E03413F058FD54
:101C4000C2F200044CF2D0712046C2F2000110F042
:101C5000FDFC4DF21801C1F6FF7149F2F8224CF279
:101C60009820C2F20000C1F6FF7244F27013C2F273
:101C700000034D68C570D27E4A60002063259D63D5
:101C800083F83C00586372B6AA42A8BF2A46920065
:101C9000DA6262B62046BDE8384010F023BD00BFCE
:101CA00040F2806070B51A21C0F2020017F0D4F83B
:101CB00049F2E460C1F6FF7013F01AFD4DF2A03155
:101CC0004DF2E030C2F20001C2F2000010F0BEFCA2
:101CD00049F2F822C1F6FF724DF21801C1F6FF7108
:101CE00092F823204E684A604CF2982044F2701318
:101CF000C2F200033021C2F20000002501248A4212
:101D0000467183F83C505C6399630EDC5AB19200D3
:101D100072B6DA6262B64DF2E030C2F20000BDE89F
:101D2000704010F0DFBC0422F2E7C022F0E700BFF1
:101D300040F29C6038B51D21C0F2020017F08CF80B
:101D400049F2E460C1F6FF704DF2E03413F0D0FCCC
:101D5000C2F200044AF6C8312046C2F2000110F077
:101D600075FC4DF21801C1F6FF7149F2F8224CF2F0
:101D70009820C2F20000C1F6FF7244F27013C2F262
:101D800000034D68C570127D4A60002063259D6385
:101D900083F83C00586372B6AA42A8BF2A46920054
:101DA000DA6262B62046BDE8384010F09BBC00BF46
:101DB00040F2BC6038B51F21C0F2020017F04CF8A9
:101DC00049F2E460C1F6FF704DF2E03413F090FC8C
:101DD000C2F200044EF6C4012046C2F2000110F027
:101DE00035FC4DF21801C1F6FF7149F2F8224CF2B0
:101DF0009820C2F20000C1F6FF7244F27013C2F2E2
:101E000000034D68C570127F4A60002063259D6302
:101E100083F83C00586372B6AA42A8BF2A469200D3
:101E2000DA6262B62046BDE8384010F05BBC00BF05
:101E300040F2DC60F8B51921C0F2020017F00CF88E
:101E400049F2E460C1F6FF704DF2E03413F050FC4B
:101E5000C2F200044DF63C612046C1F6FF7110F05D
:101E6000F5FB49F2F823C1F6FF734DF21801C1F6F4
:101E7000FF7193F91E304F684B604CF2982044F28A
:101E80007012C2F200026FF03101C2F200000026AF
:101E900032258B42C770B8BF0B46516382F83C6055
:101EA000956372B6AB42A8BF2B469B00D36262B665
:101EB0002046BDE8F84010F015BC00BF40F2F860C5
:101EC00070B51C21C0F2020016F0C6FF49F2E460B2
:101ED000C1F6FF7013F00CFC4BF630214DF2E030F0
:101EE000C2F20001C2F2000010F0B0FB49F2403231
:101EF000C1F6FF724DF21801C1F6FF7112784E68FB
:101F00004A604CF2982044F27013C2F2000363213D
:101F1000C2F20000002501248A42067083F83C507A
:101F20005C6399630EDC5AB1920072B6DA6262B6F3
:101F30004DF2E030C2F20000BDE8704010F0D2BBBC
:101F40000422F2E74FF4C672EFE700BF40F21870C8
:101F500038B51A21C0F2020016F07EFF49F2E460A3
:101F6000C1F6FF704DF2E03413F0C2FBC2F2000480
:101F70004DF20C712046C2F2000110F067FB4DF2E9
:101F80001801C1F6FF7149F2F8224CF29820C2F212
:101F90000000C1F6FF7244F27013C2F200034D68F4
:101FA000457192F820204A60002063259D6383F8E4
:101FB0003C00586372B6AA42A8BF2A469200DA6271
:101FC00062B62046BDE8384010F08CBB40F2347059
:101FD00070B51C21C0F2020016F03EFF49F2E46029
:101FE000C1F6FF7013F084FB4AF68C214DF2E0300D
:101FF000C2F20001C2F2000010F028FB49F24032A8
:10200000C1F6FF724DF21801C1F6FF7112784E68E9
:102010004A604CF2982044F27013C2F2000363212C
:10202000C2F20000002501248A42067083F83C5069
:102030005C6399630EDC5AB1920072B6DA6262B6E2
:102040004DF2E030C2F20000BDE8704010F04ABB33
:102050000422F2E74FF4C672EFE700BF40F254707B
:1020600008B5C0F20200162116F0F6FE49F2F82378
:10207000C1F6FF7393F82230CBB14DF66060C2F227
:1020800000004FF20F6112F0D1F940F2B8101421A4
:10209000C0F2020016F0E0FE4FF20F6016F052F8A8
:1020A00040F2F810C0F202000F2116F0D5FE49F2FE
:1020B000E460C1F6FF70BDE8084013F019BB00BF33
:1020C00040F26C7008B5C0F20200182116F0C4FE90
:1020D00049F2F823C1F6FF7393F82230D3B14DF6DD
:1020E0005053C1F6FF73FB21986C03681B68984737
:1020F00040F2A8100F21C0F2020016F0ADFE4FF61C
:102100000F3016F01FF840F2F810C0F202000F2155
:1021100016F0A2FE49F2E460C1F6FF70BDE8084087
:1021200013F0E6BA40F2887008B5C0F2020015213B
:1021300016F092FE49F2F823C1F6FF7393F82230AD
:10214000D3B14DF65053C1F6FF73FA21986C036872
:102150001B68984740F2A8100F21C0F2020016F049
:102160007BFE4FF60F2015F0EDFF40F2F810C0F2A5
:1021700002000F2116F070FE49F2E460C1F6FF7014
:10218000BDE8084013F0B4BA40F2A07008B5C0F240
:102190000200152116F060FE49F2F823C1F6FF7324
:1021A00093F82230D3B14DF65053C1F6FF73F821A6
:1021B000986C03681B68984740F2A8100F21C0F282
:1021C000020016F049FE4FF60F0015F0BBFF40F27B
:1021D000F810C0F202000F2116F03EFE49F2E46052
:1021E000C1F6FF70BDE8084013F082BA40F2B87043
:1021F00008B5C0F202001B2116F02EFE49F2F823AA
:10220000C1F6FF7393F82230D3B14DF65053C1F6A7
:10221000FF73FF21986C03681B68984740F2A81071
:102220000F21C0F2020016F017FE4FF60F7015F0E6
:1022300089FF40F2F810C0F202000F2116F00CFEE8
:1022400049F2E460C1F6FF70BDE8084013F050BAEF
:1022500040F2D47008B5C0F202001D2116F0FCFD5A
:1022600049F2F823C1F6FF7393F82230D3B14DF64B
:102270005053C1F6FF73FE21986C03681B689847A2
:1022800040F2A8100F21C0F2020016F0E5FD4FF653
:102290000F6015F057FF40F2F810C0F202000F2156
:1022A00016F0DAFD49F2E460C1F6FF70BDE80840BF
:1022B00013F01EBA40F2F47008B5C0F20200142107
:1022C00016F0CAFD49F2F823C1F6FF7393F82230E5
:1022D000D3B14DF65053C1F6FF73FC21986C0368DF
:1022E0001B68984740F2A8100F21C0F2020016F0B8
:1022F000B3FD4FF60F4015F025FF40F2F810C0F285
:1023000002000F2116F0A8FD49F2E460C1F6FF704B
:10231000BDE8084013F0ECB910B5044640F60C00D7
:10232000C0F20200152116F097FD49F2F823C1F61C
:10233000FF7393F82230F3B1240404F4FE0444F450
:10234000734444F002044DF660602146C2F200007E
:1023500012F06CF840F2B8101421C0F2020016F02E
:102360007BFD204615F0EEFE40F2F810C0F20200B0
:102370000F2116F071FD49F2E460C1F6FF70BDE86F
:10238000104013F0B5B900BF2DE9F041804640F68A
:1023900024000F46C0F20200152116F05DFD49F23F
:1023A000F823C1F6FF7393F822303BB949F2E46099
:1023B000C1F6FF70BDE8F04113F09AB94DF65055E3
:1023C000C1F6FF75F021A86C0368DB6C984757B124
:1023D000444608EB0706A86C14F8011B03681B6849
:1023E0009847A642F7D1A86C0368F721DB6C9847A1
:1023F00040F2A8100F21C0F2020016F02DFD394660
:102400004046002215F0F2FE40F2F810C0F2020041
:102410000F2116F021FD49F2E460C1F6FF70BDE81E
:10242000F04113F065B900BF38B5044640F63C00F2
:102430000D46C0F20200102116F00EFD49F2F823FD
:10244000C1F6FF7393F82230DBB14DF660600023D4
:102450002A46C2F20000214612F026F840F2B810D7
:102460001421C0F2020016F0F7FC29462046002293
:1024700015F0BCFE40F2F810C0F202000F2116F079
:10248000EBFC49F2E460C1F6FF70BDE8384013F0A0
:102490002FB900BF40F6500008B5C0F2020010216D
:1024A00016F0DAFC49F2F823C1F6FF7393F82230F4
:1024B000CBB14DF66060C2F200004FF60F2111F073
:1024C000B5FF40F2B8101421C0F2020016F0C4FCAF
:1024D0004FF60F2015F036FE40F2F810C0F2020061
:1024E0000F2116F0B9FC49F2E460C1F6FF70BDE8B7
:1024F000084013F0FDB800BF40F6640008B5C0F214
:102500000200132116F0A8FC49F2F823C1F6FF736C
:1025100093F82230CBB14DF66060C2F200004FF666
:102520000F3111F083FF40F2B8101421C0F2020005
:1025300016F092FC4FF60F3015F004FE40F2F81042
:10254000C0F202000F2116F087FC49F2E460C1F6E8
:10255000FF70BDE8084013F0CBB800BF40F678002C
:1025600008B5C0F20200162116F076FC49F2F823F5
:10257000C1F6FF7393F82230CBB14DF66060C2F222
:1025800000004FF60F7111F051FF40F2B810142106
:10259000C0F2020016F060FC4FF60F7015F0D2FD8D
:1025A00040F2F810C0F202000F2116F055FC49F27B
:1025B000E460C1F6FF70BDE8084013F099B800BFB1
:1025C00040F6900008B5C0F20200182116F044FC55
:1025D00049F2F823C1F6FF7393F82230CBB14DF6E0
:1025E0006060C2F200004FF60F6111F01FFF40F271
:1025F000B8101421C0F2020016F02EFC4FF60F6046
:1026000015F0A0FD40F2F810C0F202000F2116F004
:1026100023FC49F2E460C1F6FF70BDE8084013F006
:1026200067B800BF40F6AC0008B5C0F202000F2149
:1026300016F012FC49F2F823C1F6FF7393F822302A
:10264000CBB14DF66060C2F200004FF60F4111F0C1
:10265000EDFE40F2B8101421C0F2020016F0FCFBAF
:102660004FF60F4015F06EFD40F2F810C0F2020078
:102670000F2116F0F1FB49F2E460C1F6FF70BDE8EE
:10268000084013F035B800BF40F6BC0008B5C0F2F2
:102690000200102116F0E0FB49F2F823C1F6FF73A7
:1026A00093F82230CBB14DF66060C2F200004FF6D5
:1026B0000F0111F0BBFE40F2B8101421C0F202006D
:1026C00016F0CAFB4FF60F0015F03CFD40F2F81073
:1026D000C0F202000F2116F0BFFB49F2E460C1F620
:1026E000FF70BDE8084013F003B800BF2DE9F041CA
:1026F000804640F6D0000F46C0F20200102116F0CE
:10270000ABFB49F2F823C1F6FF7393F822303BB9D3
:1027100049F2E460C1F6FF70BDE8F04112F0E8BF95
:102720004DF65055C1F6FF75F021A86C0368DB6CBF
:10273000984757B1444608EB0706A86C14F8011BEC
:1027400003681B689847A642F7D1A86C0368F72175
:10275000DB6C984740F2A8100F21C0F2020016F07F
:102760007BFB4DF660603A464146C2F20000002312
:1027700011F09AFE40F2B810C0F20200142116F0D7
:102780006BFB49F2E460C1F6FF70BDE8F04112F066
:10279000AFBF00BF38B5044640F6E400C0F2020007
:1027A0001F2116F059FB49F2F823C1F6FF7393F885
:1027B0002230FBB104F00F044FF202152404C0F2E2
:1027C000100525434DF660602946C2F2000011F065
:1027D0002DFE40F2B8101421C0F2020016F03CFBAE
:1027E000284615F0AFFC40F2F810C0F202000F21AD
:1027F00016F032FB49F2E460C1F6FF70BDE83840E4
:1028000012F076BF40F6041008B5C0F202001021A5
:1028100016F022FB49F2F823C1F6FF7393F8223039
:10282000F3B14DF65053C1F6FF73FA21986C03686B
:102830001B68984740F2A8100F21C0F2020016F062
:102840000BFB4DF66060C2F200004FF60F2111F055
:10285000EDFD40F2B810C0F20200142116F0FCFAAF
:1028600049F2E460C1F6FF70BDE8084012F040BFD5
:1028700040F6181008B5C0F20200132116F0ECFA69
:1028800049F2F823C1F6FF7393F82230F3B14DF605
:102890005053C1F6FF73FB21986C03681B6898477F
:1028A00040F2A8100F21C0F2020016F0D5FA4DF642
:1028B0006060C2F200004FF60F3111F0B7FD40F238
:1028C000B810C0F20200142116F0C6FA49F2E46012
:1028D000C1F6FF70BDE8084012F00ABF40F62C10A8
:1028E00008B5C0F20200182116F0B6FA49F2F82332
:1028F000C1F6FF7393F82230F3B14DF65053C1F691
:10290000FF73FE21986C03681B68984740F2A8107B
:102910000F21C0F2020016F09FFA4DF66060C2F27D
:1029200000004FF60F6111F081FD40F2B810C0F2C7
:102930000200142116F090FA49F2E460C1F6FF702B
:10294000BDE8084012F0D4BE40F6481008B5C0F209
:102950000200102116F080FA49F2F823C1F6FF7345
:1029600093F82230F3B14DF65053C1F6FF73F821BE
:10297000986C03681B68984740F2A8100F21C0F2BA
:10298000020016F069FA4DF66060C2F200004FF6E0
:102990000F0111F04BFD40F2B810C0F202001421FB
:1029A00016F05AFA49F2E460C1F6FF70BDE808403B
:1029B00012F09EBE40F65C1008B5C0F202000F2176
:1029C00016F04AFA49F2F823C1F6FF7393F8223061
:1029D000F3B14DF65053C1F6FF73FC21986C0368B8
:1029E0001B68984740F2A8100F21C0F2020016F0B1
:1029F00033FA4DF66060C2F200004FF60F4111F05D
:102A000015FD40F2B810C0F20200142116F024FAAD
:102A100049F2E460C1F6FF70BDE8084012F068BEFC
:102A200040F66C1008B5C0F20200162116F014FA38
:102A300049F2F823C1F6FF7393F82230F3B14DF653
:102A40005053C1F6FF73FF21986C03681B689847C9
:102A500040F2A8100F21C0F2020016F0FDF94DF669
:102A60006060C2F200004FF60F7111F0DFFC40F21F
:102A7000B810C0F20200142116F0EEF949F2E46039
:102A8000C1F6FF70BDE8084012F032BE40F6841077
:102A900008B5C0F202001B2116F0DEF949F2F82356
:102AA000C1F6FF7393F82230D3B14DF65053C1F6FF
:102AB000FF73F621986C0368DB6C984740F2A8100E
:102AC0000F21C0F2020016F0C7F94FF20F6015F0A7
:102AD00039FB40F2F810C0F202000F2116F0BCF9E9
:102AE00049F2E460C1F6FF70BDE8084012F000BE94
:102AF00040F6A01010B51821C0F2020016F0ACF993
:102B000049F2E460C1F6FF7012F0F2FD4BF6845119
:102B10004DF2E030C2F20001C2F200000FF096FD6B
:102B20004DF2E0300221C2F200000FF0B7FD4CF28E
:102B30009823C2F200034DF21801C1F6FF7193F918
:102B4000052048681870002A19DB44F27013C2F29D
:102B5000000303240020A2424A609C6383F83C00E7
:102B60005863D4BF92000C2272B6DA6262B64DF29C
:102B7000E030C2F20000BDE810400FF0B3BD44F2F7
:102B80007012C2F2000200200324946382F83C0019
:102B900050635871486072B6D06262B64DF2E03050
:102BA000C2F2000001210FF073FDE0E740F6BC1017
:102BB00010B51C21C0F2020016F04EF949F2E46093
:102BC000C1F6FF7012F094FD4CF2A4514DF2E030CA
:102BD000C1F6FF71C2F200000FF038FD4DF2E03097
:102BE0000221C2F200000FF059FD4CF29823C2F20C
:102BF00000034DF21801C1F6FF7193F902204868F5
:102C00001870002A19DB44F27013C2F20003082482
:102C10000020A2424A609C6383F83C005863D4BF02
:102C20009200202272B6DA6262B64DF2E030C2F251
:102C30000000BDE810400FF055BD44F27012C2F222
:102C4000000200200824946382F83C0050639870CE
:102C5000486072B6D06262B64DF2E030C2F2000057
:102C600001210FF015FDE0E738B5054612F0E2FC52
:102C70000446284612F03CFD204438BD10B440F212
:102C80001C040023C0F2020441720261046003725A
:102C9000C36041B1194600E0026942F82310427A4C
:102CA00001339A42F8DC4FF28853C2F200031A68EB
:102CB0000AB90CE01A465369002BFBD1506100237E
:102CC00043618380C38083725DF8044B7047186052
:102CD000F5E700BF10B4036841681A780C78417AB0
:102CE000037A0C4202EA03021AD0837A03F0030348
:102CF0000AB143F0040343F008039A10082B8272D0
:102D00002AD8072B22D2032B2ED011D9042B13D073
:102D1000062B14D1C3685DF8044B023BC3607047B7
:102D2000837A03F00303002AE7D043F00403E4E7C7
:102D3000012B0BD0022B02D1C368013BC3605DF8AD
:102D4000044B70470D2BF7D00E2BF8D1C3685DF8FC
:102D5000044B0133C36070470C2B05D0F2D8092B0C
:102D6000D8D00B2BE8D0EAE7C3685DF8044B0233F8
:102D7000C360704708B54EF67443C2F20003D3F83F
:102D8000EC00FFF7A7FF08BD08B54EF67443C2F28A
:102D90000003D3F8E800FFF79DFF08BD08B54EF625
:102DA0007443C2F20003D3F8E400FFF793FF08BDB9
:102DB00008B54EF67443C2F20003D3F8E000FFF703
:102DC00089FF08BD08B54EF67443C2F20003D3F87C
:102DD000DC00FFF77FFF08BD08B54EF67443C2F272
:102DE0000003D3F8D800FFF775FF08BD08B54EF60D
:102DF0007443C2F20003D3F8D400FFF76BFF08BDA1
:102E000008B54EF67443C2F20003D3F8D000FFF7C2
:102E100061FF08BD08B54EF67443C2F20003D3F853
:102E2000CC00FFF757FF08BD08B54EF67443C2F259
:102E30000003D3F8C800FFF74DFF08BD08B54EF6F4
:102E40007443C2F20003D3F8C400FFF743FF08BD88
:102E500008B54EF67443C2F20003D3F8C000FFF782
:102E600039FF08BD08B54EF67443C2F20003D3F82B
:102E7000BC00FFF72FFF08BD08B54EF67443C2F241
:102E80000003D3F8B800FFF725FF08BD08B54EF6DC
:102E90007443C2F20003D3F8B400FFF71BFF08BD70
:102EA00008B54EF67443C2F20003D3F8B000FFF742
:102EB00011FF08BD08B54EF67443C2F20003D3F803
:102EC000AC00FFF707FF08BD08B54EF67443C2F229
:102ED0000003D3F8A800FFF7FDFE08BD08B54EF6C5
:102EE0007443C2F20003D3F8A400FFF7F3FE08BD59
:102EF00008B54EF67443C2F20003D3F8A000FFF702
:102F0000E9FE08BD08B54EF67443C2F20003D3F8DB
:102F10009C00FFF7DFFE08BD08B54EF67443C2F211
:102F20000003D3F89800FFF7D5FE08BD08B54EF6AC
:102F30007443C2F20003D3F89400FFF7CBFE08BD40
:102F400008B54EF67443C2F20003D3F89000FFF7C1
:102F5000C1FE08BD08B54EF67443C2F20003D3F8B3
:102F60008C00FFF7B7FE08BD08B54EF67443C2F2F9
:102F70000003D3F88800FFF7ADFE08BD08B54EF694
:102F80007443C2F20003D3F88400FFF7A3FE08BD28
:102F900008B54EF67443C2F20003D3F88000FFF781
:102FA00099FE08BD08B54EF67443C2F20003D86F0F
:102FB000FFF790FE08BD00BF08B54EF67443C2F29D
:102FC0000003986FFFF786FE08BD00BF08B54EF6F8
:102FD0007443C2F20003586FFFF77CFE08BD00BFC8
:102FE00008B54EF67443C2F20003186FFFF772FE85
:102FF00008BD00BF08B54EF67443C2F20003D86E98
:10300000FFF768FE08BD00BF08B54EF67443C2F274
:103010000003986EFFF75EFE08BD00BF08B54EF6D0
:103020007443C2F20003586EFFF754FE08BD00BFA0
:1030300008B54EF67443C2F20003186EFFF74AFE5D
:1030400008BD00BF08B54EF67443C2F20003D86D48
:10305000FFF740FE08BD00BF08B54EF67443C2F24C
:103060000003986DFFF736FE08BD00BF08B54EF6A9
:103070007443C2F20003586DFFF72CFE08BD00BF79
:1030800008B54EF67443C2F20003186DFFF722FE36
:1030900008BD00BF08B54EF67443C2F20003D86CF9
:1030A000FFF718FE08BD00BF08B54EF67443C2F224
:1030B0000003986CFFF70EFE08BD00BF08B54EF682
:1030C0007443C2F20003586CFFF704FE08BD00BF52
:1030D00008B54EF67443C2F20003186CFFF7FAFD10
:1030E00008BD00BF08B54EF67443C2F20003D86BAA
:1030F000FFF7F0FD08BD00BF08B54EF67443C2F2FD
:103100000003986BFFF7E6FD08BD00BF08B54EF65B
:103110007443C2F20003586BFFF7DCFD08BD00BF2B
:1031200008B54EF67443C2F20003186BFFF7D2FDE8
:1031300008BD00BF08B54EF67443C2F20003D86A5A
:10314000FFF7C8FD08BD00BF08B54EF67443C2F2D4
:103150000003986AFFF7BEFD08BD00BF08B54EF634
:103160007443C2F20003586AFFF7B4FD08BD00BF04
:1031700008B54EF67443C2F20003186AFFF7AAFDC1
:1031800008BD00BF08B54EF67443C2F20003D8690B
:10319000FFF7A0FD08BD00BF08B54EF67443C2F2AC
:1031A00000039869FFF796FD08BD00BF08B54EF60D
:1031B0007443C2F200035869FFF78CFD08BD00BFDD
:1031C00008B54EF67443C2F200031869FFF782FD9A
:1031D00008BD00BF08B54EF67443C2F20003D868BC
:1031E000FFF778FD08BD00BF08B54EF67443C2F284
:1031F00000039868FFF76EFD08BD00BF08B54EF6E6
:103200007443C2F200035868FFF764FD08BD00BFB5
:1032100008B54EF67443C2F200031868FFF75AFD72
:1032200008BD00BF1D2810B50B4600F0E98302461B
:1032300022D92C2800F064813FD8242800F0EE83A6
:1032400040F2A880282800F0748300F2D680262857
:1032500000F0F58140F2D5824EF67444C2F20004CB
:1032600042F60571C0F2000104222720C4F89C3008
:1032700012F0A6FF012010BD0E2800F097833AD867
:10328000062800F0A1836CD90A2800F0058300F21B
:103290000781082800F07E8140F275824EF6744462
:1032A000C2F2000443F25D11C0F2000104220920C1
:1032B000636212F085FF012010BD342800F0BD8349
:1032C00036D8302800F0638300F2D6802E2800F034
:1032D000528140F201824EF67444C2F2000442F67A
:1032E0006561C0F2000104222F20C4F8BC3012F046
:1032F00067FF012010BD152800F0748364D91928D8
:1033000000F0FA8100F2A580172800F08A8140F2CF
:10331000D1824EF67444C2F2000443F23101C0F28D
:10332000000104221820236612F04AFF012010BD7C
:10333000382800F0CE8275D8362800F0398140F266
:103340007F824EF67444C2F2000442F6C551C0F2C8
:10335000000104223720C4F8DC3012F031FF0120D4
:1033600010BD022800F0018240F27881042800F0AC
:103370004B8140F2BD824EF67444C2F2000443F227
:10338000AD11C0F2000104220520636112F018FFA4
:10339000012010BD202800F0448240F289812228BB
:1033A00000F0238140F2D4824EF67444C2F200044D
:1033B00042F65571C0F2000104222320C4F88C307B
:1033C00012F0FEFE012010BD112800F0B18140F284
:1033D0005A81132800F0FB8040F2B8814EF6744405
:1033E000C2F2000443F28101C0F200010422142061
:1033F000236512F0E5FE012010BD2A2800F0AC8004
:1034000040F2E0814EF67444C2F2000442F6B56127
:10341000C0F2000104222B20C4F8AC3012F0D0FE20
:10342000012010BD3A2800F08880C0F072823B284D
:1034300040F06D824EF67444C2F2000442F67551BB
:10344000C0F200010422C4F8EC3012F0B9FE0120F1
:1034500010BD1B2863D040F28B824EF67444C2F23A
:10346000000442F6E171C0F2000104221C2023672F
:1034700012F0A6FE012010BD322824D040F2928125
:103480004EF67444C2F2000442F61561C0F2000127
:1034900004223320C4F8CC3012F092FE012010BD7B
:1034A0000C281FD040F29E814EF67444C2F20004F4
:1034B00043F20D11C0F2000104220D20636312F0EB
:1034C0007FFE012010BD4EF67444C2F2000442F6A5
:1034D0002961C0F200010422C4F8C83012F070FE65
:1034E000012010BD4EF67444C2F2000443F22111D3
:1034F000C0F200010422236312F062FE012010BD1D
:103500004EF67444C2F2000442F6A161C0F200011A
:103510000422C4F8B03012F053FE012010BD4EF664
:103520007444C2F2000442F6F571C0F200010422B4
:10353000E36612F045FE012010BD4EF67444C2F25F
:10354000000442F68951C0F200010422C4F8E830B8
:1035500012F036FE012010BD4EF67444C2F2000493
:1035600042F6C961C0F200010422C4F8A83012F08A
:1035700027FE012010BD4EF67444C2F2000442F64C
:103580007961C0F200010422C4F8B83012F018FECC
:10359000012010BD4EF67444C2F2000443F27111D2
:1035A000C0F200010422236212F00AFE012010BDC5
:1035B0004EF67444C2F2000442F6D951C0F2000142
:1035C0000422C4F8D83012F0FBFD012010BD4EF6E5
:1035D0007444C2F2000443F29501C0F200010422D7
:1035E000E36412F0EDFD012010BD4EF67444C2F20A
:1035F000000442F66971C0F200010422C4F8883068
:1036000012F0DEFD012010BD4EF67444C2F200043B
:1036100043F2C111C0F20001236112F0D1FD01207B
:1036200010BD4EF67444C2F2000443F24501C0F2EC
:1036300000010422E36512F0C3FD012010BD4EF627
:103640007444C2F2000442F61971C0F2000104226F
:10365000C4F8983012F0B4FD012010BD002800F02D
:10366000FF80012840F053814EF67444C2F20004FA
:1036700043F2FD11C0F2000104220120636012F048
:103680009FFD012010BD0F2800F0F880102840F0A9
:103690003E814EF67444C2F2000443F2D101C0F2FE
:1036A000000104221020236412F08AFD012010BDC5
:1036B0001E282FD01F2840F02A814EF67444C2F2F3
:1036C000000442F6A571C0F2000104221F20E36746
:1036D00012F076FD012010BD4EF67444C2F20004D3
:1036E00042F68D61C0F2000104222D20C4F8B430EE
:1036F00012F066FD012010BD4EF67444C2F20004C3
:1037000043F21D01C0F200010422636612F058FD6D
:10371000012010BD4EF67444C2F2000442F6B971A5
:10372000C0F200010422A36712F04AFD012010BD7F
:103730004EF67444C2F2000443F2BD01C0F200012F
:103740000422636412F03CFD012010BD4EF6744467
:10375000C2F2000443F2A901C0F2000104221220C7
:10376000A36412F02DFD012010BD4EF67444C2F288
:10377000000443F2E911C0F200010422A36012F038
:103780001FFD012010BD4EF67444C2F2000443F246
:103790008511C0F2000104220720E36112F010FD40
:1037A000012010BD4EF67444C2F2000442F63D61A1
:1037B000C0F2000104223120C4F8C43012F000FD30
:1037C000012010BD4EF67444C2F2000442F6DD61E1
:1037D000C0F2000104222920C4F8A43012F0F0FC49
:1037E000012010BD4EF67444C2F2000443F23511BC
:1037F000C0F2000104220B20E36212F0E1FC012080
:1038000010BD4EF67444C2F2000442F62D71C0F2AF
:10381000000104222520C4F8943012F0D1FC0120CC
:1038200010BD4EF67444C2F2000442F69171C0F22B
:1038300000010422C4F8803012F0C2FC012010BD47
:103840004EF67444C2F2000442F6ED51C0F200019B
:1038500004223520C4F8D43012F0B2FC012010BD8F
:103860004EF67444C2F2000443F21121C0F200018A
:103870000422236012F0A4FC012010BD4EF6744413
:10388000C2F2000443F2E501C0F200010422E36346
:1038900012F096FC012010BD4EF67444C2F20004F2
:1038A00043F24911C0F200010422A36212F088FC25
:1038B000012010BD4EF67444C2F2000443F25901D7
:1038C000C0F2000104221620A36512F079FC012049
:1038D00010BD4EF67444C2F2000442F6B151C0F27B
:1038E00000010422C4F8E03012F06AFC012010BD8F
:1038F0004EF67444C2F2000443F2D511C0F2000146
:1039000004220320E36012F05BFC012010BD0020C4
:1039100010BD4EF67444C2F2000442F69D51C0F24E
:10392000000104223920C4F8E43012F049FC0120DF
:1039300010BD4EF67444C2F2000442F6F161C0F2CA
:1039400000010422C4F8A03012F03AFC012010BD9E
:103950004EF67444C2F2000442F67D71C0F20001DA
:1039600004222120C4F8843012F02AFC012010BD6A
:103970004EF67444C2F2000443F20901C0F20001A1
:1039800004221A20A36612F01BFC012010BD4EF683
:103990007444C2F2000442F65161C0F200010422F4
:1039A000C4F8C03012F00CFC012010BD4EF6744477
:1039B000C2F2000443F2F901C0F200010422A36341
:1039C00012F0FEFB012010BD4EF67444C2F200045A
:1039D00043F29911C0F200010422A36112F0F0FB3E
:1039E000012010BD4EF67444C2F2000443F26D0192
:1039F000C0F200010422636512F0E2FB012010BD59
:103A00004EF67444C2F2000442F6CD71C0F20001D9
:103A10000422636712F0D4FB012010BD4EF67444FB
:103A2000C2F2000442F64171C0F200010422C4F85F
:103A3000903012F0C5FB012010BD4EF67444C2F266
:103A4000000442F60161C0F200010422C4F8D03043
:103A500012F0B6FB012010BDF8B5044615460E461F
:103A60000846022112F024FE2846022112F020FE10
:103A700040F22413C0F20F03012253F836002272E1
:103A800000F50071216053F8351062724DF2C043A9
:103A900001F5007762F31F4300226760E260013B9B
:103AA000FDD190F8003291F8002203F00103D20713
:103AB00044BF43F00203DBB2A37221463046FFF756
:103AC000B1FB214620742846FFF7ACFB237C184449
:103AD00020742046F8BD00BF10B5037C012B0446BE
:103AE0002CD972B6E36862B6002BB8BF03336269A3
:103AF0009B1093420DDBA1698B4217DC237C012BC9
:103B000020D972B6E06862B60028B8BF03308010D2
:103B100010BD237F23B972B69200E26062B6EDE772
:103B2000A3699B0072B6E36062B6E7E7237F002BD0
:103B3000F1D172B68900E16062B6DFE772B6FFF7D5
:103B4000C9F8CFE772B62046FFF7C4F8DAE700BF3E
:103B5000091A49B238B581EAE175A5EBE175D5B12D
:103B600000294FF000040BDB4DF2E0300134C2F2CB
:103B700000000021E4B20EF08BFDAC42F4DB38BD56
:103B80004DF2E0300134C2F200000121E4B20EF047
:103B90007FFDAC42F4DB38BDF8B544F27014C2F2DC
:103BA0000004074604F12000FFF796FF4CF2982529
:103BB000C2F200054DF2E036C2F200064BF6F011FB
:103BC000E855C2F2000130460EF040FD30460221B9
:103BD0000EF064FD4DF2180295F90030C1F6FF7247
:103BE000002105205360A06323EAE37384F83C10AE
:103BF000616372B68342A8BF03469B00E36262B66C
:103C0000F8BD00BFF8B544F27014C2F200040746D4
:103C100004F12000FFF760FF4CF29825C2F2000586
:103C20004DF2E036C2F200064CF2A451E855C1F65E
:103C3000FF7130460EF00AFD304602210EF02EFDD7
:103C40004DF2180295F90230C1F6FF7200210820EA
:103C50005360A06323EAE37384F83C10616372B697
:103C60008342A8BF03469B00E36262B6F8BD00BF73
:103C7000F8B544F27014C2F20004074604F12000C3
:103C8000FFF72AFF4CF29825C2F200054DF2E0360C
:103C9000C2F200064EF2C871E855C2F20001304689
:103CA0000EF0D4FC304602210EF0F8FC4DF2180262
:103CB00095F90330C1F6FF72002112205360A06312
:103CC00023EAE37384F83C10616372B68342A8BFB1
:103CD00003469B00E36262B6F8BD00BFF8B544F24C
:103CE0007014C2F20004074604F12000FFF7F4FE4E
:103CF0004CF29825C2F200054DF2E036C2F2000601
:103D00004BF68451E855C2F2000130460EF09EFC9D
:103D1000304602210EF0C2FC4DF2180295F9053032
:103D2000C1F6FF72002103205360A06323EAE3730E
:103D300084F83C10616372B68342A8BF03469B00BF
:103D4000E36262B6F8BD00BF38B549F24034C1F64F
:103D5000FF7440F6DC1049F2E4650B21C1F6FF75F3
:103D6000C0F2020015F078F800230A2221782846D4
:103D700011F0D0FC284611F0BBFC4BF68413C1F6C1
:103D8000FF7322781A7038BD38B5054649F2E464ED
:103D900040F6E8100A21C1F6FF74C0F2020015F0E7
:103DA0005BF8294600230A22204611F0B3FC204686
:103DB00011F09EFC07EE905A0023C4F2C623F8EEE1
:103DC000676A07EE103A86EE870A002307EE903AFC
:103DD0004BF2CC13C2F2000330EE270A186807F04A
:103DE000EBFB49F2F823C1F6FF731D7138BD00BF2C
:103DF00038B5054649F2E46440F6F4100C21C1F6EA
:103E0000FF74C0F2020015F027F8294600230A22A9
:103E1000204611F07FFC204611F06AFC07EE905A14
:103E20000023C4F2C623F8EE676A07EE103A86EE66
:103E3000870A002307EE903A4BF2CC13C2F200033C
:103E400030EE270A186807F0A3FC49F2F823C1F600
:103E5000FF735D7138BD00BF38B5054649F2E464B3
:103E600040F604200D21C1F6FF74C0F2020014F0E8
:103E7000F3FF294600230A22204611F04BFC20467E
:103E800011F036FC07EE905A0023C4F2C623F8EE78
:103E9000676A07EE103A86EE870A002307EE903A2B
:103EA0004BF2CC13C2F2000330EE270A186807F079
:103EB0005BFD49F2F823C1F6FF739D7138BD00BF69
:103EC00038B5054649F2E46440F614200B21C1F6EA
:103ED000FF74C0F2020014F0BFFF294600230A223B
:103EE000204611F017FC204611F002FC07EE905A14
:103EF0000023C4F2C623F8EE676A07EE103A86EE96
:103F0000870A002307EE903A4BF2CC13C2F200036B
:103F100030EE270A186807F011FE49F2F823C1F6BF
:103F2000FF73DD7138BD00BF38B5054649F2E46462
:103F300040F620200B21C1F6FF74C0F2020014F0FD
:103F40008BFF2946204611F075FB204611F0D0FB6F
:103F500007EE905A0023C4F2C623F8EEE76A07EE94
:103F6000103A86EE870A002307EE903A4BF2CC1304
:103F7000C2F2000330EE270A186808F08DF949F202
:103F8000F823C1F6FF731D7238BD00BF38B5054672
:103F900049F2E46440F62C200E21C1F6FF74C0F211
:103FA000020014F059FF2946204611F043FB204639
:103FB00011F09EFB49F2F823C1F6FF735D7238BD24
:103FC00038B5054649F2E46440F63C200921C1F6C3
:103FD000FF74C0F2020014F03FFF2946204611F0A2
:103FE00029FB204611F084FB07EE905A0023C4F20F
:103FF000482306EE103AF8EEE77A0023C4F2C8230D
:1040000006EE903A77EE867A002387EEA60A07EE50
:10401000103A4BF2CC13C2F2000330EE070A1868D4
:1040200008F028FA49F2F823C1F6FF739D7238BDF3
:1040300038B5054649F2E46440F648200B21C1F644
:10404000FF74C0F2020014F007FF294600230A2281
:10405000204611F05FFB204611F04AFB07EE905A14
:104060000023C4F2C623F8EE676A07EE103A86EE24
:10407000870A002307EE903A4BF2CC13C2F20003FA
:1040800030EE270A186808F0E1FA49F2F823C1F681
:10409000FF73DD7238BD00BF38B5054649F2E464F0
:1040A00040F654201321C1F6FF74C0F2020014F050
:1040B000D3FE294600230A22204611F02BFB20467E
:1040C00011F016FB07EE905A0023C4F2C623F8EE57
:1040D000676A07EE103A86EE870A002307EE903AE9
:1040E0004BF2CC13C2F2000330EE270A186807F037
:1040F000E7FF49F2F823C1F6FF731D7338BD00BF17
:1041000038B5054649F2E46440F668201621C1F648
:10411000FF74C0F2020014F09FFE294600230A2219
:10412000204611F0F7FA204611F0E2FA07EE905A15
:104130000023C4F2C623F8EE676A07EE103A86EE53
:10414000870A002307EE903A4BF2CC13C2F2000329
:1041500030EE270A186807F0C7FE49F2F823C1F6C7
:10416000FF735D7338BD00BF38B5054649F2E4649E
:1041700040F680201321C1F6FF74C0F2020014F053
:104180006BFE294600230A22204611F0C3FA20467E
:1041900011F0AEFA07EE905A0023C4F2C623F8EEEF
:1041A000676A07EE103A86EE870A002307EE903A18
:1041B0004BF2CC13C2F2000330EE270A186807F066
:1041C000A7FD49F2F823C1F6FF739D7338BD00BF08
:1041D00038B5054649F2E46440F694200E21C1F654
:1041E000FF74C0F2020014F037FE294600230A22B1
:1041F000204611F08FFA204611F07AFA07EE905A15
:104200000023C4F2C623F8EE676A07EE103A86EE82
:10421000870A002307EE903A4BF2CC13C2F2000358
:1042200030EE270A186808F0FDFA49F2F823C1F6C3
:10423000FF73DD7338BD00BF30B5054649F2E46455
:1042400040F6A42083B0C1F6FF740E21C0F2020034
:1042500014F002FE294600230A22204611F05AFAE1
:10426000204611F045FA49F2F82407EE905AC1F6BB
:10427000FF740023F8EE676A07EE903AB6EE007A14
:10428000637D627CE6EE877A44F2B010C2F20000F1
:1042900001EE103A237D00EE903AFCEEE77AB8EE9C
:1042A000411AF8EE600ACDED017AF2EE047A81EE61
:1042B000271AE37C9DF80410C0EEA70A00EE103A1E
:1042C000A37CB8EE400A09F00FFE257403B030BDA0
:1042D00030B5054649F2E46440F6B42083B0C1F637
:1042E000FF741221C0F2020014F0B6FD294600232B
:1042F0000A22204611F00EFA204611F0F9F907EED5
:10430000905AF8EE676AB0EE087AC6EE877A49F2FC
:10431000F824C1F6FF740022637D217C44F2B010C2
:10432000C2F2000007EE102A01EE103A237D77EE6C
:10433000877A00EE903AFCEEE77AB8EE411AF8EE92
:10434000600ACDED017AF2EE047A81EE271AE37C61
:104350009DF80420C0EEA70A00EE103AA37CB8EE48
:10436000400A09F0C1FD657403B030BD30B50546A3
:1043700049F2E46440F6C82083B0C1F6FF740F210F
:10438000C0F2020014F068FD294600230A222046EC
:1043900011F0C0F9204649F2F824C1F6FF7411F07B
:1043A000A7F907EE905A002307EE103A637D627C6E
:1043B000217CF8EE677A01EE103A237D77EE877A5A
:1043C00000EE903AFCEEE77AB8EE411AF8EE600A99
:1043D000CDED017AF2EE047A81EE271AE37C44F205
:1043E000B010C2F20000C0EEA70A00EE103A9DF82D
:1043F0000430B8EE400A09F077FD003518BF0125FA
:10440000A57403B030BD00BF70B5064649F2E4653F
:1044100040F6D8201321C1F6FF75C0F2020049F220
:10442000F82414F019FDC1F6FF74314600230A2266
:10443000284611F06FF9284611F05AF9637D627C25
:10444000217C01EE103A237D00EE903AB8EE411A3D
:10445000F8EE600AF2EE047A81EE271A44F2B01008
:10446000A37CC2F20000C0EEA70A07EE906AB8EE85
:10447000670A09F039FDE67470BD00BF70B50646E5
:1044800049F2E46540F6EC201021C1F6FF75C0F258
:10449000020049F2F82414F0DFFCC1F6FF74314643
:1044A00000230A22284611F035F9284611F020F998
:1044B000637D627C217C01EE103A07EE906AE37C1A
:1044C000F8EE670A00EE103AB8EE411AF2EE047AFE
:1044D00044F2B010A37C81EE271AC2F20000C0EEB5
:1044E000A70AB8EE400A09F0FFFC267570BD00BFB0
:1044F00070B5064649F2E46540F600300F21C1F67A
:10450000FF75C0F2020049F2F82414F0A5FCC1F6D0
:10451000FF74314600230A22284611F0FBF8284692
:1045200011F0E6F8237D627C217C00EE903A07EEE4
:10453000906AE37CB8EE671A00EE103AF8EE600A73
:10454000F2EE047A44F2B010A37CC0EEA70AC2F2E5
:10455000000081EE271AB8EE400A09F0C5FC667526
:1045600070BD00BF10B5044640F610301421C0F2F3
:10457000020014F071FC49F2E460002321460A2293
:10458000C1F6FF7011F0C6F849F2E460C1F6FF70A1
:1045900011F0AEF807EE904A0023C4F2C62307EEEE
:1045A000103AB8EE676A0023C6EE077A06EE903A34
:1045B00077EEA67AB7EE007AF4EEC77AF1EE10FA4B
:1045C00015DD44F2BC12C2F2000245F2606147F60A
:1045D0007053535249F2F8224DF6D061C1F6FF7282
:1045E000C1F6FF7145F2606094750B5210BDF4EE98
:1045F000E67AF1EE10FA33D445F62943C4F20F639C
:1046000007EE103A27EE877ABDEEC77A17EE103A1A
:1046100003F5B34319331BB244F2BC12B7EE007A70
:10462000C2F2000245F26061F4EEC77AF1EE10FAD0
:1046300053521BDCF5EEC07AF1EE10FA13D445F6B6
:104640002943C4F20F6307EE103A67EE877AFDEE56
:10465000E77A17EE903A03F5B34319331BB2B9E783
:1046600045F69913D8E745F69913B3E747F6705323
:10467000B0E700BF38B5044640F628301321C0F239
:10468000020014F0E9FB49F2E460002321460A220B
:10469000C1F6FF7011F03EF849F2E460C1F6FF7018
:1046A00011F026F807EE904A0023C4F2C62307EE65
:1046B000103AB8EE676A0023C6EE077A06EE903A23
:1046C00077EEA67AB7EE007AF4EEC77AF1EE10FA3A
:1046D00042DD44F6CD4143F2333272B644F2BC13AC
:1046E000C2F2000345F25C6545F25E605A5319520E
:1046F00062B6B7EE007AF4EEC77AF1EE10FA15DD85
:1047000044F6CD4143F2333372B64DF6D062C1F672
:10471000FF7245F25C6545F25E605353115262B61A
:1047200049F2F823C1F6FF73DC7538BDF5EEC07AA7
:10473000F1EE10FA2CD44CF6CD43C4F24C6307EEE4
:10474000103A67EE877AFDEEE77A17EE903AC3F5F6
:10475000004109B21BB2D7E7F4EEE67AF1EE10FAA7
:1047600010D44CF6CD43C4F24C6307EE103A27EE5A
:10477000877ABDEEC77A17EE102AC2F5004109B25A
:1047800012B2AAE74FF40041CFF6FF710022A4E76E
:104790004FF40041CFF6FF710023B5E710B5044692
:1047A00040F63C301121C0F2020014F055FB49F2F2
:1047B000E460214600230A22C1F6FF7010F0AAFF30
:1047C00049F2E460C1F6FF7010F092FF07EE904AE4
:1047D0000023C4F2C62306EE103AF8EE675A00230F
:1047E000C5EE867A4DF618124DF65001C2F200025F
:1047F000C2F2000106EE903A4FF47E43C4F2FF632A
:1048000007EE103A77EEA67A4FF48033F4EEC77ACB
:10481000F1EE10FA93618B612BDC4FF47E43CCF206
:10482000FF6307EE103AF4EEC77AF1EE10FA2BD4DC
:10483000B0EE677ABEEEC87A17EE103A4FF47E40BB
:10484000C4F2FF6007EE100AF4EEC77AF1EE10FA38
:10485000D36124DC4FF47E43CCF2FF6307EE103AC1
:10486000F4EEC77AF1EE10FA12D50023C8F2010374
:1048700003E00023C7F6FF73D36149F2F822C1F6C3
:10488000FF72CB61147610BD0023C8F20103D5E797
:10489000B0EE677ABEEEC87A17EE103AEDE7002365
:1048A000C7F6FF73E9E700BF38B5054649F2E4648F
:1048B00040F650301521C1F6FF74C0F2020014F02A
:1048C000CBFA002329460A22204610F023FF204677
:1048D00010F00EFF49F2F823C1F6FF735D7638BD84
:1048E00038B5054649F2E46440F668301121C1F656
:1048F000FF74C0F2020014F0AFFA002329460A2226
:10490000204610F007FF204610F0F2FE49F2F8238F
:10491000C1F6FF739D7638BD38B5054649F2E464AB
:1049200040F67C301121C1F6FF74C0F2020014F091
:1049300093FA002329460A22204610F0EBFE204677
:1049400010F0D6FE49F2F823C1F6FF73DD7638BDCC
:1049500070B5064649F2E46540F690301221C1F682
:10496000FF75C0F2020049F2F82414F075FAC1F69E
:10497000FF74314600230A22284610F0CBFE284659
:1049800010F0B6FE637F06EE106A07EE903A002341
:10499000C4F2C62306EE903AF8EE677AB8EE466A9D
:1049A000C7EEA60A002344F2B010C2F2000086EE61
:1049B000260A07EE103A70EE870A30EE070A08F072
:1049C00007FE267770BD00BF70B5064649F2E46564
:1049D00040F6A4301421C1F6FF75C0F2020049F27E
:1049E000F82414F039FAC1F6FF74314600230A2284
:1049F000284610F08FFE284610F07AFE237F06EE40
:104A0000106A07EE903A0023C4F2C62306EE903AED
:104A1000F8EE677AB8EE466A87EEA60A002344F2FB
:104A2000B010C2F20000C6EE260A07EE103A30EED1
:104A3000070A70EE870A08F0CBFD667770BD00BFED
:104A400070B5064649F2E46540F6BC300C21C1F66B
:104A5000FF75C0F2020049F2F82414F0FDF9C1F626
:104A6000FF74314600230A22284610F053FE2846E0
:104A700010F03EFE94F91F3007EE106A07EE903AF0
:104A80000023C4F2482306EE103AF8EEE77AB8EEB7
:104A9000477A77EE867A37EE067A0023C4F2C82387
:104AA00006EE903A77EEA77A37EE077AC7EEA60AB7
:104AB00044F2B010C2F2000087EE260AF7EE007A48
:104AC00070EEE70A30EE670A08F0B6FEA67770BD12
:104AD00070B5064649F2E46540F6CC300E21C1F6C9
:104AE000FF75C0F2020049F2F82414F0B5F9C1F6DE
:104AF000FF74314600230A22284610F00BFE284698
:104B000010F0F6FD94F91E3007EE106A07EE903AA9
:104B10000023C4F2482306EE103AF8EEE77AB8EE26
:104B2000477A77EE867A37EE067A0023C4F2C823F6
:104B300006EE903A77EEA77A37EE077A87EEA60A66
:104B400044F2B010C2F20000C7EE260AF7EE007A77
:104B500030EE670A70EEE70A08F06EFEE67770BD89
:104B600038B5054649F2E46440F6DC300D21C1F663
:104B7000FF74C0F2020014F06FF900230A222946E4
:104B8000204610F0C7FD204610F0B2FD07EE905A07
:104B90000023C4F2C62306EE903AB8EE676A0023FB
:104BA000C6EE267A49F2F822C1F6FF7282F820504A
:104BB00007EE103A4BF2BC0377EE877AC1F6FF732B
:104BC000C3ED007A38BD00BF38B5054649F2E4644C
:104BD00040F6EC301121C1F6FF74C0F2020014F06F
:104BE0003BF9002329460A22204610F093FD204677
:104BF00010F07EFD49F2F823C1F6FF7383F82150CF
:104C000038BD00BF38B5044649F2E46540F60040BF
:104C10001321C1F6FF75C0F2020014F01DF9214600
:104C200000230A22284610F075FD284610F060FD8A
:104C300049F2F8230034C1F6FF7318BF012483F84A
:104C4000224038BD70B5064649F2E46540F614408E
:104C5000C1F6FF750D21C0F202004BF2CC1414F026
:104C6000FBF8C2F20004314600230A22284610F065
:104C700051FD284610F03CFD2068314607F0F8FB56
:104C800049F2F823C1F6FF73206883F82360BDE87A
:104C9000704006F09FB900BF2DE9F04149F2F824B9
:104CA000C1F6FF7400232779C4F2C62340F6E8104A
:104CB0002DED028BC0F2020008EE903A002308EEC0
:104CC000103AFBF7FDFC3846FBF7E8FC07EE907A5C
:104CD000F8EE677A4BF2CC1587EEA80AC2F200050F
:104CE00049F2E4662868C1F6FF7630EE080A06F05D
:104CF00063FC94F80580277140F6F410C0F20200BE
:104D0000FBF7DEFC4046FBF7C9FC07EE908AF8EEA5
:104D1000677A286887EEA80A30EE080A06F038FDA0
:104D2000A77984F8058040F60420C0F20200FBF762
:104D3000C7FC3846FBF7B2FC07EE907AF8EE677ACC
:104D4000286887EEA80A30EE080A06F00DFE94F8EF
:104D50000780A77140F61420C0F20200FBF7B0FCF8
:104D60004046FBF79BFC07EE908AF8EE677A2868CE
:104D700087EEA80A30EE080A06F0E0FE94F9087003
:104D800084F8078040F620200B21C0F2020014F0C6
:104D900063F83946304610F04DFC304610F0A8FC60
:104DA00007EE907AF8EEE77A286887EEA80A30EEE8
:104DB000080A07F071FA94F90A80277240F63C203D
:104DC0000921C0F2020014F047F84146304610F0C5
:104DD00031FC304610F08CFC07EE908A0023C4F2C0
:104DE000482306EE903AF8EEE77A0023C4F2C8238F
:104DF00007EE103A77EEA67A286887EE870A30EE3B
:104E0000080A07F037FBE77A84F80A8040F6482062
:104E1000C0F20200FBF754FC3846FBF73FFC07EEFC
:104E2000907AF8EE677A286887EEA80A30EE080ACA
:104E300007F00CFC94F80C80E77240F65420C0F2A6
:104E40000200FBF73DFC4046FBF728FC07EE908A8A
:104E5000F8EE677A286887EEA80A30EE080A07F0AD
:104E60002FF9677B84F80C8040F66820C0F20200BE
:104E7000FBF726FC3846FBF711FC07EE907AF8EEBC
:104E8000677A286887EEA80A30EE080A07F02CF83F
:104E900094F80E80677340F68020C0F20200FBF7A2
:104EA0000FFC4046FBF7FAFB07EE908AF8EE677AB4
:104EB000286887EEA80A30EE080A06F029FFE77B8B
:104EC00084F80E8040F69420C0F20200FBF7F8FB55
:104ED0003846FBF7E3FB07EE907AF8EE677A28682E
:104EE00087EEA80A30EE080A07F09CFC207CE773E6
:104EF000FFF7A2F9607CFFF7EBF9A07CFFF736FA29
:104F0000E07CFFF781FA207DFFF7B8FA607DFFF7BC
:104F1000EFFAA07DFFF726FBE07DFFF7ABFB207EDD
:104F2000FFF73CFC677E40F65030C0F20200FBF712
:104F3000C7FB3846FBF7B2FB94F81A80677640F659
:104F40006830C0F20200FBF7BBFB4046FBF7A6FB54
:104F5000E77E84F81A8040F67C30C0F20200FBF74E
:104F6000AFFB394600230A22304610F0D3FB30460F
:104F700010F0BEFB207FE776FFF7EAFC607FFFF7CB
:104F800023FDA07FFFF75CFDE07FFFF7A1FD94F814
:104F9000207040F6DC30C0F20200FBF791FB39468E
:104FA0000A220023304610F0B5FB304610F0A0FB7B
:104FB00007EE907AB8EE677A94F8216084F8207052
:104FC000C7EE287A4BF2BC0340F6EC30C1F6FF7313
:104FD000C0F2020037EE888A83ED008AFBF770FB8F
:104FE0003046FBF75BFB94F8227084F8216040F6B2
:104FF0000040C0F20200FBF763FB3846FBF74EFBB4
:1050000094F8236084F8227040F61440C0F2020045
:10501000FBF756FB3046FBF741FB2868314607F0AB
:1050200027FABDEC028B286884F82360BDE8F041C4
:1050300005F0D0BFF8B54DF65054C1F6FF7447F6F1
:105040001221A06C0368DB69984740F6396540F689
:10505000915140F6E1620326C0F20005C0F2000162
:10506000C0F2000240F66D0084F864606560216063
:10507000E260C0F2000040F6692340F6E50742F224
:10508000294642F2957540F65D1142F2193260618F
:10509000C0F20003C0F20007C0F20006C0F2000533
:1050A000C0F20001C0F2000242F25D00A36127617C
:1050B000E6612562A160A262C0F2000042F289634B
:1050C00042F2954742F2F94642F2256542F2C15159
:1050D00042F25D52C0F20001C0F20002E062C0F292
:1050E0000003C0F20007C0F20006C0F2000540F65F
:1050F0002440216462642363676300234FF6FF77D3
:10510000A663E563C0F2020084F84C3084F84E30A8
:1051100084F84D30A365636584F8E93084F866301F
:1051200084F8653084F8673084F86830E76527666E
:10513000FBF7D0FA0DF04AFB4DF66063C2F20003B4
:1051400047F2A90447F2112147F27932C0F2000474
:10515000C0F20001C0F2000247F2D940C3F8684132
:10516000C3F86411C3F87021C0F2000047F2E157A0
:1051700047F2197642F2893540F6F12447F62101CB
:1051800040F6F112C3F87801C0F20007C0F2000641
:10519000C0F20005C0F20004C0F20001C0F200023B
:1051A00042F68D20C3F87C71C3F87461C3F8845152
:1051B000C3F88841C3F86C11C3F89021C0F2000015
:1051C00042F2891742F2251642F2C10542F2B52495
:1051D00042F2512142F2ED12C0F20001C0F200028F
:1051E000C3F89401C0F20007C0F20006C0F2000547
:1051F000C0F2000440F63C40C3F89871C3F89C61CB
:10520000C3F8A051C3F8A441C3F8A811C3F8AC2156
:10521000C0F20200FBF75EFA4FF65803C2F2000339
:1052200047F2591EC0F2000E4FF65007C3F800E0D7
:10523000C2F2000747F2C12EC0F2000E4FF654042E
:10524000C7F800E0C2F2000447F2254EC0F2000E9B
:105250004FF62806C4F800E0C2F2000647F2595E95
:10526000C0F2000E4FF61802C6F800E0C2F20002CB
:1052700047F2796EC0F2000E4FF61400C2F800E05B
:10528000C2F2000047F2997EC0F2000E4FF63805D8
:10529000C0F800E0C2F2000542F2ED6EC0F2000E6E
:1052A0004FF63001C5F800E0C2F2000140F6E93ED9
:1052B000C0F2000E4FF62403C1F800E0C2F2000372
:1052C00047F6A90EC0F2000E4FF64C07C3F800E0F7
:1052D000C2F2000740F6693EC0F2000E4FF63404F9
:1052E000C2F20004C7F800E040F2B577C0F2000750
:1052F0004FF2FC76C2F2000627604FF62C0242F60F
:105300004917C2F20002C0F200074FF60C0042F645
:105310000504C2F20000C0F2000437604FF64405F5
:105320004FF604014FF6000342F67107C2F2000582
:10533000C2F20003C0F200071460C2F2000142F69C
:10534000B51642F6DD0442F62122C0F20006C0F294
:1053500000040760C0F2000240F65C402E600C6062
:105360001A60C0F20200BDE8F840FBF7B3B900BF15
:1053700070B54BF20352C0EB8023CAF27E5282FB1F
:1053800003122DED048B1A44DB17C3EBA21349F271
:10539000F8249A1C0546C1F6FF7440F6784082B0A6
:1053A00003FB02F300261421C0F2020008EE103ABB
:1053B00084F8246013F050FD49F2E4600A22334679
:1053C0002946C1F6FF7010F0A5F9BAEEC68A40F67C
:1053D00090400121C0F2020013F03EFD18EE100AC9
:1053E00016F07EF941EC100B49F2E4600321C1F69E
:1053F000FF7010F0CFF940F694400621C0F2020091
:1054000013F02AFD49F2E46094F92410C1F6FF700C
:1054100010F010F940F690400121C0F2020013F0A4
:105420001BFD49F2E4609FED560B0321C1F6FF70AE
:1054300010F0B0F940F69C400221C0F2020013F0D7
:105440000BFD40F2F343C3F6357307EE903A28EEB6
:10545000278A18EE100A16F043F941EC190B49F2AD
:10546000E460B0EE490AF0EE690A0321C1F6FF706C
:1054700010F090F940F6A0400121C0F2020013F0B4
:10548000EBFCB0EE490AF0EE690A49F2E460032150
:10549000C1F6FF7010F07EF949F2E460C1F6FF70CA
:1054A00010F026F94FF47E43C4F2FF6307EE903A02
:1054B000B4EEE78AF1EE10FA2FDC4FF47E43CCF223
:1054C000FF6307EE903AB4EEE78AF1EE10FA47D4A4
:1054D000F0EE487AFEEEC87A17EE902A4FF47E413D
:1054E000C4F2FF6107EE901A4DF61813C2F20003E2
:1054F000B4EEE78AF1EE10FA9A613CDC4FF47E4399
:10550000CCF2FF6307EE903AB4EEE78AF1EE10FAC0
:105510002AD50023C8F2010307E04DF61812C2F2A3
:1055200000020023C7F6FF7393614FF23462C2F2A8
:1055300000024EF6041012680192C2F200004DF60D
:1055400050014DF24C72C2F20001C2F20002019C05
:10555000046001208B61107002B0BDEC048B70BD43
:105560000022C8F20102B9E7F0EE487AFEEEC87AEE
:1055700017EE903AD9E70023C7F6FF73D5E700BFCF
:10558000000000000000E03FF0B549F24035C1F6F0
:10559000FF759BB02E781AAB013E06EB8606C3F171
:1055A0006B0303EBC6060DF1FF340DF1270730192D
:1055B00010F0F2FA04F8010FA742F8D140F23C04CF
:1055C000C0F202040FCC0AAE37460FC70FCC0FC78C
:1055D0000FCC0FC794E80F004FF0FF3487E80F009F
:1055E00001A911F8013B83EA04021AA802F00F0294
:1055F00000EB8202B14252F8402C82EA141484EA91
:10560000131303F00F0300EB830353F8403C83EACA
:1056100014146FEA0404E4D140F6A4401321C0F24C
:10562000020013F019FC009E49F2E46000231022EE
:105630003146C1F6FF7010F06DF840F6B840052114
:10564000C0F2020013F008FC49F2E460C1F6FF70FA
:1056500000231022214610F05DF8A6420ED040F63D
:10566000D840C0F20200FBF735F849F2E460C1F619
:10567000FF701BB0BDE8F04010F03AB82E7849F248
:10568000F724C1F6FF74013E06EB8606C4F102035F
:1056900003EBC60604F12807301910F07DFA04F870
:1056A000010FBC42F8D140F6C040C0F20200FBF747
:1056B00007F849F2E460297800230A22C1F6FF7056
:1056C00010F028F8D1E700BF40F6005010B50B21CC
:1056D000C0F2020013F0C0FB49F24033C1F6FF7381
:1056E00049F2E464C1F6FF741978204600230A22C7
:1056F00010F010F820460FF0FBFFBDE81040FFF758
:1057000043BF00BF2DE9F0414FF23466C2F20006FC
:1057100082B04DF6043533680093C1F6FF75009BE7
:105720002A689B1AB3F5487F00F243824DF21804B1
:10573000C1F6FF744EF24050C2F200000CF0FEFFC2
:1057400044F27010C2F20000FEF7C6F923684DF271
:10575000180898420746C1F6FF7800F3A984C0F202
:105760007F849F4227D049F2EF28FBB2C1F6FF7831
:10577000184688F80030FFF7FBFD40F6B850C0F23D
:105780000200FAF79DFF98F80000FAF787FF4CF641
:105790004C314DF2E030C2F20001C2F200000CF0D8
:1057A00055FF4DF2E030C2F200000CF09BFF336871
:1057B0000193019B2B604EF24050C2F20000276023
:1057C0000CF0FAFF002840F04C824DF68805C2F23A
:1057D00000054EF25050C2F200000CF0AFFF44F250
:1057E0009010C2F20000FEF777F906464DF2E03065
:1057F000C2F200000CF046FF854200F023824DF219
:10580000E030C2F200000CF03DFF4BF64423C1F63D
:10581000FF73834200F0E8844DF2E030C2F20000F2
:105820000CF030FF4CF22C23C1F6FF73834200F0E2
:10583000E9844DF2E030C2F200000CF023FF4BF29D
:105840007C13C2F20003834200F024844DF2E03066
:10585000C2F200000CF016FF4CF62013C2F2000357
:10586000834200F00C854DF2E030C2F200000CF0F3
:1058700009FF4DF66C23C2F20003834200F011854C
:105880004DF2E030C2F200000CF0FCFE4CF254533A
:10589000C1F6FF73834200F04A854DF2E030C2F258
:1058A00000000CF0EFFE4CF6CC33C1F6FF738342E0
:1058B00000F0CC844DF2E030C2F200000CF0E2FEC9
:1058C0004BF67803C1F6FF73834200F06A854DF210
:1058D000E030C2F200000CF0D5FE4CF2B403C2F28C
:1058E0000003834200F086854DF2E030C2F20000F2
:1058F0000CF0C8FE4EF26053C2F20003834200F087
:105900009E854DF2E030C2F200000CF0BBFE4BF27F
:105910002C33C2F20003834200F0B6854DF2E03032
:10592000C2F200000CF0AEFE4CF60C23C1F6FF7381
:10593000834200F0CE854DF2E030C2F200000CF060
:10594000A1FE4BF62843C2F20003834200F0E68535
:105950004DF2E030C2F200000CF094FE4CF6FC2355
:10596000C2F20003834200F014864DF2E030C2F22E
:1059700000000CF087FE4BF22C13C2F200038342AE
:1059800000F016864DF2E030C2F200000CF07AFE14
:105990004DF2BC63C2F20003834200F02E864DF24A
:1059A000E030C2F200000CF06DFE4DF28C03C2F24A
:1059B0000003834200F07E864DF2E030C2F2000028
:1059C0000CF060FE4EF60813C2F20003834200F0B2
:1059D00062864DF2E030C2F200000CF053FE4CF64D
:1059E0001003C2F20003834200F046864DF2E0301D
:1059F000C2F200000CF046FE4CF28833C1F6FF7391
:105A0000834200F02A864DF2E030C2F200000CF032
:105A100039FE4BF63453C2F20003834200F0A686EF
:105A20004DF2E030C2F200000CF02CFE4DF21033CB
:105A3000C2F20003834200F001874DF2E030C2F26F
:105A400000000CF01FFE4BF21C03C1F6FF738342F3
:105A500000F0E5864DF2E030C2F200000CF012FEDC
:105A60004CF65063C1F6FF73834200F0C9864DF2D5
:105A7000E030C2F200000CF005FE4BF26C73C1F690
:105A8000FF73834200F0AD864DF2E030C2F20000B9
:105A90000CF0F8FD4DF6BC23C2F20003834200F087
:105AA0003B874DF2E030C2F200000CF0EBFD4CF20F
:105AB0000433C2F20003834200F01F874DF2E0304E
:105AC000C2F200000CF0DEFD4DF64053C2F20003BE
:105AD000834200F003874DF2E030C2F200000CF088
:105AE000D1FD4CF20413C2F20003834200F0AA80FD
:105AF0004DF2E030C2F200000CF0C4FD4EF2B053A3
:105B0000C2F20003834200F0DA864DF2E030C2F2C6
:105B100000000CF0B7FD4DF64833C1F6FF73834229
:105B200000F0BE864DF2E030C2F200000CF0AAFD9B
:105B30004BF26C03C1F6FF73834200F0A2864DF274
:105B4000E030C2F200000CF09DFD4AF2D453C2F2E4
:105B500000038342636800F086864DF218079E4278
:105B6000C1F6FF7700F3798616DA40F61C50C0F2D2
:105B70000200FAF7A5FD49F2E4603146C1F6FF7074
:105B8000FDF772F8F0B23979FDF7E2FF4DF2E0303F
:105B9000C2F200000CF0ACFD4EF25050C2F2000018
:105BA00066600CF009FE002840F0878202B0BDE874
:105BB000F0814DF2E030C2F200000CF063FD4CF2D7
:105BC0007C23C1F6FF7383427FF4B0AD41F218200D
:105BD00044F27017C2F20007C0F20200FAF77AFD31
:105BE00007F12000FDF778FF4CF29828C2F2000878
:105BF0004BF6F01188F827004DF2E030C2F20001B8
:105C0000C2F200000CF022FD4DF2E0300221C2F29F
:105C100000004DF218040CF041FDC1F6FF7498F934
:105C20000030636000220521B96323EAE37387F83B
:105C30003C207A6372B68B42A8BF0B469B00FB6286
:105C400062B677E563689E42A6D049F24033C1F65A
:105C5000FF734DF2E030C2F200001E700CF042FD06
:105C60009AE740F6C850C0F20200FAF729FD4DF25B
:105C7000E030C2F200000CF005FD4DF68805C2F2DE
:105C80000005854200F01F834DF2E030C2F20000B3
:105C90000CF0F8FC4BF2DC23C2F20003834200F06C
:105CA0003B834DF2E030C2F200000CF0EBFC4BF60F
:105CB0004423C1F6FF73834200F047834DF2E03086
:105CC000C2F200000CF0DEFC4CF22C23C1F6FF7394
:105CD000834200F045834DF2E030C2F200000CF048
:105CE000D1FC4BF27C13C2F20003834200F04383E9
:105CF0004DF2E030C2F200000CF0C4FC4CF6201370
:105D0000C2F20003834200F041834DF2E030C2F260
:105D100000000CF0B7FC4DF66C23C2F20003834286
:105D200000F04E834DF2E030C2F200000CF0AAFC0D
:105D30004CF25453C1F6FF73834200F050834DF28E
:105D4000E030C2F200000CF09DFC4CF6CC33C1F602
:105D5000FF73834200F088824DF2E030C2F200000F
:105D60000CF090FC4BF67803C1F6FF73834200F011
:105D700050834DF2E030C2F200000CF083FC4CF294
:105D8000B403C2F20003834200F04E834DF2E030D0
:105D9000C2F200000CF076FC4BF24013C1F6FF7328
:105DA000834200F05B834DF2E030C2F200000CF061
:105DB00069FC4EF26053C2F20003834200F0598343
:105DC0004DF2E030C2F200000CF05CFC4BF22C33E0
:105DD000C2F20003834200F066834DF2E030C2F26B
:105DE00000000CF04FFC4CF60C23C1F6FF7383420D
:105DF00000F064834DF2E030C2F200000CF042FC8F
:105E00004BF62843C2F20003834200F071834DF247
:105E1000E030C2F200000CF035FC4CF6FC23C2F27C
:105E20000003834200F06F834DF2E030C2F20000C5
:105E30000CF028FC4BF22C13C2F20003834200F05A
:105E40007C834DF2E030C2F200000CF01BFC4DF2FE
:105E5000BC63C2F20003834200F07A834DF2E0306B
:105E6000C2F200000CF00EFC4DF28C03C2F20003F3
:105E7000834200F083834DF2E030C2F200000CF068
:105E800001FC4EF60813C2F20003834200F06B835C
:105E90004DF2E030C2F200000CF0F4FB4CF61003BF
:105EA000C2F20003834200F09D834DF2E030C2F263
:105EB00000000CF0E7FB4CF28833C1F6FF7383421D
:105EC00000F085834DF2E030C2F200000CF0DAFB06
:105ED0004BF63453C2F20003834200F0A8834DF224
:105EE000E030C2F200000CF0CDFB4DF21033C2F2F4
:105EF0000003834200F090834DF2E030C2F20000D4
:105F00000CF0C0FB4BF21C03C1F6FF73834200F0A0
:105F100099834DF2E030C2F200000CF0B3FB4CF676
:105F20005063C1F6FF73834200F0D3834DF2E0303B
:105F3000C2F200000CF0A6FB4BF26C73C1F6FF73CB
:105F4000834200F0DC834DF2E030C2F200000CF03E
:105F500099FB4DF6BC23C2F20003834200F0C483D8
:105F60004DF2E030C2F200000CF08CFB4CF2043336
:105F7000C2F20003834200F0EE834DF2E030C2F241
:105F800000000CF07FFB4DF64053C2F20003834249
:105F900000F0D6834DF2E030C2F200000CF072FB4C
:105FA0004CF20413C2F20003834200F0BE834DF2B0
:105FB000E030C2F200000CF065FB4BF28C23C2F221
:105FC0000003834200F0A6834DF2E030C2F20000ED
:105FD0000CF058FB4EF2B053C2F20003834200F0C3
:105FE000F5834DF2E030C2F200000CF04BFB4DF6B1
:105FF0004833C1F6FF73834200F0DD834DF2E03099
:10600000C2F200000CF03EFB4BF26C03C1F6FF73D2
:10601000834200F0C5834DF2E030C2F200000CF084
:1060200031FB4AF2D453C2F20003834200F0AD8345
:106030004DF2E030C2F200000CF024FB4CF6046399
:10604000C2F2000383427FF4C4AB41F20420C0F2E9
:106050000200FAF73FFB0620FDF79EFDFFF7B9BBF4
:1060600040F6AC50C0F20200FAF72AFB49F2E460B5
:106070003946C1F6FF700FF0DDFA49F2E460C1F66F
:10608000FF700FF035FBD8F800309F427FF46BAB08
:10609000FFF791BB63689E423FF47EADF0B2FDF71F
:1060A000DBFE4DF2E030C2F200000CF01BFB73E5AA
:1060B00040F69C50C0F20200D6E740F62850C0F2ED
:1060C0000200FAF707FB4DF2E030C2F200000CF0DC
:1060D000D9FA854200F002814DF2E030C2F20000B0
:1060E0000CF0D0FA4CF20413C2F20003834200F029
:1060F00004814DF2E030C2F200000CF0C3FA4BF222
:10610000DC23C2F20003834200F0C7804DF2E0308E
:10611000C2F200000CF0B6FA4BF24013C1F6FF7366
:10612000834200F0CC804DF2E030C2F200000CF06F
:10613000A9FA4BF28C23C2F20003834200F04B8198
:1061400000252F462E4640F63450C0F20200FAF7E2
:10615000B7FA616849F2E46001312944C1F6FF7081
:106160000FF068FA49F2E460C1F6FF700FF0C0FA70
:1061700040F65050C0F20200FAF7A2FA49F2E46089
:106180006168C1F6FF700FF055FA40F67050C0F22A
:106190000200FAF795FA49F2E460394600230A2230
:1061A000C1F6FF700FF0B6FA49F2E460C1F6FF7075
:1061B0000FF09EFA6168013131444DF2E0304DF24A
:1061C0001804C9B2C2F20000C1F6FF740CF06CFAF8
:1061D00030B36168013131444DF2E030C9B2C2F2EE
:1061E00000000CF067FAE1E463689E423FF4D4AC2F
:1061F000F0B2FDF7C9FD4DF2E030C2F200000CF044
:1062000071FAC9E463689E423FF4C6ACF0B2FDF790
:10621000EFFD4DF2E030C2F200000CF063FABBE497
:1062200040F68850C0F20200FAF74AFA616849F273
:10623000E46001312944C1F6FF700FF0FBF949F227
:10624000E460C1F6FF700FF053FAAFE463689E425A
:106250003FF4A2AC70B2FDF7B3FE4DF2E030C2F2F3
:1062600000000CF03FFA97E440F6BC60C0F2020078
:10627000FAF730FA0D20FDF7C5FCFFF7AABA6368FC
:106280009E423FF489ACF0B2FDF71AFE4DF2E030C9
:10629000C2F200000CF026FA7EE406252F462E46B8
:1062A00051E763689E423FF477AC70B2FDF73CFE65
:1062B0004DF2E030C2F200000CF014FA6CE410254C
:1062C0002F462E463FE740F6E050C0F20200FAF7B4
:1062D00001FA0120FDF760FCFFF77BBA40F60050A1
:1062E000C0F20200FAF7ECF949F2E460C1F6FF707F
:1062F0000FF0FEF9FFF7E8F958E440F6DC10C0F2C1
:106300000200FAF7DDF949F2E460C1F6FF700FF020
:10631000EFF9FDF719FD49E440F6F850C0F202002C
:10632000FAF7D8F90220FDF737FCFFF752BA636895
:106330009E423FF431AC70B2FDF728FE4DF2E030E2
:10634000C2F200000CF0CEF926E440F61060C0F274
:106350000200FAF7BFF90720FDF754FCFFF739BA3E
:1063600040F62C60C0F20200FAF7B4F90820FDF7FD
:1063700049FCFFF72EBA40F64860C0F20200FAF777
:10638000A9F90920FDF73EFCFFF723BA40F6646047
:10639000C0F20200FAF79EF90A20FDF733FCFFF77E
:1063A00018BA63689E423FF4F7ABF0B2FDF740FEC7
:1063B0004DF2E030C2F200000CF094F9FFF7ECBBB4
:1063C00040F68060C0F20200FAF784F90B20FDF776
:1063D00019FCFFF7FEB923252F462E46B3E640F6FB
:1063E0009C60C0F20200FAF775F90C20FDF70AFC78
:1063F000FFF7EFB963689E423FF4CEABF0B2FDF712
:106400004BFE4DF2E030C2F200000CF06BF9FFF7EA
:10641000C3BB40F6D460C0F20200FAF75BF90E206D
:10642000FDF7F0FBFFF7D5B940F6F060C0F20200CF
:10643000FAF750F90F20FDF7E5FBFFF7CAB96368DB
:106440009E423FF4A9ABF0B2FDF75AFE4DF2E030A8
:10645000C2F200000CF046F9FFF79EBB40F6147044
:10646000C0F20200FAF736F90320FDF795FBFFF7BB
:10647000B0B940F62870C0F20200FAF72BF91020EC
:10648000FDF7F6FBFFF7A5B963689E423FF484ABC6
:10649000F0B2FDF769FE4DF2E030C2F200000CF000
:1064A00021F9FFF779BB40F64C70C0F20200FAF711
:1064B00011F91120FDF7DCFBFFF78BB940F66C708A
:1064C000C0F20200FAF706F91220FDF7D1FBFFF740
:1064D00080B963689E423FF45FABF0B2FDF778FE8F
:1064E0004DF2E030C2F200000CF0FCF8FFF754BBB4
:1064F00040F68870C0F20200FAF7ECF81320FDF7BE
:10650000B7FBFFF766B940F6A470C0F20200FAF7D5
:10651000E1F81420FDF7ACFBFFF75BB963689E421E
:106520003FF43AABF0B2FDF787FE4DF2E030C2F235
:1065300000000CF0D7F8FFF72FBB40F6C470C0F294
:106540000200FAF7C7F81520FDF792FBFFF741B9F3
:1065500040F6E070C0F20200FAF7BCF81620FDF732
:1065600087FBFFF736B941F21C00C0F20200FAF7D0
:10657000B1F81820FDF77CFBFFF72BB941F20000C2
:10658000C0F20200FAF7A6F81720FDF771FBFFF73B
:1065900020B963689E423FF4FFAAF0B2FDF798FE6F
:1065A0004DF2E030C2F200000CF09CF8FFF7F4BAB4
:1065B00063689E423FF4F0AAF0B2FDF7D7FE4DF2B9
:1065C000E030C2F200000CF08DF8FFF7E5BA41F2BE
:1065D0005800C0F20200FAF77DF81A20FDF748FBD8
:1065E000FFF7F7B841F23800C0F20200FAF772F88C
:1065F0001920FDF73DFBFFF7ECB863689E423FF4BE
:10660000CBAAF0B2FDF700FF4DF2E030C2F200007D
:106610000CF068F8FFF7C0BA41F29800C0F202002F
:10662000FAF758F81C20FDF723FBFFF7D2B841F228
:106630007800C0F20200FAF74DF81B20FDF718FBB6
:10664000FFF7C7B841F2BC00C0F20200FAF742F807
:106650001D20FDF70DFBFFF7BCB863689E423FF4B9
:106660009BAAF0B2FEF706F84DF2E030C2F200004D
:106670000CF038F8FFF790BA63689E423FF48CAA9A
:10668000F0B2FDF76FFF4DF2E030C2F200000CF007
:1066900029F8FFF781BA63689E423FF47DAAF0B201
:1066A000FDF726FF4DF2E030C2F200000CF01AF8C0
:1066B000FFF772BA63689E423FF46EAAF0B2FDF72C
:1066C000DDFE4DF2E030C2F200000CF00BF8FFF7F7
:1066D00063BA41F2DC00C0F20200F9F7FBFF1E20B2
:1066E000FDF7C6FAFFF775B841F21C10C0F20200C0
:1066F000F9F7F0FF2020FDF7BBFAFFF76AB841F287
:10670000FC00C0F20200F9F7E5FF1F20FDF7B0FA28
:10671000FFF75FB841F28410C0F20200F9F7DAFF28
:106720000520FDF739FAFFF754B841F26C10C0F2BA
:106730000200F9F7CFFF0420FDF72EFAFFF749B862
:1067400041F25410C0F20200F9F7C4FF2220FDF715
:106750008FFAFFF73EB841F23C10C0F20200F9F7A1
:10676000B9FF2120FDF784FAFFF733B863689E4232
:106770003FF412AAF0B2FEF711F84DF2E030C2F287
:1067800000000BF0AFFFFFF707BA41F2EC10C0F2C8
:106790000200F9F79FFF2620FDF7A0FAFFF719B8CE
:1067A00041F2CC10C0F20200F9F794FF2520FDF76A
:1067B00095FAFFF70EB841F2B010C0F20200F9F7F7
:1067C00089FF2420FDF78AFAFFF703B841F29810F9
:1067D000C0F20200F9F77EFF2320FDF77FFAFEF7F3
:1067E000F8BF63689E423FF4D7A9F0B2FEF7B0F855
:1067F0004DF2E030C2F200000BF074FFFFF7CCB9AD
:1068000063689E423FF4C8A9F0B2FEF785F84DF2E6
:10681000E030C2F200000BF065FFFFF7BDB963681E
:106820009E423FF4B9A9F0B2FEF75AF84DF2E030BB
:10683000C2F200000BF056FFFFF7AEB963689E424C
:106840003FF4AAA9F0B2FEF72FF84DF2E030C2F201
:1068500000000BF047FFFFF79FB940F60C50C0F265
:106860000200FFF786B99E423FF496A9F0B2FEF708
:10687000E9F94DF2E030C2F200000BF033FFFFF710
:106880008BB963689E423FF487A9F0B2FEF7BAF96C
:106890004DF2E030C2F200000BF024FFFFF77CB9AC
:1068A00063689E423FF478A9F0B2FEF78DF94DF28D
:1068B000E030C2F200000BF015FFFFF76DB963681E
:1068C0009E423FF469A9F0B2FEF74AF94DF2E0307A
:1068D000C2F200000BF006FFFFF75EB963689E424C
:1068E0003FF45AA9F0B2FEF7F3F84DF2E030C2F2ED
:1068F00000000BF0F7FEFFF74FB963689E423FF4CC
:106900004BA9F0B2FEF79CF84DF2E030C2F2000065
:106910000BF0E8FEFFF740B963689E423FF43CA9E4
:10692000F0B2FEF751F84DF2E030C2F200000BF089
:10693000D9FEFFF731B900BF2DE9F04340F23C0426
:10694000C0F202040FCC91B06D460FC50FCC0FC53D
:106950000FCC0FC594E80F0085E80F0049F2FC2129
:10696000C1F6FF710D1F05F128074FF0FF3411F834
:10697000013B83EA040210A802F00F0200EB82023E
:1069800049F2F82652F8402C82EA141484EA1313D0
:1069900003F00F0300EB8303B94253F8403C83EA52
:1069A0001414C1F6FF766FEA0404E0D140F23C0C07
:1069B000C0F2020CBCE80F00EE46AEE80F00BCE8E7
:1069C0000F00AEE80F00BCE80F004BF68418AEE8ED
:1069D0000F009CE80F00C1F6FF7846F8044B98F8CA
:1069E00000408EE80F00601E00EB8000C0004FF0FA
:1069F000FF3216F8013B83EA020110AC01F00F01EF
:106A000004EB8101BE4251F8401C81EA121282EA75
:106A1000131303F00F0310A901EB830349F2F824C9
:106A200053F8403C83EA1212C1F6FF746FEA020287
:106A3000DFD1C5F1010505EB0009227014F8016BE7
:106A400004EB090528460FF0A7F886423146284690
:106A500001D00FF0BBF8BC42F0D141F23420282124
:106A6000C0F2020012F0F8F949F2E46000230A22B1
:106A700098F80010C1F6FF700EF04CFE41F2602055
:106A80000621C0F2020012F0E7F998F80030013B4D
:106A900003EB8303D90049F2E460023100231022A2
:106AA000C1F6FF700EF036FE49F2E460C1F6FF70E9
:106AB0000EF01EFE002388F8003011B0BDE8F08310
:106AC000F0B549F24035C1F6FF759BB02E781AAB90
:106AD000013E06EB8606C3F16B0303EBC6060DF120
:106AE000FF340DF1270730190FF056F804F8010FA5
:106AF000A742F8D140F23C04C0F202040FCC0AAE27
:106B000037460FC70FCC0FC70FCC0FC794E80F0045
:106B10004FF0FF3487E80F0001A911F8013B83EA29
:106B200004021AA802F00F0200EB8202B14252F8EE
:106B3000402C82EA141484EA131303F00F0300EBD1
:106B4000830353F8403C83EA14146FEA0404E4D14D
:106B500040F6A440C0F20200F9F7B2FD009E49F2EF
:106B6000E460314600231022C1F6FF700EF0D2FD22
:106B700040F6B840C0F20200F9F7A2FD49F2E46025
:106B8000C1F6FF700023102221460EF0C3FDA6427D
:106B90003CD041F2A420C0F20200F9F79BFD4BF675
:106BA0008413C1F6FF732A781A70FFF7C5FE49F205
:106BB000EF24C1F6FF7441F27820C0F20200F9F729
:106BC0007FFD49F2E460217800230A22C1F6FF70BC
:106BD0000EF0A0FD49F2E460C1F6FF700EF088FDF2
:106BE00041F28C20C0F20200F9F76AFD49F2E4603C
:106BF0006321C1F6FF700EF01DFD49F2E460C1F69D
:106C0000FF701BB0BDE8F0400EF072BD4EF2405078
:106C1000C2F200000BF0CEFD18B32D7849F2F72434
:106C2000C1F6FF74013D05EB8505C4F1020303EBDA
:106C3000C50504F1280628190EF0AEFF04F8010F6F
:106C4000B442F8D100200EF0A7FF49F2EF24C1F6BC
:106C5000FF74207041F26820C0F20200F9F730FDA5
:106C6000A9E74EF25050C2F200000BF0A3FD00283D
:106C70008FD0D2E72DE9F8434FF20E69C2F2000936
:106C800041F2F8202DED028BC0F20200F9F718FD59
:106C9000B9F8003007EE103A43F23333C4F223332D
:106CA00008EE903AB8EEC77A43F23333C4F2A33316
:106CB00008EE103A37EE287A49F2E464C7EE087A13
:106CC000C1F6FF744FF20867C2F200074FF20C687A
:106CD000C2F200084FF28C56C2F200064CF61C15A8
:106CE000C2F2000517EE900A14F0FAFC41EC100B0A
:106CF0000A2120460EF04EFD41F20030C0F20200A3
:106D0000F9F7DEFC3B8807EE903AF8EEE77A77EE8B
:106D1000A87A87EE887A17EE100A14F0E1FC41ECAD
:106D2000100B0A2120460EF035FD41F21030C0F262
:106D30000200F9F7C5FCB8F8001020460EF07AFC06
:106D400041F21830C0F20200F9F7BAFC318820464F
:106D50000EF070FC41F22830C0F20200F9F7B0FCEE
:106D6000298820460EF066FC41F24030C0F2020055
:106D7000F9F7A6FC4CF68C33C2F200030A2219681C
:106D8000204600230EF0C6FC41F24C30C0F2020057
:106D9000F9F796FC4CF25053C1F6FF730A221968BA
:106DA000204600230EF0B6FC41F25C30C0F2020037
:106DB000F9F786FC4CF27073C1F6FF730A2219686A
:106DC000204600230EF0A6FC41F26830C0F202001B
:106DD000F9F776FC4BF2CC13C2F20003186805F009
:106DE0000DFE014620460EF025FC20460EF080FCEC
:106DF000BDEC028BB9F80030B8F800203B800023CE
:106E000032802B80BDE8F883F8B50446551E4F1E2E
:106E10002270A57001220025617022712946A5719A
:106E200084F8B950C4F8A050C4F8A450C4F8A850CD
:106E3000C4F8AC50C4F8B050C4F8B450982284F8E8
:106E4000B850E77004F108001E4615F0CDFC022290
:106E5000627120460BF07EF8A579042D0CD805F15F
:106E60002803254444F8236030780BF04BFC85F868
:106E7000B400A3790133A3712046F8BDF8B50446E8
:106E8000551E4F1E2270A5700122002561702271CF
:106E90002946A57184F8B950C4F8A050C4F8A4508C
:106EA000C4F8A850C4F8AC50C4F8B050C4F8B450FA
:106EB000982284F8B850E77004F108001E4615F0D7
:106EC00093FC0222627120460BF044F8A579042D50
:106ED0000DD805F12803254444F8236096F90000F5
:106EE0000BF00EFC85F8B400A3790133A3712046A2
:106EF000F8BD00BFF8B50446551E4F1E2270A570A0
:106F000001220025617022712946A57184F8B950CB
:106F1000C4F8A050C4F8A450C4F8A850C4F8AC50A9
:106F2000C4F8B050C4F8B450982284F8B850E77050
:106F300004F108001E4615F057FC0222627120463B
:106F40000BF008F8A579042D0CD805F1280330467C
:106F500044F823600BF0D8FB254485F8B400A379EE
:106F60000133A3712046F8BDF8B50446551E4F1EE7
:106F70002270A57001220025617022712946A57139
:106F800084F8B950C4F8A050C4F8A450C4F8A8506C
:106F9000C4F8AC50C4F8B050C4F8B450982284F887
:106FA000B850E77004F108001E4615F01DFC0222DF
:106FB000627120460AF0CEFFA579042D0CD805F1A8
:106FC0002803304644F823600BF098FB254485F8ED
:106FD000B400A3790133A3712046F8BD2DE9F04137
:106FE00093F0010807460E46154610D169B1013DE0
:106FF0000024B86C15F8011F036801341B6898471A
:10700000A642F6D8B8F1000F08D1BDE8F081806C37
:107010000368F021DB6C9847002EE8D1B86C036858
:10702000F721DB6CBDE8F041184700BF2DE9F047C0
:107030009DF82040013CE4B20F2C03D84EB2002E44
:107040000D4601DBBDE8F087E0290FD9F729F9D912
:107050000835EDB2012303FA05F515F0DD0FF1D087
:10706000806C0368BDE8F0471B6818478146806C58
:107070001F46036846EA0401C9B21B689046984758
:10708000D9F84800036808F07F011B6805F0EF0598
:107090009847C02DD6D0D9F84800036807F07F0183
:1070A0001B68BDE8F0471847F0B549F2F824C1F66F
:1070B000FF7483B094F821300E461546074623B17D
:1070C000984202D0F9F732FE50B14BF2CC13C2F223
:1070D000000394F90910186831442A4605F092FC1F
:1070E00041F27C30C0F20200162111F0B5FE94F896
:1070F00022303BB34DF650502B4632469021C1F61C
:10710000FF700097FFF792FF2D0640F2A810C0F223
:10711000020005F0FE45F9F7D3FA45F410453604B0
:10712000781E45F0090506F4FE060002354300F41A
:107130007060284311F006F840F2F810C0F2020027
:10714000F9F7BEFA49F2E460C1F6FF7003B0BDE89A
:10715000F0400EF0CDBA00BFF0B549F2F824C1F608
:10716000FF7483B094F821300E461546074623B1CC
:10717000984202D0F9F7DAFD50B14BF2CC13C2F2CB
:10718000000394F90910186831442A4605F03AFCC6
:1071900041F29430C0F20200112111F05DFE94F82A
:1071A00022305BB34DF650502B4632469021C1F64B
:1071B000FF700097FFF73AFF2D0640F2A810C0F2CB
:1071C000020005F0FE45F9F77BFA45F41045360458
:1071D000791E45F0090506F4FE060902354301F45F
:1071E00070614DF66060C2F2000029430DF01EF997
:1071F00040F2B810C0F20200F9F762FA49F2E46016
:10720000C1F6FF7003B0BDE8F0400EF071BA00BFE8
:10721000F0B549F2F824C1F6FF7483B094F8213038
:107220000E461546074623B1984202D0F9F77EFD77
:1072300050B14BF2CC13C2F2000394F90910186854
:107240003144002205F0DEFB41F2A830C0F202001A
:10725000172111F001FE94F822303BB34DF6505047
:107260002B4632468021C1F6FF700097FFF7DEFE05
:107270002D0640F2A810C0F2020005F0FE45F9F715
:107280001FFA45F400453604781E45F0080506F45B
:10729000FE060002354300F47060284310F052FFF0
:1072A00040F2F810C0F20200F9F70AFA49F2E4607D
:1072B000C1F6FF7003B0BDE8F0400EF019BA00BF90
:1072C000F0B549F2F824C1F6FF7483B094F8213088
:1072D0000E461546074623B1984202D0F9F726FD1F
:1072E00050B14BF2CC13C2F2000394F909101868A4
:1072F0003144002205F086FB41F2C030C0F20200AA
:10730000122111F0A9FD94F822305BB34DF65050D4
:107310002B4632468021C1F6FF700097FFF786FEAC
:107320002D0640F2A810C0F2020005F0FE45F9F764
:10733000C7F945F400453604791E45F0080506F402
:10734000FE060902354301F470614DF66060C2F239
:10735000000029430DF06AF840F2B810C0F20200B4
:10736000F9F7AEF949F2E460C1F6FF7003B0BDE889
:10737000F0400EF0BDB900BFF0B549F2F825C1F6F6
:10738000FF7583B095F821300E461446074623B1A9
:10739000984202D0F9F7CAFC48B14BF2CC13C2F2C2
:1073A000000322461868036831465B68984741F23B
:1073B000D430C0F20200122111F04EFD95F82230B7
:1073C0003BB34DF6505023463246B021C1F6FF7014
:1073D0000097FFF72BFE240640F2A810C0F202002F
:1073E00004F0FE44F9F76CF944F430443604781E96
:1073F00044F00B0406F4FE060002344300F470600F
:10740000204310F09FFE40F2F810C0F20200F9F79E
:1074100057F949F2E460C1F6FF7003B0BDE8F040EF
:107420000EF066B9F0B549F2F825C1F6FF7583B0E4
:1074300095F821300E461446074623B1984202D0F3
:10744000F9F774FC48B14BF2CC13C2F200032246A8
:107450001868036831465B68984741F2E830C0F22B
:1074600002000D2111F0F8FC95F822305BB34DF6C7
:10747000505023463246B021C1F6FF700097FFF707
:10748000D5FD240640F2A810C0F2020004F0FE442C
:10749000F9F716F944F430443604791E44F00B042D
:1074A00006F4FE060902344301F470614DF6606093
:1074B000C2F2000021430CF0B9FF40F2B810C0F254
:1074C0000200F9F7FDF849F2E460C1F6FF7003B07D
:1074D000BDE8F0400EF00CB930B5054641F2F83089
:1074E00083B00C46C0F20200122111F0B5FC49F243
:1074F000F823C1F6FF7393F822301BB34DF65050BA
:1075000022460023D021C1F6FF700095FFF78EFDC3
:1075100040F2A810C0F202002404F9F7D1F804F4F4
:10752000FE04681E44F45044000244F00D0400F4CC
:107530007060204310F006FE40F2F810C0F2020026
:10754000F9F7BEF849F2E460C1F6FF7003B0BDE898
:1075500030400EF0CDB800BF30B5054641F20C40CA
:1075600083B00C46C0F202000D2111F075FC49F207
:10757000F823C1F6FF7393F822303BB34DF6505019
:1075800022460023D021C1F6FF700095FFF74EFD83
:1075900040F2A810C0F202002404F9F791F804F4B4
:1075A000FE04691E44F45044090244F00D0401F441
:1075B00070614DF66060C2F2000021430CF036FFAE
:1075C00040F2B810C0F20200F9F77AF849F2E4602C
:1075D000C1F6FF7003B0BDE830400EF089B800BFBF
:1075E00030B5054641F21C4083B00C46C0F20200A3
:1075F000122111F031FC49F2F823C1F6FF7393F820
:1076000022307BB304F500524DF65050C2F3C6133E
:10761000E02102F07F020095C1F6FF70FFF706FD42
:1076200004F30D0440F2A81004F50054C0F2020067
:10763000013DF9F745F82D02200400F4FE0005F4A1
:107640007065054345F46040640440F00E0004F0AA
:10765000FE44204310F076FD40F2F810C0F2020024
:10766000F9F72EF849F2E460C1F6FF7003B0BDE807
:1076700030400EF03DB800BF30B5054641F2304015
:1076800083B00C46C0F202000D2111F0E5FB49F277
:10769000F823C1F6FF7393F822309BB304F5005230
:1076A0004DF65050C2F3C613E02102F07F02009560
:1076B000C1F6FF70FFF7BAFC04F30D0440F2A81006
:1076C00004F50054C0F20200013DF8F7F9FF2D0265
:1076D000210401F4FE0105F470650D4345F4604199
:1076E000640441F00E0104F0FE444DF66060C2F205
:1076F000000021430CF09AFE40F2B810C0F20200E4
:10770000F8F7DEFF49F2E460C1F6FF7003B0BDE8B0
:1077100030400DF0EDBF00BF30B5054641F24040AE
:1077200083B00C46C0F20200122111F095FB49F221
:10773000F823C1F6FF7393F822301BB34DF6505077
:1077400022460023C021C1F6FF700095FFF76EFCB2
:1077500040F2A810C0F202002404F8F7B1FF04F4CC
:10776000FE04681E44F44044000244F00C0400F49B
:107770007060204310F0E6FC40F2F810C0F2020006
:10778000F8F79EFF49F2E460C1F6FF7003B0BDE870
:1077900030400DF0ADBF00BF30B5054641F254405A
:1077A00083B00C46C0F202000D2111F055FB49F2E6
:1077B000F823C1F6FF7393F822303BB34DF65050D7
:1077C00022460023C021C1F6FF700095FFF72EFC72
:1077D00040F2A810C0F202002404F8F771FF04F48C
:1077E000FE04691E44F44044090244F00C0401F410
:1077F00070614DF66060C2F2000021430CF016FE8D
:1078000040F2B810C0F20200F8F75AFF49F2E46003
:10781000C1F6FF7003B0BDE830400DF069BF00BF96
:1078200070B5064641F2644082B00C46C0F20200D8
:107830001721154611F010FB49F2F823C1F6FF732A
:1078400093F8223043B949F2E460C1F6FF7002B008
:10785000BDE870400DF04CBF4DF65050C1F6FF70C2
:1078600000962B462246A021FFF7E0FB41F27C4028
:10787000C0F20200F8F724FF36B140F2F810C0F26F
:107880000200F8F71DFFDEE7681E0002240404F47E
:10789000FE0400F47060204340F4504040F00D00BE
:1078A00010F050FCE9E700BF70B5064641F2884091
:1078B00082B00C46C0F202001221154611F0CCFA3B
:1078C00049F2F823C1F6FF7393F8223053B34DF613
:1078D000505022462B46A021C1F6FF700096FFF7BC
:1078E000A5FB41F27C40C0F20200F8F7E9FE691EF8
:1078F0000902240401F4706104F4FE040C4344F40E
:107900005044310144F00D04C9B24DF66060C2F23A
:10791000000021430CF08AFD40F2B810C0F20200D2
:10792000F8F7CEFE49F2E460C1F6FF7002B0BDE8A0
:1079300070400DF0DDBE00BFF8B50446806C0368F2
:107940001B69984708B90020F8BDA06C03685B6903
:107950009847C3B203F0FB01F929F4D0A26D7AB9BC
:1079600094F84D2084F84F30150666D440B20028B4
:10797000C0F24781002084F84D00A0656065F8BD25
:10798000010633D494F84F10F02904EB020124D0FF
:1079900081F84F30616D4B1E9A4224D394F84F20EA
:1079A000F02AE7D0130600F1C280002094F850308E
:1079B00084F86600032984F8650084F8673000F0D5
:1079C000CD80012384F86800A065606584F8E93003
:1079D000002384F84D300120F8BD81F86930636DD3
:1079E000013B9A42C6D20132A265ACE7A3F1F7018E
:1079F0000829C7D8012505FA01F010F4DD7F40F011
:107A0000CD800029BED194F86930F02BB2D1561C3C
:107A10002244F720370A82F8690084F8676084F806
:107A2000687084F8651084F84D10284684F8663034
:107A300084F8E950A1656165F8BD02F10C05EEB26C
:107A4000012E93D902F0FB0EBEF1F90F8ED0EF2A72
:107A500036D802F0F007802F33D140B2002886DB01
:107A6000012184F84F2084F85030A165EDB2012D3A
:107A700080D9BEF1F90F3FF47DAFEF2A00F29B8071
:107A800002F0F003F12B4ED000F29780B02B43D0E0
:107A90003BD9D02B47D043D9E02B3DD0F02B7FF4FE
:107AA00069AF0021802084F84D1084F8693060654A
:107AB0007F21A36D8B4211D20133A3650020F8BD55
:107AC000174607F0DF06902EC7D007F0BF06A02E9E
:107AD000C3D007F0EF07C02FBFD047E71046F8F735
:107AE000CFFD02F00F020023013294F8501084F809
:107AF000660084F86520012084F8671084F86830F7
:107B0000A365636584F8E900F8BD902B04D0A02B31
:107B100002D0802B7FF42EAF032363650221C8E7D8
:107B2000C02B7FF427AF022363650121C1E7F42A4C
:107B30003FF43BAF1046F8F7A3FD802884F86600B9
:107B400064D102F00F03013394F8505084F8675069
:107B5000032984F8653018BF002501D194F85150ED
:107B600084F8685000230121B028A365636584F878
:107B7000E91007D00AD8902804D0A02802D0802885
:107B80007FF426AF84F84D200120F8BDD028F9D02D
:107B9000E028F7D0C0287FF41BAFF3E7002284F879
:107BA000672084F8682084F8652084F8663084F8BB
:107BB000E9502846F8BD134664E7F82B06D018D8DC
:107BC000F32BB0D0A8D3F62B7FF4D4AE1046F8F741
:107BD00057FD0022012384F8652084F8672084F88B
:107BE000682084F86600A265626584F8E93018466A
:107BF000F8BDFA2BFFF4BEAEFC2BE7D9FE2BE5D285
:107C0000B8E61A468E4603F10C052FE7902898D067
:107C1000B02896D0A02894D0D02892D0E02890D038
:107C2000C0288ED000238FE790F86630F12B7CD0EF
:107C30000ED9FA2B2BD01FD8F32B38D0C0F081806F
:107C4000F62B7AD0F82B40F08B80036BF3B11847FA
:107C5000B02B6ED031D9D02B21D03ED9E02B42D0E1
:107C6000F02B7ED1C3698BB1B0F86710802900F189
:107C7000690028BF80211847FC2B0CD051D3FE2B64
:107C80004BD0FF2B6BD1436C002BE0D17047436B83
:107C9000002BDCD1FAE7C36B002BD8D1F6E74369A0
:107CA000002BF3D090F8671090F865001847836AAE
:107CB000002BEBD090F867001847902B29D0A02B11
:107CC00023D0802BE2D10368002BDFD090F868200E
:107CD00090F8671090F865001847C02B42D10369EF
:107CE000002BDFD1D2E78269002ACFD090F868104C
:107CF00090F8673090F86500C90101F47E5103F0F7
:107D00007F031943A1F5005110478368002BDDD193
:107D1000BCE74368002BD9D1B8E7036C002B96D1A0
:107D2000B4E7836B002B92D1B0E7036A002BC1D17B
:107D3000ACE7C368002BC9D1A8E7C36A002B86D182
:107D4000A4E7426A002AA1D090F8683090F8670052
:107D5000DB0103F47E5300F07F00184310477047A7
:107D600070477047704700BF90F86430DA0725D538
:107D700013F0FE0F22D070B590F8665085F08002A7
:107D8000602A82B004461AD9F62D66D05FD8F12D4C
:107D900076D04FD9F22D2DD0F32D1AD1806C94F8D6
:107DA0006760036829461B689847A06C0368DB6C12
:107DB00006F07F0102B0BDE870401847704790F8A8
:107DC00065608E4207D031B15B08012B08D0032BD0
:107DD00027D002B070BD5B08012B01D0022BF8D177
:107DE00094F8683094F86720009629462046FFF7FB
:107DF0001DF9EEE7806C94F86730026894F86860CB
:107E00001268294643EAC6159047A06C036805F03E
:107E10007F019B6C9847A06C0368C5F3C6119B6CEF
:107E2000C8E794F8683094F8672000962946FFF771
:107E3000FDF8CEE7F02DCCD1B0F86710802900F125
:107E4000690228BF80210123FFF7C8F8C1E7FC2D94
:107E500026D8FA2D01D2F82DBBD105F10803DBB2EB
:107E6000072BB6D8012202FA03F313F0DD0FB0D0CE
:107E7000A06C03681B68294602B0BDE87040184733
:107E8000806C94F8672094F86830066812012946DF
:107E900003F00F0302F0700532681D439047E7E7D7
:107EA000FE2D96D3D9E700BFF0B54CF62C3087B045
:107EB000C1F6FF7007F066FC00287FD14FF23464F2
:107EC000C2F200044DF65055C1F6FF7595F84C60AE
:107ED000102E1CD9002010F0D7FB0BF0ADFC4DF696
:107EE00060600021C2F200000CF098FB4DF220030C
:107EF00022680392C1F6FF73039A1868121A4FF2B0
:107F00003461642AC2F200011ED807B0F0BD2846D1
:107F1000FFF712FD0028DDD095F86630902B00F0B9
:107F2000358183F08003602B40F233814DF6505051
:107F3000C1F6FF70FFF778FE4DF650503146C1F69E
:107F4000FF70FFF711FFC5E70A680492049A1A60F0
:107F5000FDF7D8FB4BF68413C1F6FF731B78002B9B
:107F600040F024814DF24C73C2F200031A78002ACB
:107F7000CBD04EF6041122680592C2F20001059A98
:107F8000086841F28831121A8A42BED949F2EF22BA
:107F9000C1F6FF720024204615781C700DF0FCFD20
:107FA000854203D0294620460DF010FE41F2D42030
:107FB000C0F20200F8F78EFB07B0F0BD4CF66C1073
:107FC000C1F6FF7007F0DEFB00283FF477AF4DF6F7
:107FD000F016C1F6FF760EF0A7FB3368C01A4FF219
:107FE0003464B0F5356FC2F200047FF66BAF4DF22A
:107FF00050750EF099FBC2F20005236801932A68C0
:10800000019B30609B1A41F28832934200F2DB8080
:108010004CF62C30C1F6FF7007F0C4FB0646002872
:1080200000F0D8804CF66C10C1F6FF7007F0BAFB78
:108030000746002800F0D5800EF076FB4BF2CC13FB
:10804000C2F200030546186803683A461B683146C9
:1080500098470EF069FB40F65A33401B984206D908
:108060004CF68C33C2F200031A6801321A604CF6E7
:108070001C13C2F200031A88824238BF188072B6FD
:108080004CF23423C2F200031A7F02F0FF010AB15E
:1080900000221A7762B679B372B647F6FF754FF4CD
:1080A0000040B3F91E10B3F92020DD83188462B6B6
:1080B000002982EAE273A3EBE273B8BF49428B4224
:1080C000B8BF0B4607EE903A4FF47E43C4F2FF630D
:1080D000F8EEE77A06EE903A87EEA67AF7EE007AA7
:1080E000B4EEE77AF1EE10FA06DD4CF27073C1F6E9
:1080F000FF731A6801321A6072B64CF25413C2F25E
:1081000000031A7F02F0FF010AB100221A7762B65B
:1081100079B372B647F6FF754FF40040B3F91E10FD
:10812000B3F92020DD83188462B6002982EAE27365
:10813000A3EBE273B8BF49428B42B8BF0B4607EED0
:10814000903A4FF47E43C4F2FF63F8EEE77A06EE0E
:10815000903A87EEA67AF7EE007AB4EEE77AF1EE7F
:1081600010FA06DD4CF27073C1F6FF731A68013223
:108170001A604CF62C30C1F6FF7007F025FB4CF668
:108180006C10C1F6FF7007F01FFB9BE695F8683096
:1081900043B195F865309E423FF4C8AE002E3FF4DF
:1081A000C5AEC9E6802385F86630F2E74BF2CC1302
:1081B000C2F20003186804F021FC00287FF4D2AE5C
:1081C000FEF7BAFBCEE6FEF755FD23680293029B4D
:1081D0002B601DE741F29C40C0F20200F8F77AFAEA
:1081E00020E741F2C440C0F20200F8F773FA23E737
:1081F0002DE9F04F4CF210448FB0C2F2000444F26B
:108200007016C2F200060DF075FC02232046102203
:108210002721002509F0C2FA4FF060496FF060484D
:108220003046022203214EF24057FBF715FCC2F202
:108230000007C6F81490C6F81880357706F12000BC
:108240001D221C21FBF708FCC6F83490C6F83880C4
:1082500086F83C503846142204210AF057FA07F1F8
:10826000100014221E210AF051FA4FF23463C2F2B8
:1082700000034DF604321B680A93C1F6FF720A9997
:10828000116040F2D8034DF2D0302A46C0F202030A
:108290000121C1F6FF70FEF767FE012240F2E40300
:1082A0004DF28C401146C0F20203C1F6FF70FEF79A
:1082B0005BFE012241F278634DF248501146C0F254
:1082C0000203C1F6FF70FEF74FFE012240F2F003F9
:1082D0004DF204601146C0F20203C1F6FF70FEF7D2
:1082E00043FE012240F2FC034DF2C0601146C0F291
:1082F0000203C1F6FF70FEF737FE012240F20413BD
:108300004DF27C70C0F202031146C1F6FF70FEF719
:108310002BFE4EF27870C2F200000AF0AFF84BF676
:10832000F01021460122C2F2000009F095FF41F64B
:1083300024034BF678002A46C0F202030121C2F260
:10834000000049F24037FEF70FFEC1F6FF77012229
:108350004CF260403B461146C2F20000FEF754FD6D
:108360004DF68800C2F200000AF088F84AF68C2028
:1083700021460122C2F2000009F06EFF41F2706353
:108380004AF25C402A46C0F202030121C2F2000018
:10839000FEF7EAFD012241F68C034AF2185011461D
:1083A000C0F20203C2F20000FEF7DEFD012241F638
:1083B00094034BF270001146C0F20203C2F20000B7
:1083C000FEF7D2FD012241F2D4734AF22460114635
:1083D000C0F20203C2F20000FEF7C6FD012241F620
:1083E000A0034AF2E0601146C0F20203C2F20000AC
:1083F000FEF7BAFD012241F6B0034AF29C70114625
:10840000C0F20203C2F20000FEF7AEFD012241F607
:10841000BC034AF658001146C0F20203C2F2000043
:10842000FEF7A2FD012241F6C4034AF614101146DC
:10843000C0F20203C2F20000FEF796FD012241F6EF
:10844000CC034AF6D010C0F202031146C2F200007B
:10845000FEF78AFD4BF2DC20C2F200000AF00EF8B3
:108460004CF2A45021460122C1F6FF7009F0F4FE3F
:1084700041F61C034BF24C202A46C0F202030121B4
:10848000C1F6FF7049F2F826C1F6FF76FEF76CFDE3
:1084900001224BF20830331D1146C1F6FF70FEF782
:1084A000B3FC4BF64420C1F6FF7009F0E7FF4BF632
:1084B000E83021460122C2F2000009F0CDFE40F270
:1084C0000C134DF214302A46C0F202030121C1F60A
:1084D000FF70FEF749FD01224BF21040731D11465B
:1084E000C2F20000FEF790FC4CF22C20C1F6FF70A7
:1084F00009F0C4FF4CF62C1021460122C1F6FF7092
:1085000009F0AAFE41F640034BF608502A46C0F295
:1085100002030121C1F6FF70FEF726FD01224BF692
:10852000C450B31D1146C1F6FF70FEF76DFC4BF24F
:108530007C10C2F2000009F0A1FF4DF690602146C8
:108540000122C1F6FF7009F087FE41F2AC634DF6DF
:1085500078002A46C0F202030121C1F6FF70FEF73F
:1085600003FD01224DF63410F31D1146C1F6FF70D4
:10857000FEF74AFC4CF62010C2F2000009F07EFF24
:108580004BF27C3021460122C2F2000009F064FE69
:1085900041F684034DF2DC002A46C0F202030121B9
:1085A000C2F20000FEF7E0FC01224DF2981006F145
:1085B00008031146C2F20000FEF760FC4DF66C2085
:1085C000C2F2000009F05AFF4CF2C42021460122F9
:1085D000C2F2000009F040FE41F254634BF2007019
:1085E0002A46C0F202030121C2F20000FEF7BCFCE1
:1085F00001224BF6D42006F109031146C1F6FF70A3
:10860000FEF73CFC4CF25450C1F6FF7009F036FF07
:108610004DF6100021460122C2F2000009F01CFEB6
:1086200041F66C034CF2D8302A46C0F20203012115
:10863000C1F6FF70FEF798FC012240F2FD534CF2A8
:108640009440C0F200031146C1F6FF70FEF752FCE1
:108650004CF6CC30C1F6FF7009F010FF4BF23C40F5
:1086600021460122C1F6FF7009F0F6FD41F2C06318
:108670004BF63C702A46C0F202030121C2F2000010
:10868000FEF772FC01224BF6F87006F10B0311465F
:10869000C2F20000FEF7B8FB4BF67800C1F6FF709F
:1086A00009F0ECFE4DF6380021460122C1F6FF70BC
:1086B00009F0D2FD41F208734DF288402A46C0F21B
:1086C00002030121C2F20000FEF74EFC01224DF62A
:1086D000905006F10C031146C2F20000FEF794FB25
:1086E0004CF2B400C2F2000009F0C8FE4DF6D8000A
:1086F00021460122C2F2000009F0AEFD41F67013DE
:108700004BF680602A46C0F202030121C1F6FF70D9
:10871000FEF72AFC012241F680134BF63C7011460D
:10872000C0F20203C1F6FF70FEF71EFC012241F207
:1087300024734BF6F8701146C0F20203C1F6FF70C5
:10874000FEF712FC012241F248634CF2B4001146DC
:10875000C0F20203C1F6FF70FEF706FC012241F2EF
:1087600030734CF270101146C0F20203C1F6FF7074
:10877000FEF7FAFB012240F27C034AF6C4401146A0
:10878000C0F20203C2F20000FEF7EEFB012240F24B
:1087900088034AF63C601146C0F20203C2F20000B0
:1087A000FEF7E2FB012241F250734AF6F8601146EF
:1087B000C0F20203C2F20000FEF7D6FB012241F232
:1087C00060734AF6B4701146C0F20203C2F20000B0
:1087D000FEF7CAFB012241F2DC734CF6A0601146A1
:1087E000C0F20203C1F6FF70FEF7BEFB012241F6A4
:1087F00050134CF65C701146C0F20203C1F6FF70D4
:10880000FEF7B2FB012241F2EC734CF21C50114610
:10881000C0F20203C2F20000FEF7A6FB012241F6FD
:1088200060134CF218601146C0F20203C2F200005D
:10883000FEF79AFB012241F26C734DF224001146BF
:10884000C0F20203C1F6FF70FEF78EFB012241F277
:10885000F8734DF2E0001146C0F20203C1F6FF705A
:10886000FEF782FB012241F288734DF29C10114603
:10887000C0F20203C1F6FF70FEF776FB012241F25F
:10888000C4734DF258201146C0F20203C1F6FF70C6
:10889000FEF76AFB012241F608034CF66000114620
:1088A000C0F20203C2F20000FEF75EFB012241F6B5
:1088B00010034BF28850C0F202031146C2F20000CE
:1088C000FEF752FB4BF24010C1F6FF7009F0D6FDE7
:1088D0004EF2C87021460122C2F2000009F0BCFC31
:1088E00041F65C034AF608402A46C0F20203012121
:1088F000C2F20000FEF738FB01224BF2901006F1A5
:108900000D031146C1F6FF70FEF77EFA4EF260507D
:10891000C2F2000009F0B2FD4BF2D0302146012234
:10892000C2F2000009F098FC41F2D8634DF65010F5
:108930002A46C0F202030121C2F20000FEF714FB36
:1089400001224CF2543006F10E031146C2F200002F
:10895000FEF75AFA4BF22C30C2F2000009F08EFDFD
:108960004DF20C0021460122C2F2000009F074FC15
:1089700040F2BC034DF244502A46C0F202030121EA
:10898000C2F20000FEF7F0FA01224DF2006006F19B
:108990000F031146C2F20000FEF736FA4CF60C2027
:1089A000C1F6FF7009F06AFD4CF2D8502146012251
:1089B000C2F2000009F050FC40F298034BF2F45070
:1089C0002A46C0F202030121C1F6FF70FEF7CCFA7D
:1089D000012240F26D434BF2B060C0F20003114639
:1089E000C1F6FF70FEF786FA4BF62840C2F200008F
:1089F00009F044FD4CF2204021460122C2F2000061
:108A000009F02AFC41F6E4034BF6C4502A46C0F2B2
:108A100002030121C2F20000FEF7A6FA012240F291
:108A20008D434BF68060C0F200031146C2F2000095
:108A3000FEF760FA4CF6FC20C2F2000009F01EFDC1
:108A40004DF6083021460122C1F6FF7009F004FC02
:108A500040F2B0034DF648202A46C0F2020301213D
:108A6000C1F6FF70FEF780FA012240F2AD434CF2EE
:108A7000CC20C0F200031146C1F6FF70FEF73AFAAF
:108A80004BF22C10C2F2000009F0F8FC4BF69420D7
:108A900021460122C1F6FF7009F0DEFB41F62013EA
:108AA0004BF2D0102A46C0F202030121C2F20000AC
:108AB000FEF75AFA012240F229534CF67000C0F238
:108AC00000031146C1F6FF70FEF714FA4DF2BC60C8
:108AD000C2F2000009F0D2FC4DF6F410214601224A
:108AE000C1F6FF7009F0B8FB41F630134DF6C830FF
:108AF0002A46C0F202030121C2F20000FEF734FA56
:108B0000012240F275534DF68440C0F20003114635
:108B1000C2F20000FEF7EEF94DF28C00C2F2000046
:108B200009F0ACFC4AF6C83021460122C2F200002E
:108B300009F092FB40F2A4034CF684102A46C0F2DE
:108B400002030121C2F20000FEF70EFA012240F2F8
:108B5000B9534CF64020C0F200031146C2F20000A7
:108B6000FEF7C8F94EF60810C2F2000009F086FCC4
:108B70004BF2001021460122C1F6FF7009F06CFB98
:108B800041F238634CF61C402A46C0F20203012130
:108B9000C1F6FF70FEF7E8F901224CF6D03006F17D
:108BA00016031146C2F20000FEF72EF94CF6100033
:108BB000C2F2000009F062FC4DF62C202146012291
:108BC000C2F2000009F048FB41F630034BF2BC70E2
:108BD0002A46C0F202030121C1F6FF70FEF7C4F974
:108BE00001224BF6C80006F117031146C1F6FF70CB
:108BF000FEF70AF94CF28830C1F6FF7009F03EFC2E
:108C00004DF24C0021460122C2F2000009F024FB83
:108C100040F2C8034BF27C402A46C0F20203012115
:108C2000C1F6FF70FEF7A0F901224BF2385006F1B1
:108C300018031146C1F6FF70FEF7E6F84BF6345004
:108C4000C2F2000009F01AFC4CF258202146012221
:108C5000C2F2000009F000FB41F674034CF68C40B0
:108C60002A46C0F202030121C2F20000FEF77CF99D
:108C700001224CF6485006F119031146C2F20000D9
:108C8000FEF7C2F84DF21030C2F2000009F0F6FB18
:108C90004CF6903021460122C2F2000009F0DCFAC5
:108CA00041F298734BF688102A46C0F20203012164
:108CB000C1F6FF70FEF758F901224AF6805006F11E
:108CC0001A031146C2F20000FEF79EF84BF21C0098
:108CD000C1F6FF7009F0D2FB4DF654402146012247
:108CE000C1F6FF7009F0B8FA41F280634CF2F85017
:108CF0002A46C0F202030121C1F6FF70FEF734F9E3
:108D000001224CF2B46006F11B031146C1F6FF705C
:108D1000FEF77AF84CF65060C1F6FF7009F0AEFB32
:108D20004CF2D07021460122C2F2000009F094FA00
:108D300041F29C634CF694602A46C0F20203012182
:108D4000C2F20000FEF710F901224DF6983006F14C
:108D50001C031146C1F6FF70FEF756F84BF26C701B
:108D6000C1F6FF7009F08AFB4EF6C40021460122CD
:108D7000C2F2000009F070FA41F610134AF6CC2056
:108D80002A46C0F202030121C2F20000FEF7ECF80D
:108D900001224BF2CC4006F11D031146C2F2000045
:108DA000FEF732F84DF6BC20C2F2000009F066FB77
:108DB0004CF6546021460122C2F2000009F04CFA40
:108DC00041F6DC034EF608002A46C0F202030121F8
:108DD000C2F20000FEF7C8F801224DF2542006F15D
:108DE0001E031146C2F20000FEF748F84CF20430B0
:108DF000C2F2000009F042FB4DF63C602146012220
:108E0000C1F6FF7009F028FA41F604134CF65C2015
:108E10002A46C0F202030121C1F6FF70FEF7A4F852
:108E200001224CF6507006F11F031146C2F20000F9
:108E3000FEF724F84DF64050C2F2000009F01EFB88
:108E40004AF6883021460122C2F2000009F004FAF5
:108E500041F290634EF200602A46C0F20203012103
:108E6000C2F20000FEF780F801224EF2BC603B46E1
:108E70001146C2F20000FDF7C7FF4CF20410C2F227
:108E8000000009F0FBFA4BF6302021460122C2F225
:108E9000000009F0E1F941F218734BF244602A46F0
:108EA000C0F202030121C2F20000FEF75DF80122C8
:108EB00041F2E8634BF2BC701146C0F20203C2F209
:108EC0000000FEF751F8012241F2F8634DF694409C
:108ED0001146C0F20203C1F6FF70FEF745F8012209
:108EE00041F6F4034BF63410C0F202031146C2F20D
:108EF0000000FEF739F84BF28C20C2F2000009F0B6
:108F0000BDFA4BF6845021460122C2F2000009F05E
:108F1000A3F941F27C734BF64C402A46C0F202039F
:108F20000121C1F6FF70FEF71FF801224BF69030C9
:108F300006F120031146C1F6FF70FDF765FF4EF202
:108F4000B050C2F2000009F099FA4DF20C702146BF
:108F50000122C2F2000009F07FF941F240734BF6A2
:108F60007840C0F2020300220121C2F20000FDF7A6
:108F7000FBFF012240F231634CF2D460C0F20003E7
:108F80001146C2F20000FDF7B5FF4DF64830C1F6BC
:108F9000FF7009F073FA4DF2603021460122C2F2EF
:108FA000000009F059F941F64C034CF6D840C0F2E4
:108FB000020300220121C1F6FF70FDF7D5FF012257
:108FC00040F2D1434CF69450C0F200031146C1F672
:108FD000FF70FDF78FFF4BF26C00C1F6FF7009F0D8
:108FE0004DFA4BF2C00021460122C1F6FF7009F094
:108FF00033F941F640134BF67020C0F20203002211
:109000000121C2F20000FDF7AFFF01224BF62C3028
:1090100006F123031146C2F20000FDF7F5FE4AF205
:10902000D450C2F2000009F029FA4DF2A0302146D6
:109030000122C2F2000009F00FF9002241F2A873E8
:109040004CF278101146C0F20203C2F20000FDF7A4
:109050008BFF41F2B8734CF2B470C0F202030122EC
:109060000021C1F6FF70FDF77FFF4CF60460C2F2ED
:10907000000009F003FA4CF2907021460122C2F27E
:10908000000009F0E9F841F260634DF25470C0F25B
:10909000020300220121C2F20000FDF765FF012258
:1090A00049F2EF234DF60C30C1F6FF731146C2F2C0
:1090B0000000FDF7A9FE4CF27C20C1F6FF7009F01C
:1090C000DDF94CF64C3021460122C2F200004DF68B
:1090D0005059C1F6FF7909F0BFF84DF2E030012197
:1090E000C2F2000009F098FA99F86430012243F0C6
:1090F000010362F3470349F2A025002489F8643094
:1091000049F214562B464FF6FF7E214689F86540FA
:1091100089F8664089F8674089F8684089F8E9402D
:10912000C1F6FF73C1F6FF7609F1690080221D4682
:10913000C9F85CE0C9F860E0C9F8486089F84C40BB
:1091400089F84D4089F84E40C9F85440C9F8584054
:109150004DF6606613F048FB40F225514CF62C3377
:10916000C2F200062A46C1F6FF734846C0F200016B
:1091700040F2900A0195C9F800401D46C9F8044024
:10918000C9F80840C9F80C40C9F81040C9F81440A3
:10919000C9F81840C9F81C40C9F82040C9F8244053
:1091A000C9F82840C9F82C40C9F83040C9F8344003
:1091B000C9F83840C9F83C40C9F84040C9F84440B3
:1091C000C0F20F0A12F09CFF06F5A36C06F5AB6E19
:1091D00006F5B361502306F59B694022C6F818C016
:1091E000C6F81CE0B38574603046B460C6F800A0D1
:1091F000C6F81490716272850BF0D4F84CF23422E8
:10920000029240F22802C0F2020232602146224657
:109210002846F9F733FD029A85F89C404CF66C1B02
:10922000C1F6FF7BC2F200024FF62C784CF25413C9
:10923000C2F20003C0F20E080292214622465846AE
:109240000393C5F8984085F89D400695C5F80080C1
:10925000F9F714FD02998BF89C4044F2BC100A46C1
:1092600089460546183208460121CBF80080CBF824
:1092700098408BF89D40F9F701FD0399CDF80890CF
:10928000C2F200054DF6D06307950A464DF6D0654B
:109290004FF6D0578A461832C0F20E0747F6FF76CF
:1092A0004FF40048059508461D460121C9F8007095
:1092B000A9F81E60A9F82080C1F6FF75F9F7DEFC59
:1092C0004DF618190798CAF80070C2F20009AAF8FA
:1092D0001E60CDF80CA0AAF8208005F04FFD4DF6D9
:1092E000500A2846C2F2000A05954CF2747705F040
:1092F00045FD4FF6147609F12802484604214CF248
:109300009475F9F7BBFC4FF48033C1F6FF77C0F2D8
:109310000E060AF1280250460421C1F6FF75C9F86D
:109320000060C9F81830C9F81C30C9F82030C9F8F5
:10933000243008930495F9F7A1FC089BCAF8006053
:1093400007F11C02384601213D46CAF81830CAF818
:109350001C30CAF82030CAF82430F9F78FFC049F7B
:10936000089BAB6107F11C02089538462F464FF663
:109370000875C0F20E05012109933D604DF63428B1
:10938000F9F77CFC0499099B029A0D60C1F6FF78FD
:1093900040F22566C0F20006069D8B6140464BF206
:1093A000C437C1F6FF77C8F80420C8F8005088F821
:1093B000084088F80940C8F80C4088F810400BF0C5
:1093C00059FD019A314640464BF2D83812F098FECA
:1093D000C1F6FF78039979603846C7F800B03C724F
:1093E0007C72FC603C740BF045FD019A31463846B6
:1093F00012F086FE4BF2EC3740460695C8F8005056
:10940000079DC8F80450C1F6FF7788F8084088F82F
:109410000940C8F80C4088F810400BF02BFD31468D
:10942000019A404612F06CFE059AC7F800B0384623
:109430007A603C727C72FC603C744BF200480BF02A
:1094400019FD019A3146384612F05AFEC1F6FF78EE
:10945000069B88F8084040464BF2144788E808020B
:10946000C1F6FF7788F80940C8F80C4088F810402A
:109470000BF000FD019A3146404612F041FE38469D
:10948000C7F800B0C7F804A03C727C72FC603C7462
:109490000BF0F0FCDDF804B04BF22848C1F6FF7881
:1094A0005A463146384612F02BFE294640464FF0C8
:1094B000010588E8020288F8084088F80950C8F8D1
:1094C0000C4088F810404DF67C670BF0D3FC5A46F0
:1094D0003146404612F014FEC1F6FF77059B3C7200
:1094E00038464CF2E458C1F6FF7887E808047D72EC
:1094F000FC603C740BF0BEFC5A463146384612F014
:10950000FFFD4BF2BC37089BC8F804304046C2F25E
:109510000007C8F8009088F8084088F80940C8F8A3
:109520000C4088F810400BF0A5FC5A4631464046E6
:1095300012F0E6FD4DF60C28049DC7F800A0384651
:10954000C2F200087D603C727C72FC603C740BF0DF
:1095500091FC5A463146384612F0D2FD08F1180205
:1095600002214046F9F78AFB4FF62073C0F20E0342
:1095700040464CF61839C1F6FF79C8F8003005F0BE
:1095800081FF089B89F8084048464CF67017C2F2E4
:10959000000789E8080189F80940C9F80C4089F8F2
:1095A00010400BF067FC31465A46484612F0A8FDC1
:1095B0002A464FF00103384687E804017B723C726B
:1095C000FC603C740BF056FC31465A46384612F0AB
:1095D00097FD44F2B013C2F200034FF6DC52C0F222
:1095E0000E021A600A221A720DF09EF84FF23463CE
:1095F000C2F200034DF6F0151A680B92DDF82CC08C
:109600001A680C92DDF830E01B680D934DF22004CF
:109610004EF604114DF250724BF2BC03C1F6FF75C9
:10962000C1F6FF74C2F20001C2F200020D9F286071
:10963000C1F6FF734DF66266C3F64E76C4F800C0FD
:10964000C1F800E017601E600FB0BDE8F08F00BFEA
:109650002DE9F04F4CF21044C2F2000493B02046C2
:1096600008F066FC204608F00BFA204608F000FAE5
:10967000204608F0A3F8204608F0E6FA204600222B
:10968000012108F0D1F941F2EC412046C0F202017B
:109690000E220BF0B9FF20460122002108F0C4F988
:1096A00041F2FC411022C0F2020120464DF2D03AB4
:1096B0004EF278740BF0A8FFC2F20004C1F6FF7AF4
:1096C0004FF47A704DF28C490DF056F8C1F6FF79DF
:1096D000514620464DF2485808F0D8FEC1F6FF78B2
:1096E000494620464DF2046708F0D0FEC1F6FF77E8
:1096F000414620464DF2C06608F0C8FEC1F6FF762E
:10970000394620464DF27C7508F0C0FEC1F6FF7563
:109710003146204608F0BAFE4BF6F01329462046A3
:10972000019308F0B3FE019B2046C2F20003022120
:10973000019308F0E1FE2146019808F099FD41F6F9
:10974000CD725046C0F20002012108F005FC42F63D
:10975000AD324846C0F20002022108F0FDFB40F69F
:1097600069424046C0F20002032108F0F5FB41F6D1
:10977000BD623846C0F20002042108F0EDFB42F65B
:10978000F1223046C0F20002052108F0E5FB40F668
:109790001D02C0F20002284606214DF6880408F09A
:1097A000DBFBC2F200044BF678012046C2F2000156
:1097B00008F06CFE4AF68C224CF2604115462046B9
:1097C000C2F2000108F062FE2A46C2F2000216460A
:1097D0004AF25C4220461746022108F08DFE3A46C6
:1097E000C2F200024BF2DC25C2F200051746214608
:1097F00030464AF2185B0F96C2F2000B08F038FDB3
:109800004BF2700A394628460497C2F2000A08F063
:109810003DFE4AF224695946284608F037FEC2F256
:109820000009514628464AF2E06808F02FFEC2F2CD
:1098300000084946284608F029FE4AF29C7741462E
:10984000284608F023FEC2F200074AF614123946F1
:10985000144628464AF6580608F018FEC2F20006DA
:109860002246C2F20002314628464AF6D01403923C
:10987000C2F2000408F00AFE0399284608F006FE2A
:109880004CF2A45321462846029308F0FFFD029BA8
:109890002846C1F6FF730221029308F02DFE2946E7
:1098A000029808F0E5FC41F2FD320498C0F2000293
:1098B000072108F051FB41F285025846C0F2000230
:1098C000082108F049FB41F215625046C0F200023F
:1098D000092108F041FB41F6A5224846C0F20002EA
:1098E0000A2108F039FB41F295724046C0F20002AD
:1098F0000B2108F031FB41F2FD423846C0F2000274
:109900000C2108F029FB41F619023046C0F2000292
:109910000D2108F021FB41F215720398C0F20002FC
:109920000E2108F019FB41F6A502C0F20002204604
:109930000F214BF6442508F00FFBC1F6FF754BF2E3
:109940004C212846C1F6FF7108F0A0FD4BF6E83225
:109950004BF2083114462846C1F6FF7108F096FD17
:109960002246C2F2000217462846022108F0C4FD32
:109970004CF22C2429463846C1F6FF74109708F0A3
:1099800077FC4DF214312046C1F6FF7108F07EFDE0
:109990004BF210412046C2F2000108F077FD20464C
:1099A000022108F0A9FD4CF62C102146C1F6FF70EB
:1099B0004BF27C1408F05CFCC2F200044BF6085138
:1099C0002046C1F6FF7108F061FD4BF6C4512046F8
:1099D000C1F6FF7108F05AFD2046022108F08CFD07
:1099E0004DF690602146C1F6FF704CF6201408F049
:1099F0003FFCC2F200044DF678012046C1F6FF712B
:109A000008F044FD4DF634112046C1F6FF7108F010
:109A10003DFD2046022108F06FFD4BF27C302146CF
:109A2000C2F200004DF66C2408F022FCC2F20004E1
:109A30004DF2DC012046C2F2000108F027FD4DF294
:109A400098112046C2F2000108F020FD20460221B4
:109A500008F052FD4CF2C4202146C2F200004CF244
:109A6000545408F005FCC1F6FF744BF20071204617
:109A7000C2F2000108F00AFD4BF6D4212046C1F6DF
:109A8000FF7108F003FD2046022108F035FD4DF678
:109A900010002146C2F200004CF6CC3408F0E8FB7E
:109AA000C1F6FF744CF2D8312046C1F6FF7108F0C0
:109AB000EDFC4CF294412046C1F6FF7108F0E6FC43
:109AC0002046022108F018FD4BF23C402146C1F629
:109AD000FF704BF6780408F0CBFBC1F6FF744BF631
:109AE0003C712046C2F2000108F0D0FC4BF6F87140
:109AF0002046C2F2000108F0C9FC2046022108F00D
:109B0000FBFC4DF638002146C1F6FF704CF2B40460
:109B100008F0AEFBC2F200044DF288412046C2F2CA
:109B2000000108F0B3FC4DF690512046C2F200014E
:109B300008F0ACFC2046022108F0DEFC4DF6D8000F
:109B40004BF680632146C1F6FF73C2F20000039317
:109B50004BF2401408F08CFB039B1193C1F6FF7489
:109B60004BF63C7B1946C1F6FF7B20464BF6F87A54
:109B700008F08CFCC1F6FF7A594620464CF2B40935
:109B800008F084FCC1F6FF79514620464CF270186B
:109B900008F07CFCC1F6FF78494620464AF6C447E7
:109BA00008F074FCC2F20007414620464AF63C66C3
:109BB00008F06CFCC2F200063946204608F066FC4C
:109BC00031464AF6B472204603924AF6F86508F028
:109BD0005DFC039AC2F200054CF6A06EC2F20002D0
:109BE00029462046CDF810E0039208F04FFC049877
:109BF0000399C1F6FF7004904CF65C722046059202
:109C000008F044FC059A0499C1F6FF724CF21C5E00
:109C100020460592CDF818E008F038FC069B05991F
:109C2000C2F200034CF2186E20460693CDF81CE0F9
:109C300008F02CFC079A0699C2F200024DF2240E9D
:109C400020460792CDF820E008F020FC089B0799F9
:109C5000C1F6FF734DF2E00E20460893CDF824E0E4
:109C600008F014FC099A0899C1F6FF724DF29C1E87
:109C700020460992CDF828E008F008FC0A9B0999D3
:109C80009E46C1F6FF7ECDF828E020464DF2582EC4
:109C9000CDF82CE008F0FAFB0B9A0A999646C1F62B
:109CA000FF7ECDF82CE020464CF6600ECDF830E07B
:109CB00008F0ECFB0C9B0B999E46C2F2000ECDF80F
:109CC00030E020464BF2885ECDF834E008F0DEFB51
:109CD0000D9A0C999646C2F2000E2046CDF834E05B
:109CE00008F0D4FB0D994EF2C87E2046CDF838E03E
:109CF00008F0CCFB0E9A9646C2F2000E20460221D6
:109D0000CDF838E008F0F8FB21460E9808F0B0FADC
:109D1000119B41F205221846C0F20002102108F002
:109D20001BF941F285125846C0F20002112108F0D9
:109D300013F941F625125046C0F20002122108F034
:109D40000BF940F685724846C0F20002132108F074
:109D500003F941F625224046C0F20002142108F022
:109D6000FBF841F205323846C0F20002152108F036
:109D7000F3F841F625323046C0F20002162108F011
:109D8000EBF841F631522846C0F20002172108F0E4
:109D9000E3F841F6A5120398C0F20002182108F07A
:109DA000DBF841F27D320498C0F20002192108F07C
:109DB000D3F841F205120598C0F200021A2108F00A
:109DC000CBF841F205020698C0F200021B2108F010
:109DD000C3F840F2F9620798C0F200021C2108F0B3
:109DE000BBF841F285220898C0F200021D2108F05C
:109DF000B3F841F621420998C0F200021E2108F092
:109E0000ABF841F6B1520A98C0F200021F2108F0E7
:109E1000A3F841F27D420B98C0F20002202108F025
:109E20009BF841F631620C98C0F20002212108F043
:109E300093F841F28952C0F200020D9822214EF2AD
:109E4000605408F089F8C2F200044AF6084120463E
:109E5000C2F2000108F01AFB4BF290112046C1F645
:109E6000FF7108F013FB2046022108F045FB4BF27E
:109E7000D0302146C2F200004BF22C3408F0F8F941
:109E8000C2F200044DF650112046C2F2000108F063
:109E9000FDFA4CF254312046C2F2000108F0F6FA05
:109EA0002046022108F028FB4DF20C002146C2F2A8
:109EB00000004CF60C2408F0DBF9C1F6FF744DF2FB
:109EC00044512046C2F2000108F0E0FA4DF2006170
:109ED0002046C2F2000108F0D9FA2046022108F01B
:109EE0000BFB4CF2D8502146C2F200004BF628443E
:109EF00008F0BEF9C2F200044BF2F4512046C1F65C
:109F0000FF7108F0C3FA4BF2B0612046C1F6FF7151
:109F100008F0BCFA2046022108F0EEFA4CF220408C
:109F20002146C2F200004CF6FC2408F0A1F9C2F26E
:109F300000044BF6C4512046C2F2000108F0A6FA14
:109F40004BF680612046C2F2000108F09FFA2046DD
:109F5000022108F0D1FA4DF608302146C1F6FF7013
:109F60004BF22C1408F084F9C2F200044DF648219B
:109F70002046C1F6FF7108F089FA4CF2CC21204648
:109F8000C1F6FF7108F082FA2046022108F0B4FA07
:109F90004BF694202146C1F6FF704DF2BC6408F0E8
:109FA00067F9C2F200044BF2D0112046C2F2000160
:109FB00008F06CFA4CF670012046C1F6FF7108F00B
:109FC00065FA2046022108F097FA4DF6F410214672
:109FD000C1F6FF704DF28C0408F04AF9C2F2000499
:109FE0004DF6C8312046C2F2000108F04FFA4DF696
:109FF00084412046C2F2000108F048FA20460221BE
:10A0000008F07AFA4AF6C8302146C2F200004EF64D
:10A01000081408F02DF9C2F200044CF68411204611
:10A02000C2F2000108F032FA4CF640212046C2F29A
:10A03000000108F02BFA2046022108F05DFA4BF2ED
:10A0400000102146C1F6FF704CF6100408F010F91C
:10A05000C2F200044CF61C412046C1F6FF7108F024
:10A0600015FA4CF6D0312046C2F2000108F00EFA83
:10A070002046022108F040FA4DF62C202146C2F27B
:10A0800000004CF2883408F0F3F8C1F6FF744BF28C
:10A09000BC712046C1F6FF7108F0F8F94BF6C80113
:10A0A0002046C1F6FF7108F0F1F92046022108F0C0
:10A0B00023FA4DF24C002146C2F200004BF6345414
:10A0C00008F0D6F8C2F200044BF27C412046C1F6FB
:10A0D000FF7108F0DBF94BF238512046C1F6FF71F1
:10A0E00008F0D4F92046022108F006FA4CF2582074
:10A0F0002146C2F200004DF2103408F0B9F8C2F265
:10A1000000044CF68C412046C2F2000108F0BEF972
:10A110004CF648512046C2F2000108F0B7F920463B
:10A12000022108F0E9F94CF690302146C2F2000015
:10A130004BF21C0408F09CF8C1F6FF744BF6881132
:10A140002046C1F6FF7108F0A1F94AF68051204679
:10A15000C2F2000108F09AF92046022108F0CCF979
:10A160004DF654402146C1F6FF704CF6506408F09D
:10A170007FF8C1F6FF744CF2F8512046C1F6FF712A
:10A1800008F084F94CF2B4612046C1F6FF7108F082
:10A190007DF92046022108F0AFF94CF2D07021463B
:10A1A000C2F200004BF26C7408F062F8C1F6FF7462
:10A1B0004CF694612046C2F2000108F067F94DF6B2
:10A1C00098312046C1F6FF7108F060F9204602215F
:10A1D00008F092F94EF6C4002146C2F200004DF696
:10A1E000BC2408F045F8C2F200044AF6CC2120460F
:10A1F000C2F2000108F04AF94BF2CC412046C2F20B
:10A20000000108F043F92046022108F075F94CF6E8
:10A2100054602146C2F200004CF2043408F028F8E1
:10A22000C2F200044EF608012046C2F2000108F016
:10A230002DF94DF254212046C2F2000108F026F912
:10A240002046022108F058F94DF63C602146C1F63F
:10A25000FF704DF6405408F00BF8C2F200044CF6C3
:10A260005C212046C1F6FF7108F010F94CF65071E0
:10A270002046C2F2000108F009F92046022108F048
:10A280003BF94AF688302146C2F200004CF2041530
:10A2900007F0EEFFC2F200054EF200612846C2F25E
:10A2A000000108F0F3F84BF630244EF2BC6128466A
:10A2B000C2F20001C2F2000408F0E8F8264628467F
:10A2C00002214BF244684BF28C2408F015F9C2F2DB
:10A2D0000004C2F20008294630464BF2BC770496CF
:10A2E000C2F2000707F0C4FF4DF6944641462046EF
:10A2F00008F0CCF8C1F6FF763946204608F0C6F8DB
:10A300004BF634153146204608F0C0F8C2F200057D
:10A310004BF6845003902946204608F0B7F803987E
:10A32000C2F2000003900221204608F0E5F8214621
:10A33000039807F09DFF41F64D724046C0F20002BF
:10A34000232107F009FE41F295623846C0F200026F
:10A35000242107F001FE41F6A5323046C0F200028A
:10A36000252107F0F9FD41F6A142C0F2000228467E
:10A3700026214EF2B05407F0EFFDC2F200044BF676
:10A380004C412046C1F6FF7108F080F84BF6903141
:10A390002046C1F6FF714DF20C7B08F077F8C2F24F
:10A3A000000B2046022108F0A7F84DF6483521465B
:10A3B000584607F05DFFC1F6FF754BF67841284619
:10A3C000C2F2000108F062F84CF2D4612846C2F2F1
:10A3D00000014DF2603A08F059F8C2F2000A28462E
:10A3E000022108F089F84BF26C042946504607F028
:10A3F0003FFFC1F6FF744CF6D8412046C1F6FF710D
:10A4000008F044F84CF694512046C1F6FF714BF227
:10A41000C00908F03BF8C1F6FF792046022108F098
:10A420006BF84AF2D4552146484607F021FFC2F2A4
:10A4300000054BF670212846C2F2000108F026F80C
:10A440004BF62C312846C2F200014DF2A03808F03C
:10A450001DF8C2F200082846022108F04DF84CF61B
:10A4600004642946404607F003FFC2F200044CF2A0
:10A4700078112046C2F2000108F008F84CF2B471DD
:10A480002046C1F6FF714CF2907707F0FFFFC2F251
:10A4900000072046022108F02FF84CF27C252146C7
:10A4A000384607F0E5FEC1F6FF754DF254712846B7
:10A4B000C2F2000107F0EAFF4DF60C312846C2F265
:10A4C00000014CF64C3607F0E1FFC2F200062846C8
:10A4D00002214DF2E034C2F2000408F00DF82946E2
:10A4E000304607F0C5FE0199204608F09DF80F9907
:10A4F000204608F099F80299204608F095F80E9940
:10A50000204608F091F81099204608F08DF84CF696
:10A510002C112046C1F6FF7108F086F84DF69061C7
:10A520002046C1F6FF7108F07FF84BF27C312046DF
:10A53000C2F2000108F078F84CF2C4212046C2F2C1
:10A54000000108F071F84DF610012046C2F200013A
:10A5500008F06AF84BF23C412046C1F6FF7108F062
:10A5600063F84DF638012046C1F6FF7108F05CF83B
:10A570004DF6D8012046C2F2000108F055F84EF21F
:10A58000C8712046C2F2000108F04EF84BF2D031FB
:10A590002046C2F2000108F047F84DF20C012046B7
:10A5A000C2F2000108F040F84CF2D8512046C2F245
:10A5B000000108F039F84CF220412046C2F20001B7
:10A5C00008F032F84DF608312046C1F6FF7108F068
:10A5D0002BF84BF694212046C1F6FF7108F024F8C1
:10A5E0004DF6F4112046C1F6FF7108F01DF84AF649
:10A5F000C8312046C2F2000108F016F84BF20011F3
:10A600002046C1F6FF7108F00FF84DF62C212046C8
:10A61000C2F2000108F008F84DF24C012046C2F2E7
:10A62000000108F001F84CF258212046C2F2000166
:10A6300007F0FAFF4CF690312046C2F2000107F015
:10A64000F3FF4DF654412046C1F6FF7107F0ECFFD1
:10A650004CF2D0712046C2F2000107F0E5FF4EF641
:10A66000C4012046C2F2000107F0DEFF4CF654613F
:10A670002046C2F2000107F0D7FF4DF63C612046AC
:10A68000C1F6FF7107F0D0FF4AF688312046C2F2CA
:10A69000000107F0C9FF0499204607F0C5FF0399A0
:10A6A000204607F0C1FF5946204607F0BDFF51463E
:10A6B000204607F0B9FF4946204607F0B5FF41465E
:10A6C000204607F0B1FF3946204607F0ADFF31467E
:10A6D000204607F0A9FF2046022107F0DFFF4CF2D9
:10A6E00098262046012107F0D3FFC2F2000620463B
:10A6F0004EF2405507F0F6FFC2F200052922FF2175
:10A70000304612F071F800242846347008F016F82C
:10A7100005F1100008F012F820460BF03DFA49F25E
:10A72000EF2144F27013C2F20003C1F6FF716322FD
:10A7300008701C775C619A6172B69042A8BF10469F
:10A740008000D86062B64DF21802C1F6FF72087838
:10A7500083F83C4005215C631060996372B6DC624B
:10A7600062B6546013B0BDE8F08F00BF70B502212F
:10A7700082B004200BF09CFF02211E200BF098FFFA
:10A78000FEF766FF41F21050C0F20200F5F7A2FF9B
:10A7900041F25450C0F20200F5F79CFF41F28450A0
:10A7A000C0F20200F5F796FF41F2B450C0F2020089
:10A7B00049F2E465F5F784FFC1F6FF754EF22441D6
:10A7C0000A22C0F20C01002328460AF0A3FF41F23E
:10A7D000C850C0F20200F5F77DFF28460AF088FF56
:10A7E00041F2D050C0F20200F5F774FF40F6E440A9
:10A7F0000BF0B2FC044600F02FFC4BF2CC13C2F27B
:10A80000000301261C60FCF75BF9FAF745FAFAF73A
:10A8100011FC4EF28813CEF2000340F2002044F205
:10A82000B0141E60C2F200048021C1F6FF700AF06D
:10A83000C3F9204603F0B8FC204602F071FDB7EEE4
:10A84000000A204603F08AF9E288242122F010024F
:10A85000204602F0BDFBF6EE000AB0EE600A20468C
:10A8600002F058FEE288204622F48072242102F091
:10A87000AFFB1D21204602F0C9FD204603F0EAFA95
:10A880000221204602F0D6FC204602F051FC204670
:10A8900002F0CCFB41F2E050C0F20200F5F71AFFE3
:10A8A00049F2EF23C1F6FF734FF20E641878FAF7FE
:10A8B0005FFD4FF20C61C2F200044FF20862C2F277
:10A8C00000014FF28C53C2F20002C2F2000341F2C7
:10A8D000FC50248809881480C0F202001980F5F722
:10A8E000EFFE802128460AF0A5FE41F21460C0F276
:10A8F0000200F5F7E5FE40F65A3128460AF09AFEC6
:10A9000041F22860C0F20200F5F7E4FE4EF20813AF
:10A91000CEF2000341F22C601E60C0F20200F5F797
:10A92000D9FE28460AF0E4FEFCF7A4F94FF234629F
:10A93000C2F200024DF2507312680192C2F200039B
:10A94000019A1A6002B070BD2DE9F04F2DED068B13
:10A950004BF2BC03844683B0C1F6FF7300F6A844F3
:10A9600093ED000AD4ED008ADCF87CEC9FEDA35A4D
:10A97000DFEDA30A0CF6944300F6C44500F6AC499B
:10A9800000F54B681C4600F6A44001930CF69C436E
:10A990000CF5496B90ED008A93ED00AAD5ED004AC5
:10A9A00099ED003AD8ED003ADBED002A94ED004A2B
:10A9B0000CF54A630CF69840D3ED009A90ED001A1E
:10A9C00002F1FE030239A2F1020A0093F6EE001A28
:10A9D000B7EE002ABFEE009ABEF1000F9FED896A24
:10A9E00040F30881DCF8806CF0EE465A0CF53C70C0
:10A9F000002550F8307C50F8343C50F82C2C50F89E
:10AA0000284C3B4402EB234201359BB2A2422DB2BB
:10AA100040F82C2C40F8303C04DD50F8244C121B3C
:10AA200040F82C2C06EB420436F91220B4F90270DF
:10AA300010ED087A50ED076ABF1A03FB07F302EB2B
:10AA4000234307EE903AF8EEE77A67EE266A67EE60
:10AA5000877A40ED086A67EE857AF5EEC07AF1EE06
:10AA600010FA0EDD24EEA77AE7EEC77AB0EE677A29
:10AA7000F1EE667AB4EEE77AF1EE10FA58BFF0EE36
:10AA8000477A50ED036A10ED027A7545E7EEA65A53
:10AA900000F13400A7EE876AABDB36EE637A75EE21
:10AAA000C37AE7EE283A019BA7EEA83AE1EE042A22
:10AAB00036EE637AA2EEC14AA7EE086A75EEC37A53
:10AAC00026EE297AE7EE885AA4EE076A65EE8A7ABE
:10AAD00026EE216AE4EE275AB4EEC26AF1EE10FACD
:10AAE00089ED003A65EEA15AC8ED003ACBED002A97
:10AAF00083ED004A76DDB7EE006AF4EEC25AF1EE5D
:10AB000010FA67DDF7EE005A65EE805A26EE006A0D
:10AB100065EEA05A26EE206AFDEEE57A17EE902A41
:10AB2000FDEEC67A2AF8022F17EE903A21F8023F7E
:10AB3000009B9A457FF450AFDFED337AB0EEC33A15
:10AB4000B4EEE73ADFED307AF1EE10FAF0EEE33AE8
:10AB500048BF0023F4EEE73A48BFC9F80030F1EEF1
:10AB600010FA44BF0023C8F80030BEF1000F2CDDFE
:10AB700000239FED267A1E46342706E0DCF87CECA5
:10AB8000013636B2764533461FDA07FB03C3D3EDF1
:10AB9000B47A0EF1FF3EF4EEC77A07FB0EC4F1EE75
:10ABA00010FA04F52F7403F52F75E7D50FCCCCF808
:10ABB0007CEC0FC50FCC0FC50FCC0FC5013636B2DC
:10ABC00023682B6076453346DFDB03B0BDEC068B94
:10ABD000BDE8F08FF4EE495AF1EE10FA48BFF0EEFE
:10ABE000495A91E7B4EE496AF1EE10FA48BFB0EE67
:10ABF000496A82E7F0EE465A4FE700BF000000388E
:10AC000000FEFF4600000000FFE6DB2E17B7D1383C
:10AC100041689FED157AD1ED056ADFED147AE6EE15
:10AC2000877A4FF4884243F2C673C4F22C72C3F29F
:10AC3000BE7310B58260C360044617EE900A10F030
:10AC40004FFD41EC100B0FF097F851EC100B11F089
:10AC500093F8DFED077A07EE100A67EE277A04F61D
:10AC60009844C4ED007A10BD3D0AC7403D0A27C094
:10AC7000716415392DE9F84307292DED028B4668DB
:10AC80005DD00FD9402901D0422936D102F04004CD
:10AC9000E4B2C0F88C4C002C64D0BDEC028B0120D7
:10ACA000BDE8F883012928D107EE902ADFED506A2C
:10ACB0009FED507AF8EE677A00F6DC4367EEA67AED
:10ACC000F4EEC77AF1EE10FAC3ED007AE5DD00F696
:10ACD0009C4300F54A60C3ED007AC0ED007AD6EDE2
:10ACE000046AB6EE007AF4EEC76AF1EE10FAD4D533
:10ACF000F1EE677AC0ED007ACFE77A29CDD9037CEF
:10AD00007BB103EB430203EB820247F2A401C3F6DB
:10AD10007D7100EB82020346C3F8D41234339A42A9
:10AD2000FAD1BDEC028B00F6C8430022C4F22032F7
:10AD30000021C0F88C1C01201A60BDE8F88312FBCA
:10AD400002F207EE902ABDEC028BF8EEE77A9FED57
:10AD50002A7A67EE877A00F6D840C0ED007A0120A3
:10AD6000BDE8F883027C002A97D007460546B1EE7D
:10AD7000048A03E0A24205F134058EDDD5F8EC32F9
:10AD8000802B04F10104F5D1D7F88C3C002BF1D1D4
:10AD9000F86880F0004010F0A3FCD6ED017A67EE71
:10ADA000887A804617EE900A894610F099FC0B4687
:10ADB00041F6B8610246C4F21D014FF0A04010F008
:10ADC0002FFB41EC100B0EF0D7FF404653EC102B3D
:10ADD000494610F0D9FC41EC100B0EF0CDFF51ECC0
:10ADE000100B10F0C9FFC5F8D4023A7CC2E700BFCF
:10ADF0002497FF3BCDCC4C3DACC5A73770B545681B
:10AE0000D0ED035A95ED024A95ED036A9FED697AFC
:10AE10009FED695AF2EE084AF9EE087AE4EE247AD8
:10AE200000F6A44300F6A846F1EE006A2DED028B71
:10AE300066EE266ABFEE008AF0EE484AE6EE264A43
:10AE40000446FDEEE77AF6EE008A17EE902AC0F887
:10AE5000882CC3ED004AD5ED037AF4EEE87AF1EEE2
:10AE600010FAD4BFF0EE457AF0EE477AC6ED007ADC
:10AE700065EEE77A17EE900A10F032FC41EC100B09
:10AE80000EF07AFF51EC100B10F076FF07EE100A6F
:10AE9000F7EE007A77EEC77AB0EE007AC6ED007A68
:10AEA000D5ED047AA7EE878A04F69C4204F54A633E
:10AEB00082ED008A83ED008A95ED047AB4EEE87A9B
:10AEC000F1EE10FA03D5F1EE487AC3ED007ADFED2A
:10AED0003B6A95ED056A9FED3A7AD4ED037A9FEDD2
:10AEE000398AA6EE267A04F6984627EE888A17EE67
:10AEF000100A10F0F5FB41EC100B0EF03DFF51EC89
:10AF0000100B10F039FF07EE900A27EE888AF7EE53
:10AF1000007A86ED008A95ED067A77EE277A04F6B8
:10AF2000D44377EE877AF5EE006AC3ED007A95EDAB
:10AF3000067AB4EEE67AF1EE10FA09D5B0EE086AB8
:10AF4000F6EE086AE7EE466A77EEE67AC3ED007A37
:10AF500095ED077A9FED1C6ADFED1C7ADFED1C6A28
:10AF600027EE067A04F6844383ED007A95ED097A9C
:10AF7000B6EE006A37EE467A04F6B84383ED007AFF
:10AF800095ED0A7A67EE277A04F54C6367EE877AC7
:10AF900004F6BC410022C1ED007ABDEC028B1A60C0
:10AFA000D5ED0B7A67EEA67A04F6C444C4ED007AB8
:10AFB00070BD00BF00C05A4600409C453D0AC740D6
:10AFC0003D0A27C0560EC9408FC2F53C2DB29D3DAB
:10AFD0006666E63FF0B547F2A4040025C3F67D742B
:10AFE000034600F51C61C3F8D052C3F8D442343391
:10AFF0008B424FF00002F6D100F6D8454CF6CD4713
:10B00000C3F64C6700F6C84400262F600023C4F244
:10B01000203600F69845266000F5496EC0F87C3C65
:10B02000C0F88C3C00F54B6700F6AC4600F6944443
:10B030004CF6CD4100F54E632A60C3F64C714FF0DB
:10B040007E55CEF800203A60326025601960BDE878
:10B05000F040FFF7D3BE00BFF8B54FF4884243F28B
:10B06000C67341F69811C0F20201C4F22C72C3F209
:10B07000BE73044601608260C36030200BF06EF83E
:10B0800003464FF07C571F6060602046FFF7B6FE16
:10B09000636820465F60FFF7B1FE636820469F60EB
:10B0A000FFF7ACFE63682046DF60FFF7A7FE63682A
:10B0B00020461F61FFF7A2FE636846F26662C3F690
:10B0C00026725A612046FFF799FE63684FF07A5264
:10B0D0009A612046FFF792FE63682046DF61FFF722
:10B0E0008DFE63680126267420465F62FFF786FEA8
:10B0F000636848F20612C3F615629A622046FFF7AB
:10B100007DFE63680025DD622046FFF777FE41F68D
:10B11000A413C0F20203C4F8803C242363612723F4
:10B12000A3612B2323652D2363653023C4F88C3062
:10B130003323C4F890303723C4F8C8303923C4F817
:10B14000CC303C23C4F804313F23C4F808314323F6
:10B15000C4F840314523C4F844314823C4F87C3155
:10B160004B23C4F880314F23C4F8B8315123C4F8BD
:10B17000BC315423C4F8F4315723C4F8F8315B23AD
:10B18000C4F830325D23C4F834326023C4F86C3222
:10B1900040F2E733C4F870320023E36142F21C133B
:10B1A000236241F23013636242F21D13236343F6BC
:10B1B0007873636341F22733A36343F6797363645F
:10B1C00048F20573A36441F6FE03E36448F2067394
:10B1D000A3654AF2A813E36540F6627323664AF258
:10B1E000A913E3664BF2C023236740F261636367F0
:10B1F0004BF2C123C4F880304FF6BB63C4F88430EF
:10B2000041F27D43C4F888304FF6BC63C4F89430F3
:10B210004CF2496366F31F43294648F6230040F683
:10B220009B0566F31F40C4F8B050C4F8D43041F613
:10B23000C14242F6D40343F2223E4FF2AD2566F3FB
:10B240001F4266F31F4E66F31F45C4F8C000C4F8E2
:10B25000D8304FF4C75043F2233745F21F5366F3FB
:10B260001F47C4F89820C4F8ACE0C4F8C400C0F28A
:10B270000203C4F8E85048F624024CF24A6E43F246
:10B28000F1204AF2334566F31F4266F31F4EC4F8BD
:10B29000BC70C0F20200C0F20205C4F8103141F6E1
:10B2A000C24C41F2BC034FF2AE2766F31F4766F370
:10B2B0001F4CC4F8D020C4F8E4E0C4F8FC00C4F883
:10B2C000143140F61B40C4F8245143F2F22240F6F8
:10B2D0004C7545F220564AF2344E41F63673C0F2B0
:10B2E0000202C0F20206C4F8F870C0F2020E41F287
:10B2F0006147C4F80001C0F20303C4F828514FF2BB
:10B30000DE0040F67935C4F8EC70C0F20200C4F8F3
:10B310000C21C4F82061C4F89C50C4F8A8C045F2C0
:10B320007376C4F834E1C4F84C3141F27C23C0F2A6
:10B330000306C4F83801C4F8503149F249104CF6FC
:10B34000CB03C0F20300C0F20303C4F8606141F212
:10B350007D26C4F86461C4F87401C4F8883140F6ED
:10B36000ED0041F202034FF2DF0241F6377740F67B
:10B370004746C0F20202C0F20307C4F83C51C0F2D3
:10B380000406C4F87801C4F88C3145F2747544F6AB
:10B390008F6047F69033C0F20305C4F84821C4F823
:10B3A0005C71C0F20400C0F20403C4F89C6149F26D
:10B3B0004A1241F203064CF6CC07C0F20302C0F277
:10B3C0000307C4F87051C4F8A061C4F8B001C4F810
:10B3D000C43140F6196040F68E1340F648454CF2F1
:10B3E000F646C0F20405C4F88421C4F89871C0F28E
:10B3F0000406C4F8B401C4F8C83144F6906247F6B4
:10B40000913740F6D81045F2D923C0F20402C0F2B9
:10B410000407C4F8AC51C0F20500C0F20503C4F83B
:10B42000D8614CF2F74541F68606C0F20405C4F82F
:10B43000C021C4F8D471C4F8DC61C4F8EC01C4F8CC
:10B44000003240F6EB0040F6812340F6D91245F277
:10B45000DA2749F26B46C0F20502C0F20507C0F2D6
:10B460000506C4F8E851C4F8F001C4F8043249F202
:10B470006C454DF6AD2043F21D23C0F20505C0F228
:10B480000500C4F8FC21C0F20603C4F810729D2226
:10B49000C4F8146241F21216C0F2060245F21737E0
:10B4A000C4F81862C4F8245247F208264DF6AE25B7
:10B4B000C4F82802C4F8643241F2694041F2AA1388
:10B4C000C0F20505C0F20607C0F20606C4F82C0259
:10B4D000C4F860229C2043F21E22C4F8683245F270
:10B4E0001633C0F20600C0F20603C0F20602C4F82A
:10B4F0009C7240F6790E40F6FB27C4F8A062C4F8AF
:10B50000385240F60216C4F84C5247F2A405C4F86B
:10B510003C02C4F85002C4F87832C4F88C32C4F843
:10B52000A4E2C3F67D75C4F84072C4F85472C4F83E
:10B530007422C4F88822C4F87C62C4F8906223465E
:10B5400004F51C60C3F8D012C3F8D45234338342DC
:10B550004FF00002F6D104F6D8464CF6CD4704F67B
:10B56000C840C3F64C6700253760002304F69846B0
:10B57000C4F22035056004F5496EC4F87C3CC4F87B
:10B580008C3C04F6AC4004F54E6304F54B6704F6BE
:10B5900094454CF6CD413260C3F64C714FF07E5667
:10B5A000CEF800203A60026020462E601960FFF756
:10B5B00025FC2046F8BD00BF70B545689FED6C7A4C
:10B5C00095ED025A95ED036AF2EE085AF9EE087A03
:10B5D000E5EE257A00F6A44300F6A846F1EE006AEF
:10B5E0002DED028B66EE266ABFEE008AF0EE485A19
:10B5F000E6EE265A0446FDEEE77A85ED000A17EEE0
:10B60000902AC0F8882CC3ED005A95ED036ADFED4F
:10B61000597AD0ED036AF6EE008AB4EEE86AF1EEEC
:10B6200010FAC8BFF0EE477AC6ED007A66EEE77A08
:10B6300017EE900A10F054F841EC100B0EF09CFB42
:10B6400051EC100B10F098FB07EE100AF7EE007AA1
:10B6500077EEC77AB0EE007AC6ED007AD5ED047ABF
:10B66000A7EE878A04F69C4204F54A6382ED008ABD
:10B6700083ED008A95ED047AB4EEE87AF1EE10FAE3
:10B6800003D5F1EE487AC3ED007ADFED3B6A95ED24
:10B69000056A9FED3A7AD4ED037A9FED398AA6EEDA
:10B6A000267A04F6984627EE888A17EE100A10F0DC
:10B6B00017F841EC100B0EF05FFB51EC100B10F083
:10B6C0005BFB07EE900A27EE888AF7EE007A86ED9C
:10B6D000008A95ED067A77EE277A04F6D44377EE62
:10B6E000877AF5EE006AC3ED007A95ED067AB4EE3E
:10B6F000E67AF1EE10FA09D5B0EE086AF6EE086ABD
:10B70000E7EE466A77EEE67AC3ED007A95ED077AC2
:10B710009FED1C6ADFED1C7ADFED1C6A27EE067ACE
:10B7200004F6844383ED007A95ED097AB6EE006A5B
:10B7300037EE467A04F6B84383ED007A95ED0A7A3F
:10B7400067EE277A04F54C6367EE877A04F6BC410E
:10B750000022C1ED007ABDEC028B1A60D5ED0B7AA8
:10B7600067EEA67A04F6C444C4ED007A70BD00BF4B
:10B7700000C05A4600409C453D0AC7403D0A27C0CC
:10B78000560EC9408FC2F53C2DB29D3D6666E63F20
:10B7900070B545689FED6C7A95ED025A95ED036A98
:10B7A000F2EE085AF9EE087AE5EE257A00F6A4439F
:10B7B00000F6A846F1EE006A2DED028B66EE266AD1
:10B7C000BFEE008AF0EE485AE6EE265A0446FDEE39
:10B7D000E77A85ED010A17EE902AC0F8882CC3EDB0
:10B7E000005A95ED036ADFED597AD0ED036AF6EE63
:10B7F000008AB4EEE86AF1EE10FAC8BFF0EE477ABC
:10B80000C6ED007A66EEE77A17EE900A0FF068FF51
:10B8100041EC100B0EF0B0FA51EC100B10F0ACFA3A
:10B8200007EE100AF7EE007A77EEC77AB0EE007AEC
:10B83000C6ED007AD5ED047AA7EE878A04F69C421D
:10B8400004F54A6382ED008A83ED008A95ED047A5F
:10B85000B4EEE87AF1EE10FA03D5F1EE487AC3EDD2
:10B86000007ADFED3B6A95ED056A9FED3A7AD4EDFB
:10B87000037A9FED398AA6EE267A04F6984627EEDB
:10B88000888A17EE100A0FF02BFF41EC100B0EF018
:10B8900073FA51EC100B10F06FFA07EE900A27EED6
:10B8A000888AF7EE007A86ED008A95ED067A77EEC3
:10B8B000277A04F6D44377EE877AF5EE006AC3ED73
:10B8C000007A95ED067AB4EEE67AF1EE10FA09D533
:10B8D000B0EE086AF6EE086AE7EE466A77EEE67AB8
:10B8E000C3ED007A95ED077A9FED1C6ADFED1C7AB7
:10B8F000DFED1C6A27EE067A04F6844383ED007AB6
:10B9000095ED097AB6EE006A37EE467A04F6B8434A
:10B9100083ED007A95ED0A7A67EE277A04F54C6399
:10B9200067EE877A04F6BC410022C1ED007ABDECD7
:10B93000028B1A60D5ED0B7A67EEA67A04F6C44442
:10B94000C4ED007A70BD00BF00C05A4600409C455F
:10B950003D0AC7403D0A27C0560EC9408FC2F53C7C
:10B960002DB29D3D6666E63F70B545689FED6B7AEA
:10B9700095ED036AF2EE085AF9EE087AE0EE257AC0
:10B9800000F6A44300F6A846F1EE006A2DED028B06
:10B9900066EE266ABFEE008AF0EE485AE6EE265AB8
:10B9A0000446FDEEE77A85ED020A17EE902AC0F80C
:10B9B000882CC3ED005A95ED036ADFED597AD0ED7E
:10B9C000036AF6EE008AB4EEE86AF1EE10FAC8BF38
:10B9D000F0EE477AC6ED007A66EEE77A17EE900A47
:10B9E0000FF07EFE41EC100B0EF0C6F951EC100B7F
:10B9F00010F0C2F907EE100AF7EE007A77EEC77A78
:10BA0000B0EE007AC6ED007AD5ED047AA7EE878A0B
:10BA100004F69C4204F54A6382ED008A83ED008AB5
:10BA200095ED047AB4EEE87AF1EE10FA03D5F1EE72
:10BA3000487AC3ED007ADFED3B6A95ED056A9FED2C
:10BA40003A7AD4ED037A9FED398AA6EE267A04F687
:10BA5000984627EE888A17EE100A0FF041FE41EC57
:10BA6000100B0EF089F951EC100B10F085F907EE70
:10BA7000900A27EE888AF7EE007A86ED008A95ED27
:10BA8000067A77EE277A04F6D44377EE877AF5EED6
:10BA9000006AC3ED007A95ED067AB4EEE67AF1EE2F
:10BAA00010FA09D5B0EE086AF6EE086AE7EE466AC3
:10BAB00077EEE67AC3ED007A95ED077A9FED1C6A82
:10BAC000DFED1C7ADFED1C6A27EE067A04F684436C
:10BAD00083ED007A95ED097AB6EE006A37EE467A84
:10BAE00004F6B84383ED007A95ED0A7A67EE277A7B
:10BAF00004F54C6367EE877A04F6BC410022C1ED81
:10BB0000007ABDEC028B1A60D5ED0B7A67EEA67A4F
:10BB100004F6C444C4ED007A70BD00BF00C05A46AC
:10BB200000409C453D0AC7403D0A27C0560EC9400B
:10BB30008FC2F53C2DB29D3D6666E63F70B5456807
:10BB40009FED6B7AD5ED025AB2EE086AF9EE087AEB
:10BB5000E5EE867A00F6A44300F6A846F1EE006A08
:10BB60002DED028B60EE266ABFEE008AB0EE486AC9
:10BB7000A0EE266A0446FDEEE77A85ED030A17EE8D
:10BB8000902AC0F8882C83ED006A95ED036ADFEDFA
:10BB9000597AD0ED036AF6EE008AB4EEE86AF1EE67
:10BBA00010FAC8BFF0EE477AC6ED007A66EEE77A83
:10BBB00017EE900A0FF094FD41EC100B0EF0DCF83C
:10BBC00051EC100B10F0D8F807EE100AF7EE007ADF
:10BBD00077EEC77AB0EE007AC6ED007AD5ED047A3A
:10BBE000A7EE878A04F69C4204F54A6382ED008A38
:10BBF00083ED008A95ED047AB4EEE87AF1EE10FA5E
:10BC000003D5F1EE487AC3ED007ADFED3B6A95ED9E
:10BC1000056A9FED3A7AD4ED037A9FED398AA6EE54
:10BC2000267A04F6984627EE888A17EE100A0FF057
:10BC300057FD41EC100B0EF09FF851EC100B10F07B
:10BC40009BF807EE900A27EE888AF7EE007A86EDD9
:10BC5000008A95ED067A77EE277A04F6D44377EEDC
:10BC6000877AF5EE006AC3ED007A95ED067AB4EEB8
:10BC7000E67AF1EE10FA09D5B0EE086AF6EE086A37
:10BC8000E7EE466A77EEE67AC3ED007A95ED077A3D
:10BC90009FED1C6ADFED1C7ADFED1C6A27EE067A49
:10BCA00004F6844383ED007A95ED097AB6EE006AD6
:10BCB00037EE467A04F6B84383ED007A95ED0A7ABA
:10BCC00067EE277A04F54C6367EE877A04F6BC4189
:10BCD0000022C1ED007ABDEC028B1A60D5ED0B7A23
:10BCE00067EEA67A04F6C444C4ED007A70BD00BFC6
:10BCF00000C05A4600409C453D0AC7403D0A27C047
:10BD0000560EC9408FC2F53C2DB29D3D6666E63F9A
:10BD100070B545689FED6C7A95ED025A95ED036A12
:10BD2000F2EE085AF9EE087AE5EE257A00F6A44319
:10BD300000F6A846F1EE006A2DED028B66EE266A4B
:10BD4000BFEE008AF0EE485AE6EE265A0446FDEEB3
:10BD5000E77A85ED040A17EE902AC0F8882CC3ED27
:10BD6000005A95ED036ADFED597AD0ED036AF6EEDD
:10BD7000008AB4EEE86AF1EE10FAC8BFF0EE477A36
:10BD8000C6ED007A66EEE77A17EE900A0FF0A8FC8F
:10BD900041EC100B0DF0F0FF51EC100B0FF0ECFF2D
:10BDA00007EE100AF7EE007A77EEC77AB0EE007A67
:10BDB000C6ED007AD5ED047AA7EE878A04F69C4298
:10BDC00004F54A6382ED008A83ED008A95ED047ADA
:10BDD000B4EEE87AF1EE10FA03D5F1EE487AC3ED4D
:10BDE000007ADFED3B6A95ED056A9FED3A7AD4ED76
:10BDF000037A9FED398AA6EE267A04F6984627EE56
:10BE0000888A17EE100A0FF06BFC41EC100B0DF056
:10BE1000B3FF51EC100B0FF0AFFF07EE900A27EEC7
:10BE2000888AF7EE007A86ED008A95ED067A77EE3D
:10BE3000277A04F6D44377EE877AF5EE006AC3EDED
:10BE4000007A95ED067AB4EEE67AF1EE10FA09D5AD
:10BE5000B0EE086AF6EE086AE7EE466A77EEE67A32
:10BE6000C3ED007A95ED077A9FED1C6ADFED1C7A31
:10BE7000DFED1C6A27EE067A04F6844383ED007A30
:10BE800095ED097AB6EE006A37EE467A04F6B843C5
:10BE900083ED007A95ED0A7A67EE277A04F54C6314
:10BEA00067EE877A04F6BC410022C1ED007ABDEC52
:10BEB000028B1A60D5ED0B7A67EEA67A04F6C444BD
:10BEC000C4ED007A70BD00BF00C05A4600409C45DA
:10BED0003D0AC7403D0A27C0560EC9408FC2F53CF7
:10BEE0002DB29D3D6666E63F70B545689FED6C7A64
:10BEF00095ED025A95ED036AF2EE085AF9EE087ACA
:10BF0000E5EE257A00F6A44300F6A846F1EE006AB5
:10BF10002DED028B66EE266ABFEE008AF0EE485ADF
:10BF2000E6EE265A0446FDEEE77A85ED050A17EEA1
:10BF3000902AC0F8882CC3ED005A95ED036ADFED16
:10BF4000597AD0ED036AF6EE008AB4EEE86AF1EEB3
:10BF500010FAC8BFF0EE477AC6ED007A66EEE77ACF
:10BF600017EE900A0FF0BCFB41EC100B0DF004FF34
:10BF700051EC100B0FF000FF07EE100AF7EE007AFD
:10BF800077EEC77AB0EE007AC6ED007AD5ED047A86
:10BF9000A7EE878A04F69C4204F54A6382ED008A84
:10BFA00083ED008A95ED047AB4EEE87AF1EE10FAAA
:10BFB00003D5F1EE487AC3ED007ADFED3B6A95EDEB
:10BFC000056A9FED3A7AD4ED037A9FED398AA6EEA1
:10BFD000267A04F6984627EE888A17EE100A0FF0A4
:10BFE0007FFB41EC100B0DF0C7FE51EC100B0FF076
:10BFF000C3FE07EE900A27EE888AF7EE007A86EDF8
:10C00000008A95ED067A77EE277A04F6D44377EE28
:10C01000877AF5EE006AC3ED007A95ED067AB4EE04
:10C02000E67AF1EE10FA09D5B0EE086AF6EE086A83
:10C03000E7EE466A77EEE67AC3ED007A95ED077A89
:10C040009FED1C6ADFED1C7ADFED1C6A27EE067A95
:10C0500004F6844383ED007A95ED097AB6EE006A22
:10C0600037EE467A04F6B84383ED007A95ED0A7A06
:10C0700067EE277A04F54C6367EE877A04F6BC41D5
:10C080000022C1ED007ABDEC028B1A60D5ED0B7A6F
:10C0900067EEA67A04F6C444C4ED007A70BD00BF12
:10C0A00000C05A4600409C453D0AC7403D0A27C093
:10C0B000560EC9408FC2F53C2DB29D3D6666E63FE7
:10C0C00070B545689FED6C7A95ED025A95ED036A5F
:10C0D000F2EE085AF9EE087AE5EE257A00F6A44366
:10C0E00000F6A846F1EE006A2DED028B66EE266A98
:10C0F000BFEE008AF0EE485AE6EE265A0446FDEE00
:10C10000E77A85ED060A17EE902AC0F8882CC3ED71
:10C11000005A95ED036ADFED597AD0ED036AF6EE29
:10C12000008AB4EEE86AF1EE10FAC8BFF0EE477A82
:10C13000C6ED007A66EEE77A17EE900A0FF0D0FAB5
:10C1400041EC100B0DF018FE51EC100B0FF014FE2B
:10C1500007EE100AF7EE007A77EEC77AB0EE007AB3
:10C16000C6ED007AD5ED047AA7EE878A04F69C42E4
:10C1700004F54A6382ED008A83ED008A95ED047A26
:10C18000B4EEE87AF1EE10FA03D5F1EE487AC3ED99
:10C19000007ADFED3B6A95ED056A9FED3A7AD4EDC2
:10C1A000037A9FED398AA6EE267A04F6984627EEA2
:10C1B000888A17EE100A0FF093FA41EC100B0DF07D
:10C1C000DBFD51EC100B0FF0D7FD07EE900A27EEC8
:10C1D000888AF7EE007A86ED008A95ED067A77EE8A
:10C1E000277A04F6D44377EE877AF5EE006AC3ED3A
:10C1F000007A95ED067AB4EEE67AF1EE10FA09D5FA
:10C20000B0EE086AF6EE086AE7EE466A77EEE67A7E
:10C21000C3ED007A95ED077A9FED1C6ADFED1C7A7D
:10C22000DFED1C6A27EE067A04F6844383ED007A7C
:10C2300095ED097AB6EE006A37EE467A04F6B84311
:10C2400083ED007A95ED0A7A67EE277A04F54C6360
:10C2500067EE877A04F6BC410022C1ED007ABDEC9E
:10C26000028B1A60D5ED0B7A67EEA67A04F6C44409
:10C27000C4ED007A70BD00BF00C05A4600409C4526
:10C280003D0AC7403D0A27C0560EC9408FC2F53C43
:10C290002DB29D3D6666E63F70B545689FED6C7AB0
:10C2A00095ED025A95ED036AF2EE085AF9EE087A16
:10C2B000E5EE257A00F6A44300F6A846F1EE006A02
:10C2C0002DED028B66EE266ABFEE008AF0EE485A2C
:10C2D000E6EE265A0446FDEEE77A85ED070A17EEEC
:10C2E000902AC0F8882CC3ED005A95ED036ADFED63
:10C2F000597AD0ED036AF6EE008AB4EEE86AF1EE00
:10C3000010FAC8BFF0EE477AC6ED007A66EEE77A1B
:10C3100017EE900A0FF0E4F941EC100B0DF02CFD34
:10C3200051EC100B0FF028FD07EE100AF7EE007A23
:10C3300077EEC77AB0EE007AC6ED007AD5ED047AD2
:10C34000A7EE878A04F69C4204F54A6382ED008AD0
:10C3500083ED008A95ED047AB4EEE87AF1EE10FAF6
:10C3600003D5F1EE487AC3ED007ADFED3B6A95ED37
:10C37000056A9FED3A7AD4ED037A9FED398AA6EEED
:10C38000267A04F6984627EE888A17EE100A0FF0F0
:10C39000A7F941EC100B0DF0EFFC51EC100B0FF076
:10C3A000EBFC07EE900A27EE888AF7EE007A86ED1E
:10C3B000008A95ED067A77EE277A04F6D44377EE75
:10C3C000877AF5EE006AC3ED007A95ED067AB4EE51
:10C3D000E67AF1EE10FA09D5B0EE086AF6EE086AD0
:10C3E000E7EE466A77EEE67AC3ED007A95ED077AD6
:10C3F0009FED1C6ADFED1C7ADFED1C6A27EE067AE2
:10C4000004F6844383ED007A95ED097AB6EE006A6E
:10C4100037EE467A04F6B84383ED007A95ED0A7A52
:10C4200067EE277A04F54C6367EE877A04F6BC4121
:10C430000022C1ED007ABDEC028B1A60D5ED0B7ABB
:10C4400067EEA67A04F6C444C4ED007A70BD00BF5E
:10C4500000C05A4600409C453D0AC7403D0A27C0DF
:10C46000560EC9408FC2F53C2DB29D3D6666E63F33
:10C470000174704770B545689FED6C7A95ED025A6E
:10C4800095ED036AF2EE085AF9EE087AE5EE257AA0
:10C4900000F6A44300F6A846F1EE006A2DED028BEB
:10C4A00066EE266ABFEE008AF0EE485AE6EE265A9D
:10C4B0000446FDEEE77A85ED090A17EE902AC0F8EA
:10C4C000882CC3ED005A95ED036ADFED597AD0ED63
:10C4D000036AF6EE008AB4EEE86AF1EE10FAC8BF1D
:10C4E000F0EE477AC6ED007A66EEE77A17EE900A2C
:10C4F0000FF0F6F841EC100B0DF03EFC51EC100B78
:10C500000FF03AFC07EE100AF7EE007A77EEC77AE2
:10C51000B0EE007AC6ED007AD5ED047AA7EE878AF0
:10C5200004F69C4204F54A6382ED008A83ED008A9A
:10C5300095ED047AB4EEE87AF1EE10FA03D5F1EE57
:10C54000487AC3ED007ADFED3B6A95ED056A9FED11
:10C550003A7AD4ED037A9FED398AA6EE267A04F66C
:10C56000984627EE888A17EE100A0FF0B9F841ECCA
:10C57000100B0DF001FC51EC100B0FF0FDFB07EE62
:10C58000900A27EE888AF7EE007A86ED008A95ED0C
:10C59000067A77EE277A04F6D44377EE877AF5EEBB
:10C5A000006AC3ED007A95ED067AB4EEE67AF1EE14
:10C5B00010FA09D5B0EE086AF6EE086AE7EE466AA8
:10C5C00077EEE67AC3ED007A95ED077A9FED1C6A67
:10C5D000DFED1C7ADFED1C6A27EE067A04F6844351
:10C5E00083ED007A95ED097AB6EE006A37EE467A69
:10C5F00004F6B84383ED007A95ED0A7A67EE277A60
:10C6000004F54C6367EE877A04F6BC410022C1ED65
:10C61000007ABDEC028B1A60D5ED0B7A67EEA67A34
:10C6200004F6C444C4ED007A70BD00BF00C05A4691
:10C6300000409C453D0AC7403D0A27C0560EC940F0
:10C640008FC2F53C2DB29D3D6666E63F70B54568EC
:10C650009FED6C7A95ED025A95ED036AF2EE085A59
:10C66000F9EE087AE5EE257A00F6A44300F6A8462E
:10C67000F1EE006A2DED028B66EE266ABFEE008AAF
:10C68000F0EE485AE6EE265A0446FDEEE77A85EDCE
:10C690000A0A17EE902AC0F8882CC3ED005A95EDCF
:10C6A000036ADFED597AD0ED036AF6EE008AB4EE44
:10C6B000E86AF1EE10FAC8BFF0EE477AC6ED007AEC
:10C6C00066EEE77A17EE900A0FF00AF841EC100BCD
:10C6D0000DF052FB51EC100B0FF04EFB07EE100A61
:10C6E000F7EE007A77EEC77AB0EE007AC6ED007A00
:10C6F000D5ED047AA7EE878A04F69C4204F54A63D6
:10C7000082ED008A83ED008A95ED047AB4EEE87A32
:10C71000F1EE10FA03D5F1EE487AC3ED007ADFEDC1
:10C720003B6A95ED056A9FED3A7AD4ED037A9FED69
:10C73000398AA6EE267A04F6984627EE888A17EEFE
:10C74000100A0EF0CDFF41EC100B0DF015FB51EC73
:10C75000100B0FF011FB07EE900A27EE888AF7EE18
:10C76000007A86ED008A95ED067A77EE277A04F650
:10C77000D44377EE877AF5EE006AC3ED007A95ED43
:10C78000067AB4EEE67AF1EE10FA09D5B0EE086A50
:10C79000F6EE086AE7EE466A77EEE67AC3ED007ACF
:10C7A00095ED077A9FED1C6ADFED1C7ADFED1C6AC0
:10C7B00027EE067A04F6844383ED007A95ED097A34
:10C7C000B6EE006A37EE467A04F6B84383ED007A97
:10C7D00095ED0A7A67EE277A04F54C6367EE877A5F
:10C7E00004F6BC410022C1ED007ABDEC028B1A6058
:10C7F000D5ED0B7A67EEA67A04F6C444C4ED007A50
:10C8000070BD00BF00C05A4600409C453D0AC7406D
:10C810003D0A27C0560EC9408FC2F53C2DB29D3D42
:10C820006666E63F70B545689FED6C7A95ED025AF5
:10C8300095ED036AF2EE085AF9EE087AE5EE257AEC
:10C8400000F6A44300F6A846F1EE006A2DED028B37
:10C8500066EE266ABFEE008AF0EE485AE6EE265AE9
:10C860000446FDEEE77A85ED0B0A17EE902AC0F834
:10C87000882CC3ED005A95ED036ADFED597AD0EDAF
:10C88000036AF6EE008AB4EEE86AF1EE10FAC8BF69
:10C89000F0EE477AC6ED007A66EEE77A17EE900A78
:10C8A0000EF01EFF41EC100B0DF066FA51EC100B70
:10C8B0000FF062FA07EE100AF7EE007A77EEC77A09
:10C8C000B0EE007AC6ED007AD5ED047AA7EE878A3D
:10C8D00004F69C4204F54A6382ED008A83ED008AE7
:10C8E00095ED047AB4EEE87AF1EE10FA03D5F1EEA4
:10C8F000487AC3ED007ADFED3B6A95ED056A9FED5E
:10C900003A7AD4ED037A9FED398AA6EE267A04F6B8
:10C91000984627EE888A17EE100A0EF0E1FE41ECE9
:10C92000100B0DF029FA51EC100B0FF025FA07EE61
:10C93000900A27EE888AF7EE007A86ED008A95ED58
:10C94000067A77EE277A04F6D44377EE877AF5EE07
:10C95000006AC3ED007A95ED067AB4EEE67AF1EE60
:10C9600010FA09D5B0EE086AF6EE086AE7EE466AF4
:10C9700077EEE67AC3ED007A95ED077A9FED1C6AB3
:10C98000DFED1C7ADFED1C6A27EE067A04F684439D
:10C9900083ED007A95ED097AB6EE006A37EE467AB5
:10C9A00004F6B84383ED007A95ED0A7A67EE277AAC
:10C9B00004F54C6367EE877A04F6BC410022C1EDB2
:10C9C000007ABDEC028B1A60D5ED0B7A67EEA67A81
:10C9D00004F6C444C4ED007A70BD00BF00C05A46DE
:10C9E00000409C453D0AC7403D0A27C0560EC9403D
:10C9F0008FC2F53C2DB29D3D6666E63FD0F87C0CBB
:10CA0000704700BF2DE9F04F2DED028B151E83B04E
:10CA100006460F46D0F804A040F3D181D0F87C4CF4
:10CA2000017C8C4280F29A81342303FB04030022B0
:10CA3000611CC0F87C1CC3F8DC22C3F8D822A7F123
:10CA40003C094EF64F4309FB09F2C4F6C46383FB6D
:10CA50000231D317C3EBA10303EB430103EB8103C3
:10CA6000D31A07EE903AF8EEE77AB1EE0A7A06F6B4
:10CA7000BC4106F6B84377EEC77AD3ED006A91ED74
:10CA8000007A3C2FE7EE276A09DD07EE102A06F54B
:10CA90004C63D3ED007AB8EEC77AE7EE876AD6F832
:10CAA000883CB2691A44974240F30082726D1A447E
:10CAB000974240F32F82D6F890201A44974240F3D1
:10CAC0002682D6F8CC201A44974240F31D82D6F82D
:10CAD00008211A44974240F3FB81D6F844211A44B6
:10CAE000974240F3F281D6F880211A44974240F3EE
:10CAF000E981D6F8BC211A44974240F3E081D6F888
:10CB0000F8211A44974240F3D781D6F834221A44C8
:10CB1000974240F3CE81D6F8702213449F42CCBF97
:10CB20004FF021084FF01E084FEA880B0BEB08036B
:10CB300006EB8303D6ED037A5B699FEDE78A9FEDF1
:10CB4000E76AFB1A07EE103AB8EEC77A27EE888A32
:10CB500077EE267A67EE867A17EE900A0EF0C0FD21
:10CB600041EC100B0DF008F9342303FB046351EC86
:10CB7000100B00930FF000F907EE900A27EE888A59
:10CB8000009BBEEEC88A0022302DC3F8C02283ED80
:10CB9000AF8A07DD502DD4BF08F1010808F1020863
:10CBA0004FEA880BD84406EB88084FF0340E06F69F
:10CBB000D442D8F82030D2ED008AD8F81C00D8F83A
:10CBC00024100EFB0468013BC8F8C832C8F8C40240
:10CBD000C8F8CC1218EE900A0EF082FD07EE905ABB
:10CBE0009FEDBF7AF8EEE77ACDE9000167EE877A2C
:10CBF000B0EE088A17EE900A0EF072FD9DED001B54
:10CC000041EC100B0DF03CF9F0EE007A51EC100BFA
:10CC1000A8EEA78A0FF0B0F807EE900A28EE278A50
:10CC20003C2F88EDB48A00F32281DAED046A9FED8F
:10CC3000AD7ADFEDAD5ADFEDAD7A9FEDAD6A96EDE1
:10CC4000038A06F6C84393ED005A66EEA66A403D95
:10CC5000A6EE857A06F6CC4306F6D84105EE107AA4
:10CC6000F0EE476A07EE105AD3ED004AB8EEC77AE5
:10CC7000B8EEC55AE4EE876A342303FB0463E5EE9D
:10CC8000257AC3F8EC7206F68442F4EEE76AF1EE18
:10CC900010FA58BFF0EE667AF4EEC67AF1EE10FAAA
:10CCA000D4BF67EEA77ADFED937A68EE277A0B2F71
:10CCB000C3EDB87A6CDD6C2F40F33181D1ED007A91
:10CCC00092ED007A9FED8C6A27EE877AF0EE675A34
:10CCD000E7EE065A4EF685394FF0A858F0EE006A96
:10CCE000B0EE657AC4F20109B0EE476A97EEA66A23
:10CCF00083EDBA7A83EDB96ADAED007A77EEA77A36
:10CD000017EE900A0EF0ECFC02460B4640464946F0
:10CD10000EF086FB41EC100B0DF02EF8F1EE487A88
:10CD200053EC102B17EE900ACDE900230EF0D8FC3F
:10CD3000DDE900230EF028FD41EC100B0DF01CF88E
:10CD4000342351EC100B03FB04660FF015F8C6F802
:10CD5000D40203B0BDEC028BBDE8F08F002900F0D7
:10CD6000DC800024DFED657A2346024692EDB47A3A
:10CD7000B4EEE77AF1EE10FA48BF1C4603F1010366
:10CD800048BFF0EE477A994202F13402EED156E6FE
:10CD9000D1ED007A92ED007A9FED596A27EE877AFD
:10CDA000F0EE675AE7EE065A47F6E1294FF02058B1
:10CDB000F0EE006AB0EE657AC3F6D47994E7027CAF
:10CDC000002AC6D0044600254FF0800B04E0013550
:10CDD000AA4204F13404BCDDD4F8EC329F42F6D10F
:10CDE000D6F88C3C1BB1C4F8ECB2327CEFE7F068AB
:10CDF00080F000400EF074FCCDE9000138460EF0E2
:10CE00005DFC47F6E1234FF08042C3F684730EF0D9
:10CE1000BBFC00230022C4F218030EF003FB9AEDC2
:10CE2000017AF1EE047A67EE277A804617EE900ACF
:10CE300089460EF055FC02460B46404649460EF028
:10CE4000EFFA41EC100B0CF097FFDDE9000153EC19
:10CE5000102B0EF099FC41EC100B0CF08DFF51ECF7
:10CE6000100B0EF089FFC4F8D402327CAFE7C7F193
:10CE70003C0307EE903A9FED237AF8EEE77A67EEEF
:10CE8000877A17EE900A0EF02BFC41EC100B0CF099
:10CE900073FF51EC100B0EF06FFFD8EDB47A07EE74
:10CEA000100A67EE877AC8EDB47ABEE64FF0000844
:10CEB0003AE64FF01B0837E64FF0180834E64FF01B
:10CEC000150831E64FF012082EE64FF00F082BE65A
:10CED0004FF00C0828E600BF0000FA4620986C3D91
:10CEE0002497FF3B00004842CDCCCC3E00005C4282
:10CEF0000000524300442C47000040420000C6425C
:10CF0000000040C20AD7233C4FF009080CE64FF05E
:10CF1000060809E64FF0030806E60C468FE591ED9A
:10CF2000007AD2ED006A07EE909A67EE266AF8EE74
:10CF3000E77AF0EE475AE6EEA75A2B2FB0EE006ADA
:10CF4000F0EE656AD7EE066AC3EDBA5AC3EDB96A68
:10CF500006DC47F6E1294FF02058C3F6D479CBE63A
:10CF600038460EF0ABFB4BF651034FF06042C3F670
:10CF70009E730EF009FC00230022C3F6F0730EF03E
:10CF80004FFA80468946B7E670B50021064607F09D
:10CF9000EDFEC0B1B6F91E40B6F92010031D00F534
:10CFA000827533F9022B9442A8BF14469142B8BF50
:10CFB00011469D42F5D80123F48331843377BDE8CF
:10CFC000704007F08BBE70BD002070470020704796
:10CFD000F8B549F22044037AC1F6FF74242908BF4A
:10CFE000C2805B0001250E462046C1F3072117468B
:10CFF00084F83B3084F85E5084F85D5003F05CFFA9
:10D00000F1B2204603F058FFC7F30721204603F092
:10D0100053FFF9B2204603F04FFF2946204604F0A3
:10D0200023F8B0FA80F04009F8BD00BF2DE9F843BD
:10D0300049F22044037AC1F6FF740125AB4029462A
:10D040000746204684F83B3084F85E5084F85D50F3
:10D0500003F032FF0421204603F02EFF204600217A
:10D0600004F002F8B8B34FF0010846464FF000094B
:10D070003B7A012549F22040AB402946C1F6FF70BA
:10D0800084F83B3084F85E5084F85D5003F014FF60
:10D0900049F220400421C1F6FF7003F00DFF49F270
:10D0A00020404946C1F6FF7003F006FF49F22040D8
:10D0B0004146C1F6FF7003F0FFFE49F220402946C9
:10D0C000C1F6FF7003F0D0FF10B10020BDE8F88377
:10D0D000B0B2BDE8F8832B460222397A204604F02C
:10D0E0004FF80128BFD994F8381094F83950A94264
:10D0F00018D263184A1CD2B2187E84F838209542A0
:10D100004FEA00230ED922440231107E84F83810F1
:10D11000184320F0010040F001064FEA16295FFA9B
:10D1200086F8A5E74FF0FF08C1464FF0FF369FE7AE
:10D130002DE9F84349F22044037AC1F6FF74012532
:10D14000AB4029460746204684F83B3084F85E50C1
:10D1500084F85D5003F0B0FE2421204603F0ACFEBD
:10D160002046002103F080FFB8B34FF00108464687
:10D170004FF000093B7A012549F22040AB40294697
:10D18000C1F6FF7084F83B3084F85E5084F85D503F
:10D1900003F092FE49F220402421C1F6FF7003F013
:10D1A0008BFE49F220404946C1F6FF7003F084FE31
:10D1B00049F220404146C1F6FF7003F07DFE49F27E
:10D1C00020402946C1F6FF7003F04EFF10B1002049
:10D1D000BDE8F883B0B2BDE8F8832B460222397A65
:10D1E000204603F0CDFF0128BFD994F8381094F8F9
:10D1F0003950A94218D263184A1CD2B2187E84F85A
:10D20000382095424FEA00230ED922440231107E85
:10D2100084F83810184320F0010040F001064FEA6E
:10D2200016295FFA86F8A5E74FF0FF08C1464FF0D0
:10D23000FF369FE7F8B549F22044037AC1F6FF7440
:10D240000126B340074601F003052046314684F825
:10D250003B3084F85E6084F85D6003F02DFE0821A9
:10D26000204603F029FE2046002103F0FDFE98B37E
:10D2700000233A7A012649F22040B2403146C1F6F5
:10D28000FF701D4384F83B2084F85E6084F85D6085
:10D2900003F012FE49F220400821C1F6FF7003F0AE
:10D2A0000BFE49F22040C5F30721C1F6FF7003F0E1
:10D2B00003FE49F22040E9B2C1F6FF7003F0FCFD25
:10D2C00049F220403146C1F6FF7003F0CDFE08B1AF
:10D2D0000020F8BDA8B2F8BD33460222397A2046B4
:10D2E00003F04EFF0128C3D994F8381094F83900A0
:10D2F000814212D263184A1CD2B21B7E84F83820B5
:10D3000090424FEA032308D922440231127E84F866
:10D310003810134323F00303ABE76FF00303A8E7D0
:10D32000F8B549F22044027AC1F6FF745200012692
:10D3300000210546204684F83B2084F85E6084F88E
:10D340005D6003F0B9FD0E21204603F0B5FD2046D7
:10D35000002103F089FE88B3002603272B7A49F2C7
:10D3600020405B0001250021C1F6FF7084F83B30AE
:10D3700084F85E5084F85D5003F09EFD49F2204031
:10D380000E21C1F6FF7003F097FD49F220403946A7
:10D39000C1F6FF7003F090FD49F220403146C1F61E
:10D3A000FF7003F089FD49F220402946C1F6FF7065
:10D3B00003F05AFEB0FA80F04009F8BD334602226D
:10D3C000297A204603F0DCFE0128C5D994F83810EC
:10D3D00094F83900814216D263184A1CD2B21E7EDC
:10D3E00084F8382090424FEA06230CD922440231B7
:10D3F000167E84F838101E4326F4407646F44076B4
:10D40000370AF6B2AAE7FF263746A7E71F29F8B57D
:10D41000064652D80C294DD840F60D55327A49F2BD
:10D420002044C1F6FF74520001270021204684F8F1
:10D430003B2084F85E7084F85D7003F03DFD2E2182
:10D44000204603F039FD2046002103F00DFEC8B34D
:10D450000023327A49F22040520001260021C1F611
:10D46000FF701D4384F83B2084F85E6084F85D60A3
:10D4700003F022FD49F220402E21C1F6FF7003F097
:10D480001BFD49F22040C5F30721C1F6FF7003F0F0
:10D4900013FD49F22040E9B2C1F6FF7003F00CFD24
:10D4A00049F220403146C1F6FF7003F0DDFD38B18E
:10D4B0000020F8BD41EA0125B0E741F61F75ADE750
:10D4C000A8B2F8BD3B460222317A204603F058FE4E
:10D4D0000128BDD994F8381094F83900814214D24B
:10D4E00063184A1CD2B21B7E84F8382090424FEA5F
:10D4F00003230AD922440231127E84F838101343E0
:10D5000023F4F85323F01F03A3E74EF2E003CFF612
:10D51000FF739EE70023C4F2FE2307EE103A47F69E
:10D52000EE43C3F6FF6307EE903A70B5E0EE877AFC
:10D530000023C4F2FE2307EE103AFCEEE77A47F62A
:10D54000EE4382B0C3F6FF63CDED017A07EE903A69
:10D55000E0EE077A9DF80450027AFCEEE77A7F2D20
:10D56000CDED017A9DF804309CBFC5F17F052D02F9
:10D5700049F22044C1F6FF7494BF2DB200257F2BE1
:10D5800094BFC3F17F0300235200012620460021EF
:10D590001D4384F83B2084F85E6084F85D6003F0EE
:10D5A0008BFC2046222103F087FCC5F3072120468F
:10D5B00003F082FCE9B2204603F07EFC31462046AF
:10D5C00003F052FDB0FA80F0400902B070BD00BF18
:10D5D0000023C4F27C2307EE103A47F6EE43C3F66D
:10D5E000FF6307EE903AF0B5E0EE077A0023C4F24D
:10D5F000FE2307EE103AFCEEE77A47F6EE4383B0DF
:10D60000C3F6FF63CDED017A07EE903AE0EE877A3C
:10D610009DF804500646FCEEE77A3F2DCDED017AE9
:10D620009DF80400337A98BFC5F13F0549F22044C4
:10D63000C1F6FF744FF0010794BF2D0200257F282B
:10D6400094BFC0F17F020022BB40394620461543FB
:10D6500084F83B3084F85E7084F85D7003F02CFC35
:10D660000621204603F028FC2046002103F0FCFCA4
:10D67000A8B30023327A49F220400126B240314655
:10D68000C1F6FF701D4384F83B2084F85E6084F887
:10D690005D6003F011FC49F220400621C1F6FF70E5
:10D6A00003F00AFC49F22040C5F30721C1F6FF70E0
:10D6B00003F002FC49F22040E9B2C1F6FF7003F02A
:10D6C000FBFB49F220403146C1F6FF7003F0CCFC71
:10D6D00010B1002003B0F0BDA8B203B0F0BD3B46CE
:10D6E0000222317A204603F04BFD0128C1D994F87B
:10D6F000381094F83900814214D263184A1CD2B20F
:10D700001B7E84F8382090424FEA03230AD9224432
:10D710000231127E84F83810134323F47D5323F032
:10D720003F03A7E74CF28003CFF6FF73A2E700BFE9
:10D730002DE9F84F49F2204490F808E0C1F6FF7453
:10D740000E46C1F307294FEA4E0E4FF0010A494633
:10D7500007465FFA86F8204693461D4684F83BE06C
:10D7600084F85EA084F85DA003F0A6FB4146204645
:10D7700003F0A2FB2046002103F076FCC0B3002595
:10D780003B7A242E4BEA050549F2204008BFFD8074
:10D790005B0001264946C1F6FF7084F83B3084F8EF
:10D7A0005E6084F85D6003F087FB49F220404146EB
:10D7B000C1F6FF7003F080FB49F22040C5F307215A
:10D7C000C1F6FF7003F078FB49F22040E9B2C1F6E0
:10D7D000FF7003F071FB49F220403146C1F6FF7043
:10D7E00003F042FC00280CBF28460020BDE8F88F5B
:10D7F00053460222397A204603F0C2FC0128BED9E2
:10D8000094F8381094F83900814204D34FF0FF3374
:10D8100023EA0505B4E763184A1CD2B21B7E84F8DC
:10D82000382090424FEA0323F0D922440231127E7D
:10D8300084F838101343EBE72DE9F041437A2DEDDE
:10D84000028B0646B0EE408AF0EE608A49F2204430
:10D85000002B40F0E580C1F6FF740023C4F24023A2
:10D8600007EE103A47F6EE43C3F6FF6307EE903A31
:10D870000023E8EE077ACCF23C2306EE903AF4EE71
:10D88000E67AF1EE10FA00F1C780F4EEC77AF1EE15
:10D8900010FAC8BF5F2740F35681337A49F220451A
:10D8A0004FF00108C1F6FF7503FA08F34146284618
:10D8B00084F83B3084F85E8084F85D8003F0FCFAE5
:10D8C0001621284603F0F8FA2846002103F0CCFB85
:10D8D000002800F0E8800023327A4FF0010849F276
:10D8E000204002FA08F24146C1F6FF7047EA0305FC
:10D8F00084F83B2084F85E8084F85D8003F0DCFAD5
:10D9000049F220401621C1F6FF7003F0D5FA49F222
:10D910002040C5F30721C1F6FF7003F0CDFA49F2AC
:10D920002040E9B2C1F6FF7003F0C6FA49F2204088
:10D930004146C1F6FF7003F097FB0023C4F2402379
:10D9400007EE103A47F6EE43C3F6FF6307EE903A50
:10D950000023E8EE877ACCF23C2306EE903AF4EE10
:10D96000E67AF1EE10FA59D4F4EEC77AF1EE10FA35
:10D97000C8BF5F2740F3DE80337A49F220454FF07D
:10D980000108C1F6FF7503FA08F34146284684F8FA
:10D990003B3084F85E8084F85D8003F08DFA1E21B0
:10D9A000284603F089FA2846002103F05DFB002891
:10D9B00057D00025337A49F220400126B340314642
:10D9C000C1F6FF7084F83B3084F85E6084F85D60D7
:10D9D00003F072FA49F220401E21C1F6FF7003F0F5
:10D9E0006BFA3D4349F22040C5F30721C1F6FF70B1
:10D9F00003F062FA49F22040E9B2C1F6FF7003F089
:10DA00005BFABDEC028B49F220403146C1F6FF7053
:10DA1000BDE8F04103F028BB00273EE70027ABE755
:10DA2000037AC1F6FF740125AB402946204684F8ED
:10DA30003B3084F85E5084F85D5003F03DFA0821D5
:10DA4000204603F039FA2046002103F00DFB0028A0
:10DA500051D0032302224FF484713046FFF768FE51
:10DA6000FBE643460222317A284603F089FB01286F
:10DA70009FD995F8381095F83900814238D26B1843
:10DA80004A1CD2B21B7E85F8382090424FEA03230D
:10DA90002ED92A440231127E85F8381042EA030555
:10DAA00025F07F0586E743460222317A284603F0B7
:10DAB00067FB01287FF60FAF95F8381095F839000D
:10DAC000814212D26B184A1CD2B21B7E85F83820D4
:10DAD00090424FEA032308D92A440231127E85F886
:10DAE0003810134323F07F03F6E66FF07F03F3E66D
:10DAF0006FF07F055EE72B460222317A204603F065
:10DB00003FFBA842A5D994F8383094F839108B42DD
:10DB10009FD25A19D2B2914284F8382099D922441E
:10DB20000233127E84F8383002F00303022B3FF4F4
:10DB300094AE8EE79FED087A77EE877AFCEEE77A6F
:10DB400017EE907A18E79FED047A77EE877AFCEE6D
:10DB5000E77A17EE907AA0E600003C422DE9F04FFC
:10DB60002DED028B49F22044027AC1F6FF7483B096
:10DB700052000125002180462046B0EE408A84F8FC
:10DB80003B2084F85E5084F85D5003F095F90E2137
:10DB9000204603F091F92046002103F065FA0028A1
:10DBA00000F0D580B5EEC08AF1EE10FA56DCB5EE85
:10DBB000C08AF1EE10FA00F344810C26B1464FF012
:10DBC000FF0A98F8082049F22045C1F6FF75520077
:10DBD0004FF0010B0021284684F83B2084F85EB00A
:10DBE00084F85DB003F068F90E21284603F064F96B
:10DBF0002846002103F038FA0746002800F0F1809B
:10DC0000002798F8083049F220405B0001250021E8
:10DC1000C1F6FF7084F83B3084F85E5084F85D50A4
:10DC200003F04AF949F220400E21C1F6FF7003F0DB
:10DC300043F949F220403946C1F6FF7003F03CF940
:10DC400049F220403146C1F6FF7003F035F949F240
:10DC500020402946C1F6FF7003F006FA0023C4F203
:10DC6000403307EE103A47F6EE43C3F6FF6307EE84
:10DC7000903AE8EE077A98F8082049F22047FCEE3F
:10DC8000E77AC1F6FF77CDED017A9DF80450C02DFB
:10DC900098BFC5F1FC054FEA42024FF001094FF071
:10DCA0000001384694BF45EA052543F63C4584F813
:10DCB0003B2084F85E9084F85D9003F0FDF810211D
:10DCC000384603F0F9F83846002103F0CDF906464E
:10DCD00000285BD0002698F8083049F220405B000D
:10DCE00001270021C1F6FF7084F83B3084F85E7094
:10DCF00084F85D7003F0E0F849F220401021C1F68D
:10DD0000FF7003F0D9F8354349F22040C5F30721ED
:10DD1000C1F6FF7003F0D0F849F22040E9B2C1F635
:10DD2000FF7003F0C9F849F220403946C1F6FF7090
:10DD300003F09AF928B1002003B0BDEC028BBDE8D6
:10DD4000F08FA8B203B0BDEC028BBDE8F08F0646A1
:10DD50002B46022298F80810204603F011FA0128F9
:10DD60007FF620AF94F8383094F839108B422AD3DC
:10DD70000C23B5EEC08AF1EE10FA67DD002B3FF4FC
:10DD80006DAF4FF0F30A4FF000091AE74B4602223D
:10DD900098F80810384603F0F3F901289AD997F853
:10DDA000383097F83920934209D2591CC9B28A42B7
:10DDB00087F8381003D9023387F838308BE700260C
:10DDC000CFF6FF7687E75A1CD2B2914284F838200A
:10DDD000CED922440233127E84F8383002F00C038C
:10DDE000C7E75B46022298F80810284603F0C8F9F6
:10DDF00058457FF606AF95F8382095F839008242ED
:10DE00001CD2A91802EB0B03DBB2097E85F838306F
:10DE100098424FEA012111D92B44023293F818A0FD
:10DE200085F838204AEA010A2AF00C0A4AEA090968
:10DE30005FFA89FA4FEA19275646E2E6FF27564667
:10DE4000DFE60026B1464FF0F30ABAE60C2B3FF4AA
:10DE500005AFACE6F8B549F22044037AC1F6FF7489
:10DE60000125AB4029460746204684F83B3084F81C
:10DE70005E5084F85D5003F01FF80021204603F047
:10DE80001BF80021204603F017F82946204603F02E
:10DE900013F82946204603F0E7F808B10020F8BD42
:10DEA0003B7A84F85E505B0006460146204684F8C3
:10DEB0003B3084F85D5002F0FFFF0A21204602F05B
:10DEC000FBFF3146204602F0F7FF7021204602F0AA
:10DED000F3FF2946204603F0C7F8B0FA80F0400966
:10DEE000F8BD00BFFFFFFFFFF3EE047A80EE277A54
:10DEF0002DE9F04F98464FF4AA43C4F6571307464E
:10DF000091460E4649F22044C1F6FF742DED068B72
:10DF100017EE100A83B008EE103AB0EE60AAF0EEE9
:10DF2000418A0DF0DDFB9FED9E0B41EC110B0BF0D8
:10DF3000A7FFCAEE087AB0EE409AF0EE609A01258B
:10DF400008EA0508F1EE677A17EE900A0DF0C8FBB3
:10DF50009FED930B41EC110B0BF092FFC8EE887A0A
:10DF60005BEC10ABF1EE677A17EE900A0DF0B8FBA0
:10DF70009FED8B0B41EC110B0BF082FF3B7A84F889
:10DF80005E50AB40294620468DED000B84F83B30B7
:10DF900084F85D5002F090FF2621204602F08CFFAD
:10DFA0000021204602F088FF45F61C234FF0204256
:10DFB000C3F6E47351EC190B0DF0E6FB00230022CD
:10DFC000C4F2E0030DF0E0FB0DF0B6FEC1B2204656
:10DFD00002F072FF2946204603F046F83B7A84F8A7
:10DFE0005E50AB402946204684F83B3084F85D50B3
:10DFF00002F062FF2821204602F05EFF0021204649
:10E0000002F05AFF002152465B460020C3F6F07131
:10E010000DF006FA00230022C4F220130DF0B4FB29
:10E020000DF08AFEC1B2204602F046FF2946204686
:10E0300003F01AF83B7A84F85E50AB40294620463C
:10E0400084F83B3084F85D5002F036FF2A212046E8
:10E0500002F032FF0021204602F02EFF9DED000B62
:10E06000002153EC102B0020C3F6F0710DF0D8F90D
:10E0700000230022C4F260130DF086FB0DF05CFE5D
:10E08000C1B2204602F018FF2946204602F0ECFFFC
:10E090003A7A84F85E504FEA481309F00308022EDA
:10E0A00043EA0828294602FA05F3204628BF02263B
:10E0B00084F83B3084F85D5002F0FEFE24212046B7
:10E0C00002F0FAFE2046002148EA063602F0CCFFB4
:10E0D00000283BD000233A7A012549F22040AA408B
:10E0E0002946C1F6FF701E4384F83B2084F85E5039
:10E0F00084F85D5002F0E0FE49F220402421C1F690
:10E10000FF7002F0D9FE49F22040C6F30721C1F6A4
:10E11000FF7002F0D1FE49F22040F1B2C1F6FF706B
:10E1200002F0CAFE49F220402946C1F6FF7002F013
:10E130009BFF28B1002003B0BDEC068BBDE8F08F3B
:10E14000B0B203B0BDEC068BBDE8F08F2B460222C7
:10E15000397A204603F014F80128BBD994F8381016
:10E1600094F83900814214D263184A1CD2B21B7E43
:10E1700084F8382090424FEA03230AD9224402311E
:10E18000127E84F83810134323F44C5323F02003F9
:10E19000A1E74CF6DF43CFF6FF739CE7AFF30080B7
:10E1A00000000000000024402DE9F041074649F23C
:10E1B0002044C1F6FF74012520463D7102F090FE17
:10E1C000052008F0D9FA3B7A84F85E50AB40002174
:10E1D000204684F83B3084F85D5002F06DFE30211B
:10E1E000204602F069FE4021204602F065FE6021D3
:10E1F000204602F061FE2946204602F035FF10B1AC
:10E200000020BDE8F0813B7A84F85E5006465B0052
:10E210000146204684F83B3084F85D5002F04CFE05
:10E220002621204602F048FE3146204602F044FEF8
:10E230006C21204602F040FE2946204602F014FFE1
:10E240003B7A84F85E505B003146204684F83B30D0
:10E2500084F85D5002F030FE2821204602F02CFEAA
:10E260002946204602F028FEF221204602F024FE34
:10E270002946204602F0F8FE3B7A84F85E505B00A7
:10E280003146204684F83B3084F85D5002F014FE9D
:10E290002C21204602F010FE0F21204602F00CFE39
:10E2A0002221204602F008FE2946204602F0DCFE2C
:10E2B0003B7A84F85E505B003146204684F83B3060
:10E2C00084F85D5002F0F8FD3C21204602F0F4FD98
:10E2D0004421204602F0F0FD4621204602F0ECFDEC
:10E2E0002946204602F0C0FE3B7A40F23712FA80FF
:10E2F0005B003146204684F83B3084F85E5084F859
:10E300005D5002F0D9FD2421204602F0D5FD2946BA
:10E31000204602F0D1FD3721204602F0CDFD2946EE
:10E32000204602F0A1FE3B7A84F85E505B00314645
:10E33000204684F83B3084F85D5002F0BDFD30216A
:10E34000204602F0B9FD4021204602F0B5FDFF2134
:10E35000204602F0B1FD2946204602F085FE3B7AB8
:10E3600084F85E505B003146204684F83B3084F8E8
:10E370005D5002F0A1FD0221204602F09DFD3146D4
:10E38000204602F099FD7321204602F095FD2946B2
:10E39000204602F069FE4FF4C87008F0EDF93B7AB0
:10E3A00084F85E505B003146204684F83B3084F8A8
:10E3B0005D5002F081FD2E21204602F07DFD1D21E1
:10E3C000204602F079FD1D21204602F075FD294608
:10E3D000204602F049FE3B7A84F85E505B003146ED
:10E3E000204684F83B3084F85D5002F065FD04213E
:10E3F000204602F061FD3146204602F05DFD042119
:10E40000204602F059FD2946204602F02DFE3B7AB7
:10E4100084F85E505B003146204684F83B3084F837
:10E420005D5002F049FD0621204602F045FD2946D7
:10E43000204602F041FD3021204602F03DFD2946F4
:10E44000204602F011FE3B7A84F85E505B003146B4
:10E45000204684F83B3084F85D5002F02DFD0A21FF
:10E46000204602F029FD3146204602F025FD10210C
:10E47000204602F021FD2946204602F0F5FD3B7AB8
:10E4800084F85E505B003146204684F83B3084F8C7
:10E490005D5002F011FD0E21204602F00DFD3146C7
:10E4A000204602F009FD3146204602F005FD2946CE
:10E4B000204602F0D9FD3B7A84F85E505B0031467D
:10E4C000204684F83B3084F85D5002F0F5FC1021C2
:10E4D000204602F0F1FC3C21204602F0EDFC3C21FC
:10E4E000204602F0E9FC2946204602F0BDFD3B7AB9
:10E4F00084F85E505B003146204684F83B3084F857
:10E500005D5002F0D9FC2221204602F0D5FC7F218B
:10E51000204602F0D1FC7F21204602F0CDFC2946A6
:10E52000204602F0A1FD3B7A4FF036085B00A7F8C9
:10E5300006803146204684F83B3084F85E5084F8EB
:10E540005D5002F0B9FC2421204602F0B5FC3146B2
:10E55000204602F0B1FC4146204602F0ADFC2946BF
:10E56000204602F081FD7D722846BDE8F08100BFA3
:10E570002DE9F8430023C4F2013307EE103A47F6C1
:10E58000EE43C3F6FF6307EE903AE0EE077A0646E5
:10E59000FCEEE77A17EE904A002C71D0802C39D926
:10E5A000337900242746002B3ED149F22045C1F69D
:10E5B000FF75337A49F220405B0001260021C1F645
:10E5C000FF7085F83B3085F85E6085F85D6002F08D
:10E5D00073FC49F220402221C1F6FF7002F06CFC6E
:10E5E00049F220403946C1F6FF7002F065FC49F25D
:10E5F00020402146C1F6FF7002F05EFC49F2204047
:10E600003146C1F6FF7002F02FFDB0FA80F04009EC
:10E61000BDE8F883C4F18004337944EA0424C4F3E8
:10E620000727E4B2002BC0D0B6F80680337A49F24F
:10E630002045C1F6FF7528F0100800215B003171FC
:10E64000A6F806804FF00109284685F83B3085F88A
:10E650005E9085F85D9002F02FFC2846242102F0A0
:10E660002BFC4FEA1821284602F026FC08F0EF01A7
:10E67000284602F021FC4946284602F0F5FC98E7BE
:10E68000037A49F22045C1F6FF75012717EE901A6B
:10E69000BB400771284685F83B3085F85E7085F8E9
:10E6A0005D7002F009FC2846222102F005FC284694
:10E6B0007F2102F001FC28467F2102F0FDFB394654
:10E6C000284602F0D1FCB6F80680337A48F01008EC
:10E6D0001FFA88F8BB40A6F806802146284685F830
:10E6E0003B3085F85E7085F85D7002F0E5FB2846EA
:10E6F000242102F0E1FB4FEA1821284602F0DCFB5E
:10E700005FFA88F1284602F0D7FB3946284602F026
:10E71000ABFCB0FA80F04009BDE8F883F8B50646D6
:10E720000D4619B1012948D00020F8BD037A49F2FD
:10E730002044C1F6FF745B000127204684F83B307B
:10E7400084F85E7084F85D7002F0B6FB20212046EC
:10E7500002F0B2FB2946204602F0AEFB55212046CE
:10E7600002F0AAFB3946204602F07EFC0028DBD1ED
:10E77000F588337A45F00405ADB25B00F5800146BB
:10E78000204684F83B3084F85E7084F85D7002F0B7
:10E7900093FB2421204602F08FFB290A204602F039
:10E7A0008BFBE9B2204602F087FB3946204602F097
:10E7B0005BFCB0FA80F04009F8BD037A49F22044CE
:10E7C000C1F6FF745B000021204684F83B3084F8DA
:10E7D0005E5084F85D5002F06FFB2A21204602F063
:10E7E0006BFB2946204602F067FB7321204602F0AE
:10E7F00063FB2946204602F037FC0746002893D1E8
:10E80000337A84F85E505B000146204684F83B3042
:10E8100084F85D5002F050FB2021204602F04CFBB2
:10E820003946204602F048FB8821204602F044FB8E
:10E830002946204602F018FC00287FF475AFF788BF
:10E84000337A27F004075B00F7800146204684F8FE
:10E850003B3084F85E5084F85D5002F02DFB24219B
:10E86000204602F029FB390A204602F025FB07F07A
:10E87000FB01204602F020FB2946204602F0F4FB73
:10E88000B0FA80F04009F8BD2DE9F04F9BB0044686
:10E8900006F0CCF91690002800F05F820021204697
:10E8A00006F064FA1790002800F060824FF6F053EB
:10E8B000C0F20E03199345F24C6945F24E6734F9E4
:10E8C0000930049345F25266E35F099345F25460C0
:10E8D000A35F089345F25661235E189345F2586290
:10E8E000635E059345F25A6AA35E079334F90A30D2
:10E8F000069304F5AC431A4604F5C5491E46CDF807
:10E90000449002F13C093E320B9206F140020C9217
:10E9100006F142020D9206F144020E9206F1460201
:10E920000F9206F14802119B109232464A3203922E
:10E930001A46183211921A461A3245F2506512924E
:10E9400045F25E681A4645F25C6C45F2606E1C3218
:10E950001E3334F905B0139234F9088034F90CC031
:10E9600034F90EE0CDF808901493179B18989A1C70
:10E970000192169A03F5817302321593019B0A9254
:10E980004FF0000A5D4633F9022F019302EB0212A9
:10E9900002EB0222520022F34F42029B04991E888E
:10E9A00004EB460701FB0CF9B7F91C3003FB08998F
:10E9B00029F3CF390FFA89F1049112B201FB0EF954
:10E9C00029F3CF39914409F30F090136A7F81C90B8
:10E9D0000299B6B240F25B47BE4294BF0E80A1F8E6
:10E9E00000A00B99099F0E8804EB460907FB0CFB5E
:10E9F000B9F9D4783B4407FB08BB2BF3CF3B0FFAA4
:10EA00008BF7099707FB0EF727F3CF37174407F368
:10EA10000F070136A9F8D4780B99B6B240F2A34794
:10EA2000BE4294BF0E80A1F800A00C990E8804EBA2
:10EA3000460707F590571C37B7F9009005FB0CF512
:10EA40004B4409FB085525F3CF352DB205FB0EF9D4
:10EA500029F3CF39914409F30F090136A7F8009043
:10EA6000B6B240F2FC47BE4294BF0E80A1F800A0AF
:10EA70000D990E88089904EB460707F5E0571637FD
:10EA8000B7F9009001FB0CFB4B4409FB08BB2BF3CF
:10EA9000CF3B0FFA8BF9CDF8209009FB0EF929F343
:10EAA000CF39914409F30F090136A7F800900D9969
:10EAB000B6B240F24B57BE4294BF0E80A1F800A000
:10EAC0000E990E8804EB460707F51A572E37B7F94B
:10EAD000009000FB0CF04B4409FB080020F3CF3002
:10EAE00000B200FB0EF929F3CF39914409F30F0965
:10EAF0000136A7F80090B6B240F28D57BE4294BFDF
:10EB00000E80A1F800A00F990E88059904EB460726
:10EB100007F547570A37B7F9009001FB0CFB4B4448
:10EB200009FB08BB2BF3CF3B0FFA8BF9CDF8149000
:10EB300009FB0EF929F3CF39914409F30F09013686
:10EB4000A7F800900F99B6B240F2D257BE4294BFD8
:10EB50000E80A1F800A010990E88079904EB4607D3
:10EB600007F575573037B7F9009001FB0CFB4B44A4
:10EB700009FB08BB2BF3CF3B0FFA8BF9CDF81C90A8
:10EB800009FB0EF929F3CF39914409F30F09013636
:10EB9000A7F800901099B6B240F21467BE4294BF35
:10EBA0000E80A1F800A003990E88069904EB460791
:10EBB00007F593471A37B7F9009001FB0CF14B4466
:10EBC00009FB081121F3CF3109B2069101FB0EF9BF
:10EBD00029F3CF394A4402F30F020136B6B2B6F533
:10EBE000CA6F3A808ABF039A0399A2F800A047F639
:10EBF000E12298BF0E8002FB03F323F34F431199E8
:10EC00000E8804EB460707F5AC470FFA83F9B7F90E
:10EC1000622003EB6203A7F86230C9EB020222F321
:10EC20004F020136B6B2B6F50B7F34BF0E80A1F8A5
:10EC300000A012990E8804EB460707F5B5470FFAB6
:10EC400082F9B7F93A3002EB63027A87C9EB030322
:10EC500023F34F030136B6B2B6F5DC7F94BF0E80C6
:10EC6000A1F800A013990E8804EB460707F5BC47EE
:10EC70000FFA83F9B7F92C2003EB6203BB85C9EBCC
:10EC8000020222F34F020136B6B2B6F5AA7F94BF54
:10EC90000E80A1F800A014990E8804EB460707F532
:10ECA000C1470FFA82F9B7F9563002EB6302A7F8B1
:10ECB0005620C9EB030323F34F030136B6B21BB250
:10ECC000E02EC3EB031394BF0E80A1F800A05B00FD
:10ECD00003F30F030A9A22F8023F019B0A92159A46
:10ECE00093427FF450AE0499002213461E4661F30E
:10ECF0000F02079965F30F03354661F30F05099974
:10ED000061F31F42089961F31F43059960F30F06F1
:10ED100061F31F46069945F2546E45F2586C45F270
:10ED2000506045F24C6761F31F45E251235044F8AF
:10ED30000E60204644F80C50169C0022214605F037
:10ED4000FBFF204605F0CAFF1798199A90420AD097
:10ED50001BB0BDE8F04F05F0C1BF0146204606F0EC
:10ED600005F80028F4D11BB0BDE8F08F4FF6F05342
:10ED7000C0F20E03199317939DE500BFF8B540F25A
:10ED80001C030446C0F2020303600021012004F1C9
:10ED900018020B46607222612172E16000E0226974
:10EDA00042F82310627A01339A42F8DC4FF288531A
:10EDB000C2F200031A680AB9B9E01A465369002B77
:10EDC000FBD1546120464FF6FC630025C0F20E03D0
:10EDD0006561A580E580A572294640F81C3B40F698
:10EDE000B8020DF001FD294640F6481204F6D400A1
:10EDF0000DF0FAFC04F59050294640F6FA121C304A
:10EE00000DF0F2FC04F5E050294640F69822163049
:10EE10000DF0EAFC04F51A50294640F61C322E305B
:10EE20000DF0E2FC04F54750294640F6A6320A30C0
:10EE30000DF0DAFC04F57550294640F62A423030D0
:10EE40000DF0D2FC04F59340294640F6A2421A3058
:10EE50000DF0CAFC45F23C6345F23E6045F2406766
:10EE600045F2426145F24462E55245F2466625525A
:10EE700045F2486345F24A60E553655245F24C67F6
:10EE8000A55245F24E6145F25062A553E55245F256
:10EE90005266255245F2546345F25660E553655279
:10EEA00045F25867A55245F25A6145F25C62A55396
:10EEB000E55245F25E66255245F2606341F69910CF
:10EEC000E553655246F26767A05246F6843204F570
:10EED000AC402946A7536230E2524FF48B620DF0EA
:10EEE00083FC04F5B540294640F272323A300DF009
:10EEF0007BFC04F5BC40294640F2AA222C300DF0E0
:10EF000073FC04F5C14029464FF4E17256300DF010
:10EF10006BFC46F2982046F29A2146F29C2246F279
:10EF20009E23255265522046A552E552F8BD1C602D
:10EF300048E700BF10B5044606F03EF9204610BD74
:10EF400049F2A0224EF635714EF65810C1F6FF7206
:10EF5000C0F20001C2F200000DF0D2B838B549F29B
:10EF6000A0254EF63574C1F6FF75C0F200044EF6CA
:10EF700060102A462146C2F200000DF0C1F84EF69C
:10EF800068102A462146C2F20000BDE838400DF064
:10EF9000B7B800BF49F2A0224EF635714EF6701098
:10EFA000C1F6FF72C0F20001C2F200000DF0A8B875
:10EFB00049F2A0224EF635714EF67810C1F6FF7276
:10EFC000C0F20001C2F200000DF09AB849F2A0228E
:10EFD0004EF635714EF68010C1F6FF72C0F2000198
:10EFE000C2F200000DF08CB849F2A0224EF6357145
:10EFF0004EF68810C1F6FF72C0F20001C2F20000A6
:10F000000DF07EB82DE9F04F00F5807EB1E8A00A42
:10F01000B2E84015C5EA0643C6EA2544C7EA0845F2
:10F02000C8EA2746C9EA0A47CAEA2948CBEA0C498E
:10F03000CCEA2B4AA0E8F8078645E7D1BDE8F04FB7
:10F0400070474FF000022DE9F00F00F5807C00BF03
:10F05000B1E8A00AC5EA0203C2EA2544C7EA0205EC
:10F06000C2EA2746C9EA0207C2EA2948CBEA0209EE
:10F07000C2EA2B4AA0E8F8078445E9D1BDE8F00FC1
:10F0800070474FF000022DE9F00F00F5807C00BFC3
:10F09000B1E8A00AC2EA0543C2EA0504C2EA07458C
:10F0A000C2EA0706C2EA0947C2EA0908C2EA0B49EE
:10F0B000C2EA0B0AA0E8F8078445E9D1BDE8F00FE1
:10F0C00070472DE9F00F089C00F5007B51F8045BB8
:10F0D00053F8046BC5EA0647C6EA254952F8045BB3
:10F0E00054F8046BC5EA0648C6EA254AA0E880073A
:10F0F0008345EBD1BDE8F00F704700BF2DE9F84321
:10F100004FF00008064600F11805474641463046D4
:10F11000002F4FD005F02AFEF0B12C68B4F5803FE7
:10F1200007F1040100F1040E07F5827C27D05EF898
:10F13000042B34FB02F334FB12F903F30F0209F33F
:10F140000F03C2EA03430A6893FA12F341F8043B3F
:10F150008C45ECD805F0C2FD08F10108B8F1040FA8
:10F1600005F10405D2D1002F40D0304639460022A7
:10F1700005F0E2FD3846BDE8F84305F0AFBD07F104
:10F180000C0100F10C0451F8083C54F8082C93FAD7
:10F1900012F341F8083C54F8042C51F8043C93FA5B
:10F1A00012F38C4541F8043C04F1080401F1080114
:10F1B000E9D8CFE705F0E6FD07460028CCD028685F
:10F1C000B0F5803FC8D0391D07F582740B6830FB5D
:10F1D00003F230FB13F302F30F0203F30F03C2EA4F
:10F1E000034341F8043B8C42F0D8B5E7BDE8F8830F
:10F1F00070B584692CB3B4F5803F06464FF000012A
:10F2000025D005F0BFFD054600B3011D00F5827055
:10F210000B6834FB03F234FB13F302F30F0203F326
:10F220000F03C2EA034341F8043B8842F0D830465A
:10F230000022294605F080FD2846BDE8704005F013
:10F240004DBD214605F092FD0028F6D170BD05F0B8
:10F250008DFD04460028F9D030462146002205F0F5
:10F260006BFD2046BDE8704005F038BD49F2A02294
:10F270004EF635714EF69010C1F6FF72C0F20001E5
:10F28000C2F200000CF03CBF49F2A0224EF63571EC
:10F290004EF69810C1F6FF72C0F20001C2F20000F3
:10F2A0000CF02EBF49F2A0224EF635714EF6A0109A
:10F2B000C1F6FF72C0F20001C2F200000CF020BFE4
:10F2C0002DE9F84F4EF6AC13C2F2000348F21F02CC
:10F2D00019681B79096848F20050C1F6FF70C4F242
:10F2E00000028142137035D24EF6C413C2F20003FD
:10F2F0001B7893BB4EF6BC19C2F200094EF6B41847
:10F300004EF6A8154EF6B816C2F20008C2F2000575
:10F31000C2F20006D9F800A0D8F800B02C883788CF
:10F32000BAF1000F45D0BBF1000F3AD00BF1040247
:10F330000AF1040102EB470201EB4401FFF762FE10
:10F34000403740347F2C1ED82C807F2F0CD837803C
:10F35000BDE8F88FA0F58070CCE74EF20823CEF21E
:10F36000000301221A60C5E700245846348005F0E6
:10F37000B5FC4EF6C013C2F200031A68C8F80020AC
:10F380001C60BDE8F88F002450462C8005F0A6FCD8
:10F390004EF6C813C2F200031A68C9F800201C60B8
:10F3A000D3E70AF1040101EB4401FFF74AFE4034C0
:10F3B000C8E7BBF1000F07D00BF1040101EB4701D7
:10F3C000FFF75FFE4037BDE74FF4807259460DF0FE
:10F3D0000BFAB7E7F8B50021054605F0C7FCC8B140
:10F3E00072B64EF6BC13C2F200031968002938D079
:10F3F0004EF6C812C2F20002166866B34EF6A814A2
:10F40000C2F2000400271E601060278062B6084622
:10F4100005F064FC2846012105F0A8FCD0B172B6C5
:10F420004EF6B413C2F200031C6814B34EF6C012B9
:10F43000C2F2000215688DB14EF6B811C2F2000199
:10F4400000261D6010600E8062B62046BDE8F840C0
:10F4500005F044BCF8BD106062B6DBE7106062B630
:10F46000F8BD4EF6A812C2F200021860118062B612
:10F47000D0E74EF6B812C2F200021860148062B6ED
:10F48000F8BD00BF4EF6AC10F8B5C2F20000012185
:10F4900005F0ECFD48F23C03C4F204034EF6BC1444
:10F4A00019684EF6B410C2F20004C2F2000048F22D
:10F4B00040020025C4F2040241F4004125600560C9
:10F4C0001960116841F0020111601A684FF470412F
:10F4D00042F00202C4F202011A600B68AB427DDB0B
:10F4E0004FF28003C4F202031B68AB4276DB4FF499
:10F4F0007142C4F202024FF0804313601368002B84
:10F50000FCDB4FF20410C4F202004FF26003C4F2BD
:10F5100002034FF2FE054FF2040E0560C4F2020E24
:10F5200000251D604FF2080101234FF20C07CEF8B1
:10F530000030C4F20201C4F202079E46C0F2007E0F
:10F540004FF4803C4FF21002C1F800E0C4F2020216
:10F55000C7F800C041F61B7763F31F474FF214064C
:10F560004FF2E0044FF284001760C4F20206C4F2C6
:10F570000204C4F202004FF288014FF4F852C4F2C0
:10F580000201C1F61F7241F61B77326063F31F4719
:10F5900025600360C4F200730B604FF28C0E4FF2D3
:10F5A00090064FF294054BF208044BF20C004BF21C
:10F5B0001801C4F2020EC4F20206C4F20205C4F23B
:10F5C0000404C4F20400C4F204014FF4C063CEF892
:10F5D00000C037602A60236003600B604EF6AC14F5
:10F5E000C2F200044BF204002368C4F2040048F2A3
:10F5F000004202214FF4C065C1F6FF7205601A6037
:10F6000099802279996002F180424FF2220102F53D
:10F610000432C4F2020140F201164FF47E45196132
:10F62000DE8000214FF48070CFF6FF7506278D260F
:10F63000D882DD609982D88399619F83117016709A
:10F6400005F0B0FC22794EF6C4115311C2F200014C
:10F6500048F21B06C4F200069B00087003F16043E9
:10F6600002F01F004FF4704548F20064012132702F
:10F67000C4F2020502F11007814003F56143C1F6AF
:10F68000FF7401204FF2C122C9F200004FF08076D2
:10F69000C0F200022E60286044F827201960F8BDEF
:10F6A00049F2A0224EF635714EF6AC10C1F6FF724B
:10F6B000C0F20001C2F200000CF022BD49F2A0220B
:10F6C0004EF635714EF6CC10C1F6FF72C0F2000155
:10F6D000C2F200000CF014BD49F2A0224EF63571C2
:10F6E0004EF6D410C1F6FF72C0F20001C2F2000063
:10F6F0000CF006BD49F2A0224EF635714EF6DC1034
:10F70000C1F6FF72C0F20001C2F200000CF0F8BCBA
:10F7100049F2A0224EF635714EF6E410C1F6FF72A2
:10F72000C0F20001C2F200000CF0EABC49F2A022D3
:10F730004EF635714EF6EC10C1F6FF72C0F20001C4
:10F74000C2F200000CF0DCBC90F89D3090F89C20D8
:10F75000DBB2934215D001331F2B84BF00210B462F
:10F7600010B598BFD9B20633002250F8234080F874
:10F770009D10214605F0E0FA2046BDE8104005F056
:10F78000ADBA7047D0F898300BB10120704710B572
:10F79000044605F04BFAC4F89800003018BF012069
:10F7A00010BD00BF10B50446D0F8980018B1043061
:10F7B00010BD09F0C9FC05F039FAC4F8980000281A
:10F7C000F7D0043010BD00BFD0F89810B1B190F858
:10F7D0009C2001321F2A10B4CABF0024D4B2224692
:10F7E00090F89D309342FBD00632002340F822105F
:10F7F00080F89C405DF8044BC0F89830704700BF1B
:10F8000010B4047F4160022CC26003D05DF8044B49
:10F8100005F0F0BC83685DF8044B1847F0B449F27A
:10F820007033C1F6FF7348F21F02996BC4F20002F5
:10F8300008791070586B48F21C02C4F20002047977
:10F840001470097911701A6B002A4FD05968C96871
:10F850008A4247D80168CC8B240402F1FF3073D46C
:10F86000C0F30E00C883C88B80B2C882996B096848
:10F87000C88B000460D4C2F30E00C883C88B002478
:10F8800080B212F1FF32C88218BF01221C63596B8B
:10F89000086849F270310568C1F6FF7101F12C0466
:10F8A000A54241D00968CC6814F0804F046805680F
:10F8B00015BF248824780235013544F000440560E2
:10F8C0004C63996B48F21B03C4F200030979197069
:10F8D00049F27031C1F6FF7112B14A6B12791A7098
:10F8E000F0BC7047521A1A630122D0E71968D86B2E
:10F8F0000A630024CFF60F74CC620468CD682668D2
:10F900004FF60104C0F2000425F080450327A6420B
:10F91000CD6083F82D701FD1037F4260022BC2603F
:10F920001ED0F0BC05F066BC086891F82C10C468C5
:10F9300041F000414163C4E7CC8BC2F3080004F4FA
:10F940007E442043C88399E7CC8BC0F3080004F4BD
:10F950007E442043C88386E733461146F0BC1847EF
:10F960008368F0BC184700BF00207047704700BF95
:10F970004EF6F413C2F2000302224FF6CC71C0F22D
:10F980000E015A600022D9629A7083F8242083F80D
:10F99000302083F83220704741F23801C4F20B0165
:10F9A00041F230020B6823F0805323F00A030B600E
:10F9B000C4F20B0213689907FCD541F22C03C4F280
:10F9C0000B031A68920703D51A6822F002021A6024
:10F9D00041F22803C4F20B034EF64822196821F0C5
:10F9E000080119601968C2F2000241F00801012003
:10F9F00019601060704700BF830769D1F0B54EF6FB
:10FA00004C24C2F2000423780BB10320F0BD41F274
:10FA10002402C4F20B0215461368DE07FCD42B68DF
:10FA20009B07F9D4637803B9490241F23003C4F269
:10FA30000B0341F234021C681C60C4F20B0241F259
:10FA40003804136823F4081323F0310343F0805380
:10FA500041F22C05C4F20B0543F00A03C4F20B0477
:10FA6000136023682E684EF6482246F002064FF4D3
:10FA7000805EC2F200022E60C4F20B0E002541F23D
:10FA800008071560C4F20B0741F2040641F20C05A9
:10FA9000CEF8000043F08053C4F20B06C4F20B050D
:10FAA0001120396043F00A03C1F222104FF4813172
:10FAB0003160236028601368002BFCD041F23003D2
:10FAC000C4F20B0300201A6802F003021A60F0BDB2
:10FAD0004FF0FF30704700BF830740F0AD802DE945
:10FAE000F0414EF64C25C2F200052B7813B10320ED
:10FAF000BDE8F08141F22402C4F20B0214461368FF
:10FB0000DF07FCD423689E07F9D46B7803B9490258
:10FB100041F23003C4F20B0341F234021C681C6052
:10FB2000C4F20B0241F23804136823F4081323F0E3
:10FB3000310343F0805341F22C06C4F20B0643F02C
:10FB40000A03C4F20B041360236837684EF6482298
:10FB500047F002074FF4805E3760C2F20002C4F241
:10FB60000B0E41F20807C4F20B0700261660CEF810
:10FB7000000041F2040641F20C00396043F080536A
:10FB8000C4F20B06C4F20B00012143F00A034FF448
:10FB90008137C1F622013760236001601368002BB2
:10FBA000FCD041F23003C4F20B0341F22402196885
:10FBB00001F003011960C4F20B0213685907FCD469
:10FBC00041F2240141F23002C4F20B01C4F20B02F3
:10FBD00041F2340741F2080841F20C0C41F21006E0
:10FBE0008E461446C4F20B07C4F20B08C4F20B0C89
:10FBF000C4F20B060B68DB07FCD4DEF80030980774
:10FC0000F8D43B6843F001033B60136813600020A5
:10FC10006B68C8F80030C0F60250CCF800001368DA
:10FC2000DB07FCD5236803F001032360306810F480
:10FC30000070DFD1BDE8F0814FF0FF30704700BFAA
:10FC4000F0B54FF23466C2F2000683B03368019318
:10FC50004FF44044C4F20204019F0546A4464FF00D
:10FC6000004EFF20236843F480632360C4F82CE037
:10FC70006063E36A002BFCDADCF83830DBB2FF2B80
:10FC800006D033680093009BDB1BB3F5967FE9D366
:10FC90004FF44043C4F202034FF00046186841F0AD
:10FCA000400440F480601860DE6218465C63C36AFA
:10FCB000002BFCDA4FF44044C4F2020418204FF049
:10FCC0000047266822FA00F346F48066DBB226601D
:10FCD000E7626363E36A002BFCDA083810F1080F6F
:10FCE000EFD1002932D008290CBF8721FF214FF422
:10FCF0004043C4F202034FF000401A6842F48062AD
:10FD00001A60D8621A465963D36A002BFCDA4FF4A2
:10FD10004042C4F20202164600274FF00044FF2181
:10FD2000136843F480631360D4625163D36A002B79
:10FD3000FCDAB36BD8B21B06687001D403B0F0BD17
:10FD40000137B7F5807FEBD103B0F0BD9521CEE749
:10FD50002DE9F0414EF660258378C2F20005032BB1
:10FD60002B780F4682B00446164618BF4F02002B70
:10FD70006AD00021207806F067FC3A46112120461F
:10FD8000FFF75EFF60BB4FF23460C2F200004FF439
:10FD9000404103680093C4F20201DDF800808C4604
:10FDA0004FF0004EFF270B6843F480630B60C1F8EF
:10FDB0002CE04F63CA6A4FF44043002AC4F20203A6
:10FDC000F8DADCF83820D2B2FF2A627040F0918075
:10FDD00003680193019BC8EB0303B3F5967FE2D957
:10FDE0002078012106F030FC2B784EF66022C2F21A
:10FDF00000022BB349F27033C1F6FF730020D97AA9
:10FE000010700A46E1B1CC0706D54FF46142CEF23C
:10FE10000002D86910600A46880706D54EF204121F
:10FE2000CEF20002196A1160DA7A510700F1EE8011
:10FE3000120705D54EF20C12CEF200029B6A136037
:10FE4000002002B0BDE8F08149F27033C1F6FF73C3
:10FE50004EF65C22C2F20002D97A126801202870A4
:10FE6000002933D072B6D97A11F0010F08460DD0AF
:10FE70004EF2801CCEF2000CD868DCF800E00EEAEE
:10FE8000000EC3F81CE00846CCF800E089070BD54B
:10FE90004EF2841ECEF2000E1869DEF8001001400A
:10FEA0001962CEF80010D87A41070BD54EF2881EA1
:10FEB000CEF2000E5869DEF8001001405962CEF80B
:10FEC0000010D87A010700F1A98062B61B68D968D2
:10FED00091423FF44EAF44F20100C0F23F000021D6
:10FEE0001860C8F23F0142F08040DA601861196082
:10FEF0003FE7FE2A7FF474AF4FF480604FF6FF7146
:10FF0000C9F20001C8F21F0018608E4659631A46F4
:10FF100059631846596306F5FE77B11CD36A13F08E
:10FF2000F00FFBD0C0F834E0836B01F8013C1B12EA
:10FF300001F8023C02318F42F0D106F5FD7106F561
:10FF40000076B14210D24FF44042C4F2020217468A
:10FF5000D36A13F0F00FFBD0BB6B181201F8020B41
:10FF6000B14201F8013CF3D34FF44043C4F2020321
:10FF70004FF480614FF6FF72C8F21F01C9F2000210
:10FF8000196019465A63CA6A4FF4404312F0F00FE1
:10FF9000C4F20203F7D020789B6B012106F054FBDA
:10FFA0002B784EF66022C2F200025BB349F2703346
:10FFB000C1F6FF730020D97A10700A4611B3C80742
:10FFC00006D54FF46142CEF20002D86910600A46AD
:10FFD0008F0706D54EF20412CEF20002196A1160A4
:10FFE000DA7A560706D54EF20812CEF20002596AA6
:10FFF0001160DA7A150705D54EF20C12CEF2000226
:020000021000EC
:100000009B6A1360012002B0BDE8F0814EF2081235
:10001000CEF20002596A1160DA7A09E74EF28C1EBC
:10002000CEF2000E9869DEF8001001409962CEF819
:1000300000104AE7F0B44FF44046C4F202064FF015
:100040000047336843F4806333603D46F7623446CB
:1000500071633346511C02F20127E26A002AFCDA7E
:100060001A6811F8016C42F480621A60DD625E6306
:10007000E26A002AFCDA1A6811F8026B42F4806224
:10008000B9421A60DD625E63E7D14FF44041C4F2C9
:100090000201CA6A4FF44043002AC4F20203F8DAAC
:1000A0001A684FF0004542F48062FF241A60194636
:1000B000DD625C63CA6A4FF44043002AC4F2020363
:1000C000F8DA1A684FF0004542F48062FF241A60A3
:1000D0001946DD625C63CA6A4FF44043002AC4F2E9
:1000E0000203F8DA1A684FF0004542F48062FF24F8
:1000F0001A601946DD625C63CA6A4FF44043002A05
:10010000C4F20203F8DA9B6BDBB203F01F02437008
:10011000A2F10500B0FA80F04009F0BC704700BFC2
:100120002DE9F041064682B0002900F0AC804EF681
:1001300060258378C2F20005032B2B780C46174606
:1001400018BF4C02002B3FD00021307806F07CFA1B
:10015000224618213046FFF773FD002800F09880F2
:100160003078012106F070FA2B784EF66022C2F248
:1001700000022BB349F27033C1F6FF730020D97A25
:1001800010700A46E1B1CC0706D54FF46142CEF2B9
:100190000002D86910600A46880706D54EF204129C
:1001A000CEF20002196A1160DA7A510700F1A480D8
:1001B000120705D54EF20C12CEF200029B6A1360B4
:1001C000002002B0BDE8F08149F27033C1F6FF7340
:1001D0004EF65C22C2F20002D97A12680120287021
:1001E00000293DD072B6D87A10F0010F01460DD02B
:1001F0004EF2801CCEF2000CD968DCF800E00EEA6A
:10020000010EC3F81CE00146CCF800E080070BD5D6
:100210004EF2841ECEF2000E1869DEF80010014086
:100220001962CEF80010D97A48070BD54EF2881E15
:10023000CEF2000E5869DEF8001001405962CEF887
:100240000010D97A09070AD54EF28C1ECEF2000EA4
:100250009869DEF8001001409962CEF8001062B68D
:100260001B68D96891423FF46FAF44F20100C0F2BD
:100270003F0000211860C8F23F0142F08040DA6080
:100280001861196060E74EF66025C2F2000567E765
:100290003A46FE213046FFF7CDFE00283FF460AF1E
:1002A0004FF23461C2F200014FF440420B680193F7
:1002B000C4F20202DDF8048094464FF0004EFF20A5
:1002C000136843F480631360C2F82CE05063D36A70
:1002D0004FF44044002BC4F20204F8DADCF8387022
:1002E000FFB2FF2F10D00B680093009BC8EB0303F5
:1002F000B3F5167FE4D333E74EF20812CEF20002D4
:10030000596A1160DA7A53E700220D213046FFF76F
:1003100097FC00287FF424AF23684FF0004243F499
:10032000806323602146E2626763CA6A4FF44043F8
:10033000002AC4F20203F8DA9B6B13F0FF047FF487
:100340000FAF3078012106F07FF92B784EF660224E
:10035000C2F2000253B349F27033C1F6FF73147056
:10036000D97A0A4611B3C80706D54FF46142CEF2D6
:100370000002D86910600A468F0706D54EF20412B3
:10038000CEF20002196A1160DA7A560706D54EF2EB
:100390000812CEF20002596A1160DA7A150705D503
:1003A0004EF20C12CEF200029B6A1360012008E7A5
:1003B0004EF65C23C2F2000342F20302C3F60002CF
:1003C0001A6070472DE9F04F837987B0012B0546FD
:1003D000029205D001232B71002007B0BDE8F08FF9
:1003E00042799007F6D553070E4626D5EB68AF69DC
:1003F000BB4200F03781002F00F058812A6A147C3C
:10040000591E09347A1EE14022FA04F4A14200F296
:100410005181002B00F04E81641A05F1080806E0B6
:10042000A968286A00F062FC013C0028D2D042464C
:10043000002CF5D1EF603B4600E0EB68029A002A01
:1004400000F09C8049F2B0324EF670414EF6702BAF
:10045000C1F6FF72C2F20001029F0192C2F2000BCC
:100460000391286A0279013A02EA532212F0FF0945
:10047000C3F3080840F08B80B8F1000F40F087808C
:10048000A968002940F0BE80EB69002B00F0D08005
:10049000AB60C8F50074017C4269A4B2023B8B409A
:1004A0004A44BC4203EB020973D9BCB2B8F1000F55
:1004B00004D1A869EB68834280F086804846012118
:1004C00000F030FA002885D008EB0B03181983429E
:1004D0004ED008F10408321DD844934238BF464537
:1004E00043EA060E2CBF01220022591C1EF0030F06
:1004F00002F00102C1EB000E18BF00220EF101094B
:100500009C46002A6ED0B9F1090F6BD9AEF10302F7
:10051000920801324FEA820AA6F104084FF0000E59
:1005200000940EF1010E58F8044F4CF8044B964518
:10053000F7D3CA45009C06EB0A0C03EB0A0E13D056
:1005400016F8228003F822800EF1010398420BD0A6
:100550009CF801308EF801300EF10203984203D06E
:100560009CF802308EF80230C1F1010108440644C3
:10057000EB683F1B2344EB607FF473AFAA699A4298
:1005800075D26A79AB6142F080026A717BE0AB6838
:100590007FE7B4F5007F89D1019B1B6899452CD07A
:1005A0004EF66C23C2F20003494618680378FE2B0E
:1005B00051D03246FFF7B4FD00283FF40BAF06F5EB
:1005C00000764FF40074D3E700F05EF900283FF4A2
:1005D00001AF039A01991378C1F8009043F0010329
:1005E000137071E7013B721E00F1FF3C12F801EF3E
:1005F00003F801EF9C45F9D1B6E7019A4FF0FF33BC
:100600001360CDE705AA00F071FB00283FF4E5AECA
:10061000286A059B90F820404FF6F872C0F6FF72EA
:100620004FF6F871102C08BF0A469342FFF430AF22
:1006300005F10802012100F0EDF900283FF4CAAEEF
:10064000EB69002B30D16A79AB68EB6162F07F0215
:100650006A71286A1DE73046FFF73EFAB0FA80F06B
:100660004009A9E7029900297FF4ECAE0BE04EF6B1
:100670006423C2F200036A791B6823B1029B13B1A1
:1006800042F080026A7111070AD5AB79002B3FF462
:10069000A1AE120611D400F0F7F800283FF49AAE8C
:1006A000029807B0BDE8F08FAB68D2E7AF60EF60AB
:1006B0003B46C3E6EB69AB60AFE60121286900F079
:1006C00031F900283FF486AE4EF670232C7DC2F23D
:1006D000000313EB44143FF47DAEAB794EF6642275
:1006E000012B9CBFAB69E361C2F20002EB691268A7
:1006F00063831B0CA38232B104F1160104F11800CC
:100700009047238B63826B7903F07F036B71C2E7A1
:1007100000B583B002AB012203F8011D1946FFF7B3
:1007200051FE03B05DF804FB2DE9F84F90F820303E
:10073000C66949F2B038102B05460F469146C1F6FE
:10074000FF7822D006EBD116D8F800108E422FD1B8
:100750004EF67044C2F200044EF6702307F07F0795
:10076000C2F2000343F8279023782A7E43F0010366
:10077000012A237054D9AA684EF66823C2F20003F6
:10078000114419600120BDE8F88F06EB1126D8F856
:100790000010B1420CD14EF67044C2F200044EF685
:1007A0007023FFB2C2F20003314623F81790DBE753
:1007B0004EF67044C2F200044EF66C2A2378C2F260
:1007C000000AA3B9DAF800000378FE2B2BD04EF60E
:1007D0007022C2F200023146FFF7BAFAE8B195F88A
:1007E0002030C8F80060102BD9D03146B4E7DAF8D1
:1007F00000000378FE2B32D04EF67022C2F20002C7
:10080000FFF78EFC48B14EF6682BC2F2000BDBF806
:10081000001099B900232370D4E70020BDE8F88FB9
:100820000120BDE8F88F4EF67020C2F2000031467C
:10083000FFF7E2F8B0FA80F04009CFE7DAF80000FD
:100840000378FE2B15D04EF67022C2F20002FFF79D
:1008500067FC0028E1D00023CBF80030DAE74EF641
:100860007020C2F20000FFF737F9B0FA80F04009BB
:10087000C8E74EF67020C2F20000FFF72DF9B0FA7B
:1008800080F04009E5E700BF70B54EF67044C2F253
:10089000000423780BB9012070BD4EF66C25C2F21E
:1008A000000549F2B03328680278C1F6FF73FE2ACA
:1008B000196820D04EF67022C2F20002FFF730FC19
:1008C000B8B14EF66826C2F20006316819B90023A5
:1008D0002370012070BD28680378FE2B15D04EF6DA
:1008E0007022C2F20002FFF71BFC10B1002333603C
:1008F000EDE7002070BD4EF67020C2F20000FFF759
:10090000EBF8B0FA80F04009DAE74EF67020C2F258
:100910000000FFF7E1F8B0FA80F040090028E5D1C7
:10092000E7E700BF2DE9F84349F2B035C1F6FF759E
:1009300088462B68834218D04EF67044C2F20004F9
:100940004EF66C2722780646C2F20007C2B9386814
:100950000378FE2B38D04EF67022C2F200023146E8
:10096000FFF7F6F910B32E6003E04EF67044C2F2C2
:100970000004217848EA010121700120BDE8F883D4
:1009800038680278FE2A14D04EF670221946C2F258
:100990000002FFF7C5FB48B14EF66829C2F2000914
:1009A000D9F80010D9B900232370D0E70020BDE8A2
:1009B000F8834EF670201946C2F20000FFF78CF85B
:1009C000B0FA80F04009E6E74EF67020C2F200006F
:1009D0003146FFF711F8B0FA80F04009C2E73868F5
:1009E0000378FE2B0BD04EF67022C2F20002FFF706
:1009F00097FB0028DAD00023C9F80030D3E74EF681
:100A00007020C2F20000FFF767F8B0FA80F04009EA
:100A1000EFE700BF2DE9F04F136889B0002B00F01D
:100A2000AF8003F1010A00230693C3685E1CB04641
:100A3000002B44D05446A04538BF022401910592B2
:100A40004EF670234EF670424EF66C21C2F2000351
:100A5000C2F20002C2F2000138BFA246B44205460B
:100A6000029203914FF00007994628D895F820305C
:100A7000EE6949F2B03B102BC1F6FF7B2BD0DBF8BF
:100A8000001006EBD416B1422BD104F07F034EF6D2
:100A9000702659F82330C2F2000623F0704393B158
:100AA0000134A246EE680137BE4208D9A04538BFDE
:100AB000022406F1010638BFA246B442D6D900206E
:100AC00009B0BDE8F08F631C0199CAEB03029142A3
:100AD00073D01C46E6E7DBF8001006EB1426B142A3
:100AE00019D0029B1B78F3B94EF66C23C2F20003B7
:100AF00018680378FE2B38D04EF67022C2F200023E
:100B00003146FFF725F90028D9D095F82030CBF8E9
:100B10000060102BB9D1E3B24EF6702639F81330CD
:100B2000C2F20006BBE7039B186802784EF66C23FE
:100B3000C2F20003FE2A049300F0A6804EF6702253
:100B4000C2F20002FFF7ECFA049B0028B7D04EF681
:100B50006822C2F2000204921168D1B902991868A1
:100B600000220A700378FE2BC6D14EF67020C2F226
:100B700000003146FEF740FFB0FA80F04009C2E7BE
:100B8000A1F10103B3FA83F35B09D0F800A0069347
:100B90004BE7039A079310680278FE2A00F09B80C7
:100BA0004EF67022C2F20002FFF7BAFA079B002845
:100BB00085D0049900220A60D0E7012C7FF67FAF30
:100BC000EB6801339C423FF67AAF6FF070422146EA
:100BD0002846FFF7A9FD00283FF471AFA2455ED279
:100BE00004F1FF38B8F1010F7FF669AFEB6801330C
:100BF0004345FFF464AF4EF668234EF67049C2F2E7
:100C00000003C2F2000901932EE007EBD817BA42A5
:100C10000AD000213846FFF785FE00283FF44FAF89
:100C200095F82020102A2AD008F07F0246F82240AA
:100C300099F80020297E42F00102012989F800205C
:100C400003D9AA68019B17441F60C24527D008F149
:100C5000FF38B8F1010F3FF432AFEA680132904536
:100C600004F1FF343FF62BAF95F82020EF69102AEE
:100C7000DBF80020C9D107EB1827BA42C9D15FFAC7
:100C800088F226F81240D3E74EF67020C2F2000038
:100C9000FEF722FFB0FA80F04009049B55E7059B60
:100CA000196871B101297FF60AAFEB6801339942E7
:100CB0003FF605AF52462846FFF736FD00283FF4C1
:100CC000FEAE059BC3F800A0069B13B10AF1010319
:100CD0002B600120F4E64EF67020C2F20000FEF711
:100CE000FBFEB0FA80F04009079B60E72DE9F84F62
:100CF000C36801338B423DD390F82030C46949F278
:100D0000B038102B17460E460546C1F6FF7813D0B3
:100D100004EBD114D8F800108C4213D14EF6702396
:100D200006F07F01C2F20003012053F8213023F0C6
:100D300070433B60BDE8F88F04EB1124D8F8001035
:100D4000A14220D04EF6704AC2F2000A4EF66C293B
:100D50009AF80030C2F2000903BBD9F8000003780A
:100D6000FE2B3FD04EF67022C2F200022146FEF763
:100D7000EFFF10B90020BDE8F88F95F82030C8F8D3
:100D80000040102BCAD14EF67023F1B2C2F200031C
:100D9000012033F811303B60BDE8F88FD9F800002E
:100DA0000378FE2B12D04EF67022C2F20002FFF73B
:100DB000B7F90028DED04EF6682BC2F2000BDBF844
:100DC0000010E1B900238AF80030C6E74EF6702023
:100DD000C2F20000FEF780FEB0FA80F04009002861
:100DE000E9D1C7E74EF67020C2F200002146FEF7B7
:100DF00003FEB0FA80F040090028BED1BAE7D9F866
:100E000000000378FE2B0BD04EF67022C2F20002D7
:100E1000FFF786F90028ADD00023CBF80030D1E7EA
:100E20004EF67020C2F20000FEF756FEB0FA80F0D7
:100E30004009EFE790F8392090F83800101A704711
:100E400090F8383090F839209A4205D95A1C03445A
:100E500080F83820187E70474FF0FF30704700BF91
:100E600090F8383090F839209A4286BF1B18187EC7
:100E70004FF0FF30704700BF704700BF38B50546E0
:100E8000B0F85E0090B195F85D301446C3F12102D0
:100E900094420CD805F13B001844224604F0CEFEE3
:100EA00095F85D30234485F85D30204638BD01203B
:100EB00014462871EEE700BFB0F85E306BB190F8D1
:100EC0005D30202B07D8C218013380F85D30012037
:100ED00082F83B107047012303710020704700BF68
:100EE0000023426980F8383080F8393080F85C306F
:100EF00080F85D3080F85E3080F85F3006CA30B42C
:100F00000D68046943662A4383660A60A3704169D9
:100F100090F861300C680B4440F224121D7A5B7B20
:100F2000C0F20F0202EBC5051B026D6803F4E0631B
:100F300043F064032B6090F862300B449D7CDB7DB2
:100F400002EBC5021B02526803F4E06343F0640342
:100F5000136022684B681A4205D003692C225A702C
:100F6000036904229A71036920225A71036980225D
:100F70009A7030BC704700BF2DE9F0474FF23467DC
:100F8000C2F2000782B03B68009340F22419DDF8FA
:100F9000008002690646C0F20F0900214FF49675E1
:100FA000D3789B065BD53B680193019BC8EB030399
:100FB0000F2BF5D949B1102BF2D000209070336976
:100FC00080229A7002B0BDE8F087726996F86130AD
:100FD00013440521187A05F06BFB726996F86130AD
:100FE0001344012193F812A0504605F061FB092437
:100FF0000021504605F028FB2B46013BFDD1012185
:10100000504605F021FB2B46013BFDD1013CEFD1C1
:10101000706996F8611001444FF416720C7A4B7B9C
:1010200009EBC4011B02496803F4E06343F0640365
:101030000B6096F862300344997CDB7D09EBC101BB
:101040001B02496803F4E06343F064030B60013A58
:10105000FDD13269D3789B064FF00101A3D4012062
:1010600002B0BDE8F08700BFF0B503691222DA7064
:101070000269937803F0200385B004460D46002BE7
:1010800061D0B42393704FF23461C2F2000122693F
:101090000B680093009E05E00B680193019B9B1B6E
:1010A000042B42D8D37803F0200303F0FF00002B79
:1010B000F2D094F85D30002B31D04FF0000E4FF09D
:1010C000020C04EB0E0393F83B3013710B6803938F
:1010D000039F206907E09B060DD50B680293029BD6
:1010E000DB1B052B28D8C378DBB203F0020202F029
:1010F000FF06002AEFD080F803C02669F378DBB240
:10110000DF0632462DD49F062BD5DB0731D40EF1F6
:10111000010E94F85D305FFA8EFE7345D1D8002041
:101120001DBB002384F85E3004E0907023698022A8
:101130009A70042005B0F0BD8670236980220420D7
:101140009A7005B0F0BD03F0FF06FFF715FF10B968
:10115000042005B0F0BD236984F85F60B0229A7066
:1011600091E78023B3700420DAE726698023B37007
:10117000D7E7BEF1000F0CBF02200320F6E700BF47
:101180002DE9F04306690024122780F8384080F8E2
:101190003940F770D0F810E09EF8024004F02004C7
:1011A00089B00546884616461F46002C48D0B42311
:1011B0008EF802304FF23464C2F200042A692368C8
:1011C0000093009905E0236801930198401A0428D0
:1011D0002DD8D07800F0200000F0FF090028F2D0D0
:1011E0004FEA480343F00103DBB213712368029313
:1011F00002982A6905E0236803930399091A0529CF
:1012000015D8D17801F0020101F0FF090029F2D0D0
:101210000220D0702B6993F8039019F011091BD1AB
:10122000FEB9002F0CBFA02280229A7004E082F841
:1012300002902B6980229A70484609B0BDE8F0837D
:1012400004F0FF09FFF798FE0028F5D02B6985F818
:101250005F90B0229A70ADE780229A704FF000093B
:10126000EAE7012E76D0A0229A7029690B79CE4642
:101270004FF0A80C23680493049A05E023680593B3
:10128000059B9B1A052B4CD8CB7803F0020303F087
:10129000FF08002BF2D0C8702969CB78DBB213F0BD
:1012A000100F0A465CD19B065AD5013EF6B2012EBC
:1012B0004BD0BEF11F0F3DD90B79012EDAD1236837
:1012C0000693069805E023680793079B1B1A052BD6
:1012D00055D8D37803F0020303F0FF01002BF2D0BE
:1012E0000223D3702A69D378DBB2D9063AD49B069D
:1012F00036D5B0239370BEF11F0F2B6941D805EB93
:101300000E02197911760EF1010E5FFA8EFE00BF02
:1013100000BF00BF0FB180229A7085F839E0F14616
:101320008AE781F802802B6980229A70F14685F85D
:1013300039E081E705EB0E0391F8048083F818800B
:101340000EF1010E5FFA8EFEB7E781F802C029693F
:101350000A46AEE7A8229A702A69CE461379AEE70C
:10136000F14669E710214FF49673D170013BFDD12E
:101370002A69937803F0F703F14693705CE7917064
:10138000D1E71A79C3E700BF38B549F22044C1F666
:10139000FF742269D578EDB2E9062BD51023D370FE
:1013A0006B0626D505F0040505F0FF03002D6CD073
:1013B0004EF67143C2F20003616E002249F22045ED
:1013C0001A7084F85D20C1F6FF75002974D0884733
:1013D00095F85D30002B6FD02369D0229A70236975
:1013E00094F83B201A712369012284F85C200222C0
:1013F000DA7038BD05F0400303F0FF00002BD1D1B7
:101400009379DBB203F0600160295CD0937803F03C
:10141000100303F0FF01D3B115F0010545D194F895
:101420005C1094F85D0049F220438842C1F6FF73D6
:1014300055D95818013190F83B0083F85C101071B1
:101440002369D0229A7023690222DA70D1E784F8E6
:101450006010937943F020039371236994F8390065
:10146000197949F220421F28C9B2C1F6FF72BED8CD
:101470004EF67144C2F200042478002CB7D0141840
:101480000130217682F83900B1E7226984F83930D9
:10149000C023937023694EF67142C2F2000219799B
:1014A000012111700222DA70A3E7C023937023692F
:1014B0001A790222DA709CE70122002384F85D2069
:1014C00084F83B3088E703F0DF039371A36E23B108
:1014D00084F8380094F839009847226996E7157126
:1014E000AEE700BF38B549F28C44C1F6FF742269FB
:1014F000D578EDB2E9062BD51023D3706B0626D52F
:1015000005F0040505F0FF03002D6CD04EF6714385
:10151000C2F20003616E002249F28C451A7084F811
:101520005D20C1F6FF75002974D0884795F85D30BD
:10153000002B6FD02369D0229A70236994F83B2046
:101540001A712369012284F85C200222DA7038BD06
:1015500005F0400303F0FF00002BD1D19379DBB2FB
:1015600003F0600160295CD0937803F0100303F06E
:10157000FF01D3B115F0010545D194F85C1094F842
:101580005D0049F28C438842C1F6FF7355D9581863
:10159000013190F83B0083F85C1010712369D02270
:1015A0009A7023690222DA70D1E784F86010937987
:1015B00043F020039371236994F83900197949F2B3
:1015C0008C421F28C9B2C1F6FF72BED84EF67144D4
:1015D000C2F200042478002CB7D014180130217610
:1015E00082F83900B1E7226984F83930C02393705A
:1015F00023694EF67142C2F200021979012111707D
:101600000222DA70A3E7C023937023691A790222B9
:10161000DA709CE70122002384F85D2084F83B30D7
:1016200088E703F0DF039371A36E23B184F83800D9
:1016300094F839009847226996E71571AEE700BF24
:1016400038B549F2B434C1F6FF742269D578EDB2E9
:10165000E9062BD51023D3706B0626D505F00405BB
:1016600005F0FF03002D6CD04EF67143C2F200036B
:10167000616E002249F2B4351A7084F85D20C1F61B
:10168000FF75002974D0884795F85D30002B6FD026
:101690002369D0229A70236994F83B201A71236938
:1016A000012284F85C200222DA7038BD05F0400384
:1016B00003F0FF00002BD1D19379DBB203F060017E
:1016C00060295CD0937803F0100303F0FF01D3B1DD
:1016D00015F0010545D194F85C1094F85D0049F2CD
:1016E000B4338842C1F6FF7355D95818013190F8C8
:1016F0003B0083F85C1010712369D0229A70236933
:101700000222DA70D1E784F86010937943F0200365
:101710009371236994F83900197949F2B4321F287A
:10172000C9B2C1F6FF72BED84EF67144C2F20004CF
:101730002478002CB7D014180130217682F83900B3
:10174000B1E7226984F83930C023937023694EF6DB
:101750007142C2F200021979012111700222DA707D
:10176000A3E7C023937023691A790222DA709CE7F9
:101770000122002384F85D2084F83B3088E703F0E1
:10178000DF039371A36E23B184F8380094F8390015
:101790009847226996E71571AEE700BF30B440F272
:1017A0006805C0F20F05417100210560C272037324
:1017B00001718172417330BC704700BF38B549F286
:1017C00020444379C1F6FF7401255B00082242736F
:1017D00084F83B3084F85E5084F85D50417B2046AD
:1017E000FFF76AFB29462046BDE83840FFF73CBCBE
:1017F0002DE9F84349F220444379C1F6FF740125ED
:101800005B0084F83B3084F85E5084F85D50437B85
:1018100001F0F00949EA050806460F01204648EAAA
:101820000301FFF749FB29462046FFF71DFC7379AA
:1018300084F85E50AB4084F83B3084F85D50717B97
:1018400041F0050149EA01012046FFF735FB4FF061
:101850003C0929462046FFF707FCFFB24B46013BF7
:10186000FDD1737984F85E50AB4084F83B3084F846
:101870005D50717B204648EA0101FFF71DFB40F6F1
:10188000B83829462046FFF7EFFB4346013BFDD120
:10189000737984F85E50AB4084F83B3084F85D5037
:1018A000717B294339432046FFF706FB2946204632
:1018B000FFF7DAFB737984F85E50AB4084F83B3075
:1018C00084F85D50717B41F0050139432046FFF7F4
:1018D000F3FA29462046FFF7C7FBB9F10109FCD10D
:1018E000737984F85E50AB4084F83B3084F85D50E7
:1018F000717B294339432046FFF7DEFA294620460B
:10190000FFF7B2FBB8F10108FCD12846BDE8F88327
:101910002DE9F84349F220444379C1F6FF740125CB
:101920005B0084F83B3084F85E5084F85D500F46CD
:10193000417B07F0F008064648EA01012046FFF720
:10194000BBFA29462046FFF78FFB737984F85E5077
:10195000AB4084F83B3084F85D50717B41F004016A
:1019600048EA01012046FFF7A7FA4FF03C09294653
:1019700020463F01FFF778FBFFB24B46013BFDD10C
:10198000737984F85E50AB4084F83B3084F85D5046
:10199000717B204648EA0101FFF78EFA40F6B8381D
:1019A00029462046FFF760FB4346013BFDD1737992
:1019B00084F85E50AB4084F83B3084F85D50717B16
:1019C00020463943FFF778FA29462046FFF74CFBBB
:1019D000737984F85E50AB4084F83B3084F85D50F6
:1019E000717B41F0040139432046FFF765FA29462F
:1019F0002046FFF739FBB9F10109FCD1737984F86E
:101A00005E50AB4084F83B3084F85D50717B2046DB
:101A10003943FFF751FA29462046FFF725FBB8F175
:101A20000108FCD1BDE8F883F0B540F27803C0F2BC
:101A30000F03144606460F460FCB85B0757A0DF19D
:101A4000100E0EE90F00A5423CBF05F1FF34E4B2D1
:101A500004AB03EB8404304654F8101C394461F0A5
:101A60007F01C9B205B0BDE8F040FFF751BF00BF2C
:101A7000C17901F0FD01C17141F00801FFF748BFD4
:101A8000C17901F0FE01C17141F00801FFF740BFCB
:101A90002DE9F04F01F00701C90083B041F040018A
:101AA00092460546FFF734FF41F2F17349F22044B4
:101AB0000AF10702C0F201030AF1FF3B0092019311
:101AC000C1F6FF7401264FF03C09ACE06A7984F856
:101AD0005E60520084F83B2084F85D6095F80DE06C
:101AE00001F0F00A4AF0010849F220400F01C1F666
:101AF000FF7048EA0E01FFF7DFF949F220400121AB
:101B0000C1F6FF70FFF7B0FA697984F85E604900AA
:101B100084F83B1084F85D60697B49F2204041F015
:101B200005014AEA0101C1F6FF70FFF7C5F949F264
:101B300020400121C1F6FF70FFF796FAFFB24A4636
:101B4000013AFDD16A7984F85E60520084F83B2046
:101B500084F85D60697B49F2204048EA0101C1F6E2
:101B6000FF70FFF7A9F949F22040012140F6B8388B
:101B7000C1F6FF70FFF778FA4246013AFDD16A7963
:101B800084F85E60520084F83B2084F85D60697BD5
:101B900049F2204041F001013943C1F6FF70FFF7DF
:101BA0008BF949F220400121C1F6FF70FFF75CFA82
:101BB0006A7984F85E60520084F83B2084F85D60A6
:101BC000697B49F2204041F005013943C1F6FF70BD
:101BD000FFF772F949F220400121C1F6FF70FFF7CB
:101BE00043FA4A46013AFDD16A7984F85E605200B0
:101BF00084F83B2084F85D60697B49F2204041F025
:101C000001013943C1F6FF70FFF756F949F2204050
:101C10000121C1F6FF70FFF727FAB8F10108FCD1E6
:101C2000009B5B450CD02A68019B12681BF8011FC2
:101C30009A423FF44BAF28469047009B5B45F2D158
:101C400003B0BDE8F08F00BF10B501210446FFF7D7
:101C50005FFE4DF2C043C0F20103013BFDD1A37A08
:101C600003B910BD20468021BDE81040FFF750BEEB
:101C7000012A2DE9F843064603D9817941F008018C
:101C80008171727213B1012A00F04D81322004F08B
:101C900073FD49F220447379717BC1F6FF7401250D
:101CA0005B0084F83B3084F85E5084F85D50737BB1
:101CB00020461943FFF700F929462046FFF7D4F9DB
:101CC0004FF47A7004F058FD737984F85E50AB409D
:101CD00084F83B3084F85D50717B204641F0300140
:101CE000FFF7EAF829462046FFF7BEF9737984F832
:101CF0005E50AB4084F83B3084F85D50717B2046E9
:101D000041F03401FFF7D8F84FF03C08294620464F
:101D1000FFF7AAF94346013BFDD1737984F85E5081
:101D2000AB4084F83B3084F85D50717B204641F035
:101D30003001FFF7C1F840F6B83729462046FFF7D3
:101D400093F93B46013BFDD141F6B069C0F204096D
:101D50004B46013BFDD1737984F85E50AB4084F86B
:101D60003B3084F85D50717B204641F03001FFF735
:101D7000A3F829462046FFF777F9737984F85E5077
:101D8000AB4084F83B3084F85D50717B204641F0D5
:101D90003401FFF791F829462046FFF765F94346DD
:101DA000013BFDD1737984F85E50AB4084F83B3041
:101DB00084F85D50717B204641F03001FFF77CF8DC
:101DC00029462046FFF750F93B46013BFDD1B9F1CA
:101DD0000109FCD1737984F85E50AB4084F83B3044
:101DE00084F85D50717B204641F03001FFF764F8C4
:101DF00029462046FFF738F9737984F85E50AB40E6
:101E000084F83B3084F85D50717B204641F034010A
:101E1000FFF752F829462046FFF726F94346013BD3
:101E2000FDD1737984F85E50AB4084F83B3084F880
